:020000040000FA
:100000000002040000000000589E0000589E0000FE
:10001000589E0000589E0000589E0000589E000008
:10002000589E0000589E0000589E0000589E0000F8
:10003000589E0000589E0000589E0000589E0000E8
:10004000589E0000589E0000589E0000589E0000D8
:10005000589E00008A710000B0710000589E000098
:10006000589E0000589E0000589E0000589E0000B8
:10007000589E0000589E0000589E0000589E0000A8
:10008000589E0000589E0000589E0000589E000098
:10009000589E0000589E0000589E0000589E000088
:1000A000589E0000589E0000589E0000589E000078
:1000B000589E0000589E0000589E0000589E000068
:1000C000589E0000589E0000589E0000589E000058
:1000D000589E0000589E0000589E0000589E000048
:1000E000589E0000589E0000589E0000589E000038
:1000F000589E0000589E0000589E0000589E000028
:10010000589E0000589E0000589E0000589E000017
:10011000589E0000589E0000589E0000589E000007
:10012000589E0000589E0000589E0000589E0000F7
:10013000589E0000589E0000589E0000589E0000E7
:10014000589E0000589E0000589E0000589E0000D7
:10015000589E0000589E0000589E0000589E0000C7
:10016000589E0000589E0000589E0000589E0000B7
:10017000589E0000589E0000589E0000589E0000A7
:10018000589E0000589E0000589E0000589E000097
:10019000589E0000589E0000589E0000589E000087
:1001A000589E0000589E0000589E0000589E000077
:1001B000589E0000589E0000589E0000589E000067
:1001C000589E0000589E0000589E0000589E000057
:1001D000589E0000589E0000589E0000589E000047
:1001E000589E0000589E0000589E0000589E000037
:1001F000589E0000589E0000589E0000589E000027
:10020000FFFFFF00FFFFFF00589E0000589E000008
:10021000589E0000589E0000589E0000589E000006
:10022000589E0000589E0000589E0000589E0000F6
:10023000589E0000589E0000589E0000589E0000E6
:10024000589E0000589E0000589E0000589E0000D6
:10025000589E00008A710000B0710000589E000096
:10026000589E0000589E0000589E0000589E0000B6
:10027000589E0000589E0000589E0000589E0000A6
:10028000589E0000589E0000589E0000589E000096
:10029000589E0000589E0000589E0000589E000086
:1002A000589E0000589E0000589E0000589E000076
:1002B000589E0000589E0000589E0000589E000066
:1002C000589E0000589E0000589E0000589E000056
:1002D000589E0000589E0000589E0000589E000046
:1002E000589E0000589E0000589E0000589E000036
:1002F000589E0000589E0000589E0000589E000026
:10030000589E0000589E0000589E0000589E000015
:10031000589E0000589E0000589E0000589E000005
:10032000589E0000589E0000589E0000589E0000F5
:10033000589E0000589E0000589E0000589E0000E5
:10034000589E0000589E0000589E0000589E0000D5
:10035000589E0000589E0000589E0000589E0000C5
:10036000589E0000589E0000589E0000589E0000B5
:10037000589E0000589E0000589E0000589E0000A5
:10038000589E0000589E0000589E0000589E000095
:10039000589E0000589E0000589E0000589E000085
:1003A000589E0000589E0000589E0000589E000075
:1003B000589E0000589E0000589E0000589E000065
:1003C000589E0000589E0000589E0000589E000055
:1003D000589E0000589E0000589E0000589E000045
:1003E000589E0000589E0000589E0000589E000035
:1003F000589E0000589E0000589E0000589E000025
:100400008F272200007F22000001880000000000EA
:100410000C00070060FC280001002000110007000C
:10042000000020000000E000020032000000020096
:1004300000000000DE9D0200000000000040DA0025
:100440000000FE004440A900002F20000000E00052
:100450000300320000002000A00188004440A800F2
:100460000000060091018800800078000000EB0089
:1004700015003700E280400032A0B4009101BA00BC
:10048000E280400032A0B4009102BA00E280400055
:1004900032A0B4000002EB00472BDE00F507B200EB
:1004A000602CE10004003A000059EB008301E900F0
:1004B000FDFF3E00040037006128E100010032002A
:1004C0000082EB00040007001101BA000200E00006
:1004D000E8FF3A00000006003159BA008301E90044
:1004E0000C0032002159BA008301E90008003200F3
:1004F0000400E00003003A00E280400032A0B400B3
:10050000F5FF370011D9BA008301E900FAFF3A007C
:100510008100E800E180400032A0B4000000060045
:1005200000000000000000000000000000000000CB
:1005300000000000000000000000000000000000BB
:1005400000000000000000000000000000000000AB
:10055000000000000000000000000000000000009B
:1007E0000000000000000000889FBE008A9FBE003D
:1007F000010578000100E0000400350008003C001D
:100800000000E0002000320005003700600010000A
:10081000E080180002003B0001F02C001A003700B5
:100820000004BE006011B8006B0920000982CF00EF
:10083000020039000882CF000441B0006942520032
:100840000E00320008003B008281710061016400EB
:100850008904D1000884D3008B05E8000442E80035
:10086000F9FF3A00050037000804440089844C0071
:100870008B05E9000442E900FBFF3A002C01070068
:100880000AF0A70001F0A0004F05BE004F04BE0013
:1008900000000600F4FF2F004B0137001400200079
:1008A00049013700889FBE008A9FBE008C1F7800D8
:1008B000600107006701330003866C006450E100AB
:1008C0002E0032006420E100330032006150E1006C
:1008D0002F0032006120E100310032008585550093
:1008E000EB07B000090020000804200005003700D5
:1008F0000804440089844C000A00310006034300C8
:1009000087834B000001530081815B00F8FF3300B7
:100910000203BE000800A0000804440089844C00C3
:10092000F6FF3900C639DD00830173000100320093
:10093000130020008904D1000884D3000998A30083
:10094000050032000800A7000300A0008904D100C0
:100950000884D3008B05E8008904D1000884D30003
:100960000001EB000281D200F100070001F0A100BC
:100970000CF0A70001F0A0003F0137006420E10067
:10098000410132000801BE000200BE00F7FF37003F
:100990006120E1003C0132006000B800F3FF370045
:1009A0000000200001F82700F0FF370003F0A2004C
:1009B000889FBE008A9FBE008C1F78001D01070023
:1009C000240133006450E1004F0032006420E10054
:1009D0005200320003826C0007003B000905D00082
:1009E0000306D000820F54000C065D00020039009F
:1009F00002003200890178000306780085825500E4
:100A000004003D000003FD008103FD008502EA00B3
:100A10008B854200840F720002003B0060001000D2
:100A2000E08018006011B8000005EB007A28E100B2
:100A30000A00390006007800C75DDD00F707B20044
:100A4000878075002D003700828171000A017800CF
:100A5000610560008180D1000080D3008502E9003B
:100A6000F9FF3B00060440008784480002003B0079
:100A700060041400E0841C000988A3000700320011
:100A80008A81710082817100610164008904D10052
:100A90000884D3008B05E800170037000978A3000D
:100AA00013003A000B00E000130034008B05E9004E
:100AB0000804440089844C000A4474000978A300A7
:100AC0000D003A000B00E000070034008B05E90040
:100AD0000804440089844C0001003A000B00200007
:100AE0000978A300F7FF32000001EB000200370095
:100AF000828171000A0178008D0007000CF0A700C8
:100B000001F0A000DC0037006420E10002003A00A0
:100B1000838F6C00DC0033000801BE000200BE00C1
:100B2000D5003700889FBE008A9FBE008C1F7800CA
:100B3000C0000700C700330003866C006450E1006A
:100B4000240032006420E100270032006150E100FF
:100B5000220032006120E100210032008B8542003A
:100B6000EB07B1000134B800003AB80008044200B5
:100B700089844A00013AB8000030B80088804000FB
:100B800009014A0004003300000040008180480051
:100B9000020149008B05E900C909DD0083017000ED
:100BA0000100320013002000C814DE004814DD00EC
:100BB0004709DE001200B200C808DE000884700099
:100BC0005B00070001F0A1000CF0A70001F0A000FD
:100BD000A90037006120E100AB0032000801BE002F
:100BE0000200BE00F7FF37006150E100FCFF3A0051
:100BF000A50037000001BE00A60007000470A70092
:100C000003F0A10003F8A30013003A006509B10046
:100C100010003200090035006928E10002003500AB
:100C2000010028000000050000004000818048000D
:100C30008502E900FCFF3A0000000600F88F420040
:100C4000050035008100D1000080D3008502E80056
:100C5000FCFF3A00000006008000EB0000000500E9
:100C60006022B800060220000000D0008180D2007F
:100C70000482D2008582D2000000A000020252004D
:100C800083825A00030031000202420083824A003C
:100C90000000A1000603E900F3FF3A00000006008F
:100CA000EFFF07000400BE00000006000001BE00C8
:100CB000780007000470A70003F0A1006509B100E7
:100CC000160032000D0035006828E10006003500EE
:100CD000F0FF2F00F1FF27000300E00013003B00AE
:100CE000010028000000050000004000818048004D
:100CF0008502E900FCFF3A0008003700F88F420047
:100D000002003C008000EB00000005008100D100E3
:100D10000080D3008502E800FCFF3A000300E000F9
:100D200002003B0060001000E08018000000060098
:100D300081002000618055000B003D000B00200069
:100D400061FE2F000100E1001D003400828171006E
:100D5000610164008904D1000884D3000000E80028
:100D6000FAFF3A0071002000610064000300700087
:100D7000020060000900320061044400E0844C007D
:100D80000988A500050032008B05E8006808E1002D
:100D900002003A008904D1000884D300F20F200039
:100DA0000258E10005003D00C75DDD00F907B20013
:100DB0008980750008007800000006000BF8270005
:100DC0008B00780000000500889FBE008A9FBE004F
:100DD000841F7800170007004F00780011003300CF
:100DE000F0FF2F00838F6C0006003B0004056500B8
:100DF0000A00A7000800370009F0A6001000200034
:100E000008003700820F5400838F5C000300390014
:100E10001000200001003E000000200009F0A700A3
:100E20000000EA004F05BE004F04BE000000E000D5
:100E3000000006000004BE00160007000003BE000C
:100E40000405BE000200BE0012000700844F7500BA
:100E5000000006000200BE006450E10005003600FC
:100E60006420E100020036000968A30001003A0096
:100E70000800BE000160A0004F0678004F05BE00CC
:100E80004F04BE0000000600F0FF2F00F1FF270016
:100E9000F9FF3700C70ADE00F107B200F50FB20014
:100EA00008003200E1CF4200020032000170A000D1
:100EB00024000500810F70000100320004080500C5
:100EC00044000500810F700002003A001400050084
:100ED0008502E9000000400081C04800FCFF3B00A3
:100EE0000170A00024000500005E0000BCE20000CC
:100EF000613F0000DD830000C29C00007E200000F6
:100F0000A3FD00001F4100009DC30000217F0000E1
:100F1000FCA20000401E00005F010000E3BD0000D5
:100F20003E60000082DC0000237D00009FC10000C5
:100F3000421C0000FEA00000E1BF00005D030000B5
:100F400080DE00003C620000BEE00000025C0000A9
:100F5000DF810000633D00007C220000C09E000095
:100F60001D430000A1FF000046180000FAA4000085
:100F7000277900009BC5000084DA00003866000075
:100F8000E5BB000059070000DB8500006739000061
:100F9000BAE400000658000019470000A5FB000055
:100FA00078260000C49A0000653B0000D987000045
:100FB000045A0000B8E60000A7F900001B45000035
:100FC000C69800007A240000F8A60000441A000029
:100FD00099C70000257B00003A64000086D8000015
:100FE0005B050000E7B900008CD20000306E000005
:100FF000EDB30000510F00004E100000F2AC0000F5
:101000002F71000093CD0000114F0000ADF30000E0
:10101000702E0000CC920000D38D00006F310000D4
:10102000B2EC00000E500000AFF10000134D0000C4
:10103000CE900000722C00006D330000D18F0000B4
:101040000C520000B0EE0000326C00008ED00000A8
:10105000530D0000EFB10000F0AE00004C12000094
:1010600091CF00002D730000CA9400007628000084
:10107000ABF500001749000008560000B4EA000074
:1010800069370000D58B000057090000EBB5000060
:10109000366800008AD4000095CB00002977000054
:1010A000F4AA000048160000E9B70000550B000044
:1010B00088D60000346A00002B75000097C9000034
:1010C0004A140000F6A80000742A0000C896000028
:1010D000154B0000A9F70000B6E800000A54000014
:1010E000D78900006B3500004C450000540000001B
:1010F0004946000000540000484500004E00000032
:10110000454C000053450000004700004F540000CC
:101110004F000000474F0000535500004200000000
:101120005245000054550000524E0000005200008D
:10113000454D000000500000524900004E54000090
:10114000004900004E5000005554000000460000C9
:101150004F520000005400004F0000004E450000B8
:1011600058540000005200004541000044000000B7
:10117000444100005441000000530000544100006D
:10118000525400000053000054410000525400002B
:1011900052000000535400004F5000000053000064
:1011A000544F00005052000000530000454E000014
:1011B000440000005245000043450000495600002D
:1011C00045000000434C00004B000000444100007B
:1011D0005400000042490000545200004541000004
:1011E000440000004144000043000000415500005D
:1011F00058000000505300005500000050550000FA
:101200004C4C0000555000000041000055580000B3
:10121000504900004E0000004652000045510000B9
:1012200000440000555400005900000044450000EF
:101230004C410000590000004D41000043520000A5
:101240004F000000454E0000440000000052000026
:10125000554E0000004C00004953000054000000AF
:101260004558000049540000004400004542000079
:1012700055470000004E00004557000000000000E8
:101280003E200000000800002008000000000000D0
:10129000203D00002000000056520000454700009D
:1012A000207400006F6F0000206C00006F7700005A
:1012B0002C200000697300002074000068650000A5
:1012C000726500002061000020730000686F00005C
:1012D000727400003F0000002E2000003C0000005F
:1012E0003E0000002E200000000D00000A28000033
:1012F000002900003E20000000420000757300003D
:101300002050000069720000617400006520000038
:10131000763100006100000046690000726D000037
:10132000776100007265000020760000352E000015
:1013300036200000287200003437000033290000F6
:1013400020000000202800000041000033000000C1
:101350004234000000420000350000004238000026
:10136000005500004E4B000000290000004900001D
:10137000090000004F0900000048000009000000BB
:101380004C090000004500006E740000657200000A
:10139000207200006177000020760000616C000080
:1013A00075650000206600006F720000204200009A
:1013B00052470000000000003062000000300000D2
:1013C000303000002C000000303000000030000001
:1013D0003132000033340000353600003738000069
:1013E00039410000424300004445000046300000FF
:1013F00078000000436F0000756C0000646E000010
:1014000027740000206B000065650000702000005C
:1014100075700000000000005350000049310000CA
:10142000000000000029000000200000570000001C
:10143000205200000049000032430000310000004B
:101440003A200000000000002E000000315700008C
:10145000303100000000000008080000080800000B
:101460000800000000000000204800007A00000092
:101470000000000000410000525400003100000054
:1014800042420000494F000031000000524100007C
:101490005731000000000000314100004C530000B3
:1014A000000000004F430000443100000000000035
:1014B0000000000000000000290000000000000003
:1014C00000000000000000001A00FA000000EB001D
:1014D000100F98000000EB00506988000000EB003E
:1014E000406988000000EB00A04088000000EB008D
:1014F000606988000000EB00100798000000EB0016
:1015000040079800140037000000EB002007980007
:101510000B0037004E009000AE0090004500DD004B
:1015200081004000E0D22000808040000040EB00BD
:10153000804878002E0090000000E8002007980006
:101540002E009000FF0F5000F2FF34004E0090007C
:101550000000E800400798004E009000E40F5000A3
:10156000E9FF34000000EB00706E8800A1408000AD
:10157000E00220000088B900610220008080400065
:10158000E093200000804000D66C020000000000C4
:10159000D140800000202000008060000000E000BA
:1015A0000400320071002000C0592000EE990200B2
:1015B0000000000000942800D66C0200000000002B
:1015C000ED003700706E80000000E0006300320024
:1015D000706E80000000E900706E88000000EB0073
:1015E000200798001E00370042698000706E80005E
:1015F000AE0090004500DD0081004000E0D22000F8
:10160000008040009040780080C22000000041002F
:1016100001487800706E8000AE0090004500DD004B
:1016200081004000E0D2200000804000104078009F
:101630003271020000000000406980000000E800F4
:10164000406988002E0090000000E8002007980004
:1016500041698000F00F2000008060004069880030
:10166000706E8000AE0090004500DD0081004000FB
:10167000E0D2200000804000104078000004E0002C
:10168000D9FF3A000000EB00706E8800330037008D
:1016900080B8200010407800624060000004E00044
:1016A0002E003200A1408000E00220000088B90036
:1016B000FA004000E0932000008040001000780015
:1016C000000001000000E00024003200A140800082
:1016D000E00220000088B900610220008080400004
:1016E000E093200000804000D66C02000000000063
:1016F00000942800D66C02000000000051698000B0
:1017000040698000808F50001400320050698000D2
:10171000200798000D003700AE00900080C2200026
:10172000008040001040780032710200000000008C
:10173000AE009000F00F20000080600020079800AD
:101740002E0090000000E80020079800AE009000F6
:1017500040698000808F5000EFFF3A001471020052
:10176000000000000004E000C9FF32002071020008
:1017700000000000604798006E4090000080FB0071
:10178000200F98002E089000E80F50001100320042
:10179000AE089000E88F500007003C002E09900032
:1017A0000200E0003C003200AE099000E28F5100E0
:1017B000440032004B0037002E089000EA0F500022
:1017C00013003200AE089000ED8F50001000320080
:1017D000440037004169800050698000808F5000CC
:1017E00065003200406980000000E900406988001F
:1017F00041698000F00F200000806000406988008F
:1018000030942800D66C0200000000005A00370017
:1018100010002000100F9800406980008000E80050
:10182000F00F20008080600050698000808F5000A1
:101830000D0032004169800080C22000808040009D
:101840000040EB0080487800406980000000E8001C
:101850004069880041698000F00F2000008060002E
:10186000406988000800370070C0B3003271020080
:10187000000000004169800080C22000808040009C
:101880000040EB008048780070942800026D020050
:1018900000000000380037001E0090000000E80043
:1018A000100798001E009000F40F500032003A001C
:1018B0004E770200000000000000EB0010079800C7
:1018C0002D0037001E009000E40F50002A00340065
:1018D000B6860200000000000000EB001007980030
:1018E00025003700406980008000E800F00F2000EC
:1018F0008080600050698000808F500016003200A8
:101900006E409000FF4F50001B0036006E4090006C
:101910000004E000180035006E40900032710200B3
:1019200000000000416980006E41900080C22000EC
:101930000080400002487800406980000000E80014
:101940004069880041698000F00F2000008060003D
:10195000406988000800370070C0B300327102008F
:10196000000000004169800080C2200080804000AB
:101970000040EB00804878001E0890000000E00066
:1019800010FF3200406980007007980050698000A5
:10199000600798000000EB00100F98000000EB00BB
:1019A000000F98000000EB0060698800D1408000C3
:1019B00000202000008060000000E000B104320040
:1019C000603002000000000051002000305A20006A
:1019D000789A02000000000010002000000F98001C
:1019E000A80437005169800080C2200000804000B8
:1019F00010407800604798006E4090000080FB0027
:101A00006101B900320F9800430F9800D007200001
:101A1000010020003E099000CE099000800F510087
:101A2000818F590069043E003E089000CE08900066
:101A30000060010067043700640437006304370066
:101A40006204370061043700600437005F04370028
:101A50005E0437005D0437005C0437005D04370026
:101A60005A043700590437005A0437005704370026
:101A70005604370055043700540437005304370028
:101A80005204370051043700500437004F04370028
:101A90004E0437004D0437004C0437004B04370028
:101AA0004A04370049043700480437004704370028
:101AB0004604370047043700240437009B023700F0
:101AC000EE003700FB003700AA013700980137000D
:101AD0003E043700720237003C0437003B043700F5
:101AE0003C0437003B043700D0033700E9033700DC
:101AF000B40337001503370014033700130337000E
:101B00001203370011033700100337000F033700AB
:101B10000E0337000D0337000C0337002B0437008A
:101B20002A043700B3013700950037002704370037
:101B3000460037000D013700FF003700230437004F
:101B40006B00370077013700200437001F0437008F
:101B50001E0437001D0437001C0437001B04370027
:101B60001A0437006C0037001804370017043700D8
:101B70001604370015043700140437001304370027
:101B80009101370011043700100437000F043700AB
:101B90000C0137000D0437000C0437000B0437002C
:101BA000C602370094033700D6023700C803370057
:101BB000AB03370005043700D20037002E00370092
:101BC000410037004901370000043700300037007A
:101BD00032003700150037001F003700FB033700C5
:101BE000FA0337005900370021003700F7033700A8
:101BF00023003700F5033700F403370033033700C1
:101C00006D013700F1033700F00337001E00370085
:101C100022013700ED033700EC033700EB033700F8
:101C2000AF02370073003700BF023700A406070079
:101C30000000E000E7033A00506980006007980068
:101C40004069800070079800E20337008E9A020016
:101C500000000000DF033700F9070700A040800004
:101C60000000E000DB03320057080700D90337000B
:101C70000B060700D70337007D090700D50337009F
:101C800055090700D3033700C9080700D1033700FF
:101C9000A274020000000000CE033700A0408000C4
:101CA0000000E00005003A00D1012000305D200076
:101CB000789A020000000000C60337000673020095
:101CC00000000000C303370080B8200010407800F7
:101CD0000000A10081B82000804878006101200048
:101CE000805A2000789A020000000000B9033700F3
:101CF00080B82000104078000000A00081B82000CB
:101D00008048780051012000E05B2000789A0200B2
:101D100000000000AF03370080B8200010407800BA
:101D20000020A00081B8200080487800C101200078
:101D3000B07E2000EE9902000000000070942800A0
:101D4000026D020000000000A203370080B82000EE
:101D5000104078000020A10081B820008048780061
:101D6000B1012000007D2000EE990200000000007B
:101D700070942800026D02000000000095033700F7
:101D8000506980000000E8005069880051698000B7
:101D9000F00F20000080600050698800AE05070049
:101DA000C2030700200798002E009000D06F0200A9
:101DB0000000000080942800D66C020000000000A3
:101DC0002E0090006E6F020000000000809428003A
:101DD000D66C0200000000002E009000366D02005C
:101DE0000000000070942800026D02000000000056
:101DF00078033700506980000000E80050698800CF
:101E000051698000F00F2000008060005069880058
:101E100091050700A5030700200798002E009000F9
:101E2000AE970200000000000080FB002007980031
:101E30002E009000D06F0200000000008094280067
:101E4000D66C0200000000002E0090006E6F0200B1
:101E50000000000080942800D66C02000000000002
:101E60002E009000366D02000000000070942800E3
:101E7000026D020000000000560337001E9B0200A6
:101E8000000000000000E00052033200510020007A
:101E900030632000789A02000000000023C2BF00D7
:101EA000614060000004E000FCFF32000000FE0022
:101EB000480337001E9B0200000000000000E00005
:101EC00044033200A100200080632000789A0200C1
:101ED00000000000400620004C97020000000000B7
:101EE000BE9502000000000023C2BF0061406000F8
:101EF0000004E000FCFF320081BF2A000140010025
:101F0000340337000E0507000000E8004007980082
:101F100002003700E0750200000000004E00900053
:101F20000000E900400798004E0090000000E0002B
:101F3000F8FF3A0027033700010507000000E8001A
:101F40004007980002003700BE7502000000000044
:101F50004E0090000000E900400798004E009000FD
:101F60000000E000F8FF3A001A033700F40407000D
:101F70000000E800400798000B00370061012000D6
:101F800020642000EE9902000000000002760200AA
:101F900000000000C06C02000000000070942800E7
:101FA000026D0200000000004E0090000000E900F9
:101FB000400798004E0090000000E000EFFF3A005C
:101FC00004033700A04080000000E00005003A0054
:101FD000D1012000305D2000789A0200000000004E
:101FE000FC023700C082A900C282A800C8A2A900D2
:101FF000CAA2A80021E3A800200020004C970200FC
:1020000000000000A0C0B3000E9602000000000017
:1020100080007800001B2000808F50000F003600E9
:1020200090C0B3000E96020000000000800078000F
:10203000702B2000808F5000080036001101200016
:1020400080652000EE9902000000000070942800D6
:10205000026D0200000000000E003700C082A900DF
:10206000C282A900C8A2A900CAA2A900C0942800DF
:10207000026D020000000000210120009066200097
:10208000EE9902000000000070942800026D02002A
:102090000000000021E3A900CE023700A04080002C
:1020A0000000E00005003A00D1012000305D200072
:1020B000789A020000000000C6023700C082A90022
:1020C000C282A900C8A2A900CAA2A90021012000B9
:1020D00090662000EE990200000000007094280035
:1020E000026D020000000000BA023700F10020007B
:1020F000A0392000EE99020000000000289602009E
:102100000000000011002000903A2000EE9902002B
:102110000000000070942800026D02000000000022
:10212000AC0237003A96020000000000A902370016
:1021300083040700400798006100200070682000B9
:10214000EE990200000000004E009000106F0200A7
:102150000000000021002000D0682000789A0200D2
:10216000000000004E009000789702000000000080
:1021700098023700720407004007980061002000B1
:1021800070682000EE990200000000004E009000F0
:10219000106F0200000000002100200090EC2000E1
:1021A000789A0200000000004E0090004C97020058
:1021B0000000000087023700D04080000090A0009F
:1021C000D040880083023700A04080000000E0007B
:1021D00005003A00D1012000305D2000789A02000D
:1021E000000000007B02370036760200000000008D
:1021F000780237001000200060698800100020007D
:102200002007980010003700516980002E009000D0
:1022100080804000F00F20008080600080C220009D
:102220000080400090407800E0C3B30080CF5000B1
:1022300002003A000000EB00606988002E00900068
:102240000000E80020079800516980002E009000EF
:1022500080804000F00F20008080600080C220005D
:1022600000804000104078000004E000E6FF3A00E3
:10227000AE00900020022000808F50000200340049
:102280001000200060698800606980000000E000A4
:1022900050023A00506980000000E8005069880050
:1022A00051698000F00F20000080600050698800B4
:1022B0007E0207002007980051698000F00F20007F
:1022C0008080600080C22000008040009040780044
:1022D000D0C3B30080CF500044003A002E009000DD
:1022E0000000E0003E0034002E009000E50F50009A
:1022F0003B003C00506980000000E8005069880005
:1023000051698000F00F2000008060005069880053
:102310002E0090000000E900200798000000EB006C
:10232000400798000B0037002E009000CE00900070
:102330004500DD0081004000E0D2200080804000A8
:102340000040EB00804878004E0090000000E8005C
:10235000400798004E009000FF0F5000F2FF34003D
:102360000000EB004007980015003700AE01900018
:102370004E0290005169800080C220000080400021
:10238000104178004518DD0084004000E0D22000B4
:1023900000804000024878004E0090000000E800F5
:1023A00040079800506980000000E80050698800EC
:1023B00051698000F00F20000080600050698800A3
:1023C0005169800080C22000008040009040780069
:1023D000E0C3B30080CF5000E4FF3A00FD013700B6
:1023E0001000200060698800FA0137002E0090007C
:1023F0000000E0001B003A000000EB0040079800DE
:10240000140037004E0090000040E8006E6F02009C
:1024100000000000C0962800D66C020000000000FA
:102420004E0090004500DD0080007800E0D22000E2
:1024300000804000D66C02000000000000972800D9
:10244000026D0200000000004E0090000000E80055
:10245000400798004E009000E40F5000E9FF340060
:10246000DC0137002E0090000000E000090034007D
:102470002E009000E50F500006003C0070942800EC
:10248000026D020000000000AE009000716E880036
:10249000D00137001000200060698800CD013700AE
:1024A000506980000000E800506988005169800090
:1024B000F00F20000080600050698800FB010700D9
:1024C00050079800E403070051698000F00F2000D6
:1024D0008080600080C22000008040009040780032
:1024E00090C2B30080CF50000D003A00A1408000A0
:1024F000E00220000088B900FC004000E0932000CA
:1025000000804000900078005E0090000100010013
:1025100070942800026D020000000000AD01370039
:102520001000200060698800AA0137001000200018
:102530006069880010002000200798001000370014
:10254000516980002E00900080804000F00F200034
:102550008080600080C220000080400090407800B1
:1025600020C2B30080CF500002003A000000EB0010
:10257000606988002E0090000000E80020079800A5
:10258000516980002E00900080804000F00F2000F4
:102590008080600080C220000080400010407800F1
:1025A0000004E000E6FF3A00606980000000E000FF
:1025B00088013A0071002000F0682000EE990200C6
:1025C0000000000020C2B3003271020000000000D1
:1025D0002300370051698000F00F20000080600068
:1025E000506988005169800080C22000008040004E
:1025F0001040780032710200000000005169800034
:1026000080C2200000804000104078000000FB00E5
:102610005007980080B820001040780064406000A7
:102620000004E000050032005E009000AE9702005A
:10263000000000000080FB0050079800A1408000CF
:10264000E00220000088B900E8004000E09320008C
:1026500000804000900078005E00900001000100C2
:10266000506980000000E8005069880051698000CE
:10267000F00F20008080600080C2200000804000B9
:102680009040780020C2B30080CF5000D1FF3A00C4
:1026900050698000F10F200001006000506988003F
:1026A00020C2B300327102000000000070942800C4
:1026B000026D02000000000046013700A1408000CA
:1026C000E00220000088B90080007800E09320003C
:1026D0000080400010007800000001003D0137003C
:1026E000A1408000E00220000088B9008080E8005E
:1026F000E0932000008040001000780000000100FE
:1027000034013700A1408000E00220000088B900B9
:10271000E4004000E09320000080400010007800BA
:10272000000001002B013700A1408000E0022000E2
:102730000088B900E6004000E093200000804000DF
:102740001000780000000100220137007100200015
:10275000F0682000EE99020000000000530107001D
:1027600050079800506980000000E9005069880017
:1027700051698000F00F20000080600050698800DF
:10278000EF0207000000E800400798000F03070071
:10279000000F78001E00E000420032001E007800AA
:1027A0008040780070B72000014878003D00370075
:1027B0005E009000C69602000000000070B7200086
:1027C00010407800E84F500007003200B0C3B3005B
:1027D000327102000000000070B720001040780045
:1027E0006E6F02000000000080B8200010407800EA
:1027F000644060000004E000050032005E009000CC
:10280000AE970200000000000080FB005007980017
:10281000A1408000E00220000088B900E8004000EC
:10282000E093200000804000900078005E0090005F
:10283000010001002007980000C2B30032710200BD
:1028400000000000AE009000F00F2000808F5000CC
:1028500014003C006100200060692000EE99020035
:102860000000000080B82000104078006440600044
:102870000004E000050032002E009000AE97020038
:10288000000000000080FB00200798002E00900050
:10289000C69602000000000000C2B30032710200C0
:1028A000000000004E0090000000E9004007980082
:1028B0004E0090000000E000BDFF3A007094280038
:1028C000026D020000000000C2003700610020001D
:1028D00060692000EE9902000000000098020700E5
:1028E0000000E80040079800B8020700000F7800D9
:1028F0001E00E000290032001E00780080407800B1
:1029000070B720000148780024003700A140800003
:10291000E00220000088B900EA004000E0932000B7
:10292000008040001000780000000100604798001F
:1029300080B8200010407800644060000004E0008F
:10294000040032006E409000AE97020000000000CC
:10295000604798006E4090000080FB00C696020021
:102960000000000070B7200010407800E84F5000D1
:1029700007003200B0C3B300327102000000000053
:1029800070B72000104078006E6F02000000000059
:1029900000C2B30032710200000000004E0090003F
:1029A0000000E900400798004E0090000000E000A1
:1029B000D6FF3A0070942800026D0200000000006B
:1029C0008400370081002000C0692000789A02004E
:1029D00000000000A1408000E00220000088B90053
:1029E000EC004000E09320000080400010007800E0
:1029F000000001007700370081002000406A2000BD
:102A0000789A020000000000A1408000E00220004F
:102A10000088B900EE004000E093200000804000F4
:102A200010007800000001006A003700E10020007B
:102A3000C06A2000789A020000000000A1408000D7
:102A4000E00220000088B900F0004000E093200080
:102A50000080400010007800000001005D00370099
:102A6000E1002000A06B2000789A02000000000026
:102A7000A1408000E00220000088B900F200400080
:102A8000E09320000080400010007800000001006A
:102A900050003700C1002000B0672000EE9902000E
:102AA00000000000A1408000E00220000088B90082
:102AB000F4004000E0932000008040001000780007
:102AC00000000100C06C020000000000410037005F
:102AD0001B02070040079800D1002000806D2000F5
:102AE000EE990200000000004E009000C696020021
:102AF000000000004E0090000000E8004007980031
:102B000008003700A1408000E00220000088B900E2
:102B1000F6004000E09320000080400010007800A4
:102B2000000001004E0090000000E90040079800FE
:102B30004E0090000000E000F2FF3A007094280080
:102B4000026D02000000000022003700FC010700B7
:102B50000000E80040079800A1002000506E20000F
:102B6000EE990200000000000D003700A140800037
:102B7000E00220000088B900F8004000E093200047
:102B8000008040001000780000000100C06C0200CE
:102B90000000000000C2B30032710200000000001B
:102BA0004E0090000000E900400798004E009000A1
:102BB0000000E000EDFF3A0001012000806C2000E1
:102BC000789A020000000000020037001000200088
:102BD00060698800506980000000E8005069880042
:102BE00051698000F00F200000806000506988006B
:102BF000606980000000E0001C00320051012000EC
:102C0000F06E2000EE99020000000000EE0090003F
:102C100050698000808F50000700310050698000AB
:102C2000804078006E00900000C050006E6F02007F
:102C300000000000060037005069800080407800E6
:102C40006E00900000C050006E6F02000000000097
:102C50000000EB006069880010002000000F980061
:102C600070942800026D020000000000516980008D
:102C700040698000808F500002003A001000200060
:102C8000000F98000E0890000000E00055FB320095
:102C90007E009000506988007E00900040698800A6
:102CA0000000EB00100F980030FA37000600FA0021
:102CB0000000EB00100798000000EB00000F780008
:102CC000516980001E00900080804000F00F2000BD
:102CD0008080600080C2200000804000904078002A
:102CE00000C3B30080CF500043003400516980001E
:102CF0001E00900080804000F00F20008080600067
:102D000080C22000008040009040780090C3B30053
:102D100080CF500038003C00516980001E009000B8
:102D200080804000F00F20008080600080C2200082
:102D300000804000104078008000FB0000FD2F0064
:102D4000008F40001E0090000000E800100798006F
:102D5000120037001E0078006A00B900000F7800EA
:102D6000516980001E00900080804000F00F20001C
:102D70008080600080C22000008040001040780009
:102D80000000FB009E00400000FD2F00008F40006F
:102D90001E0090000000E8001007980051698000B4
:102DA0001E00900080804000F00F200080806000B6
:102DB00080C220000080400090407800F0C2B30044
:102DC00080CF500051013400516980001E009000F6
:102DD00080804000F00F20008080600080C22000D2
:102DE000008040009040780090C3B30080CF500036
:102DF000D8FF340045013700516980001E00900063
:102E000080804000F00F20008080600080C22000A1
:102E1000008040009040780000C3B30080CF500095
:102E200035013A001E0090000000E80010079800ED
:102E3000516980001E00900080804000F00F20004B
:102E40008080600080C220000080400090407800B8
:102E500020C6B30080CF50000B00320051698000C3
:102E60001E00900080804000F00F200080806000F5
:102E700080C22000008040009040780020C4B30051
:102E800080CF50002D003A001E0090000000E800A6
:102E900010079800120037001E0078000000400064
:102EA000000F7800516980001E0090008080400073
:102EB000F00F20008080600080C220000080400071
:102EC000104078000000FB009E00400000FD2F0035
:102ED000008F40001E0090000000E80010079800DE
:102EE000516980001E00900080804000F00F20009B
:102EF0008080600080C22000008040009040780008
:102F000010C3B30080CF5000E3FF3200516980004E
:102F10001E00900080804000F00F20008080600044
:102F200080C22000008040009040780000C3B300C1
:102F300080CF5000D8FF3200F40037005169800084
:102F40001E00900080804000F00F20008080600014
:102F500080C22000008040009040780080C7B3000D
:102F600080CF50000B003200516980001E0090009D
:102F700080804000F00F20008080600080C2200030
:102F8000008040009040780080C5B30080CF5000A2
:102F90008E003A001E0090000000E8001007980024
:102FA000470037001E0078004400DD00000F780065
:102FB000516980001E00900080804000F00F2000CA
:102FC0008080600080C22000008040009040780037
:102FD000F0C2B30080CF5000180034005169800067
:102FE0001E00900080804000F00F20008080600074
:102FF00080C22000008040009040780090C3B30061
:1030000080CF50000D003C00516980001E009000F0
:1030100080804000F00F20008080600080C220008F
:1030200000804000104078000000FB009E0040003F
:1030300000FD2F00008F40001E0037005169800006
:103040001E00900080804000F00F20000081600092
:10305000516980001E00900080804000F00F200029
:103060008080600080C22000008040009040780096
:1030700000C2B30080C0700080C220000000410088
:1030800001487800516980001E0090008080400057
:10309000F00F20008080600080C22000008040008F
:1030A000104078000000FB009E00400090FA2F00C6
:1030B000008F40001E0090000000E80010079800FC
:1030C000516980001E00900080804000F00F2000B9
:1030D0008080600080C22000008040009040780026
:1030E000F0C2B30080CF50000B0034005169800063
:1030F0001E00900080804000F00F20008080600063
:1031000080C22000008040009040780090C3B3004F
:1031100080CF5000A3FF3400516980001E00900052
:1031200080804000F00F20008080600080C220007E
:10313000008040009040780000C4B30080CF500071
:103140000B003400516980001E0090008080400018
:10315000F00F20008080600080C2200000804000CE
:103160009040780060C4B30080CF50008DFF3400E1
:10317000516980001E00900080804000F00F200008
:103180008080600080C22000008040009040780075
:1031900000C6B30080CF50005C003400516980004D
:1031A0001E00900080804000F00F200080806000B2
:1031B00080C22000008040009040780060C6B300CC
:1031C00080CF500077FF34005000370051698000F5
:1031D0001E00900080804000F00F20008080600082
:1031E00080C220000080400090407800F0C2B30010
:1031F00080CF500045003400516980001E009000CF
:1032000080804000F00F20008080600080C220009D
:10321000008040009040780090C3B30080CF500001
:103220003A003C00516980001E0090008080400000
:10323000F00F20008080600080C2200000804000ED
:10324000104078008000FB0000FD2F00008F400040
:10325000120037001E0078006A00B900000F7800E5
:10326000516980001E00900080804000F00F200017
:103270008080600080C22000008040001040780004
:103280000000FB009E00400000FD2F00008F40006A
:103290001E0090000000E8001007980051698000AF
:1032A0001E00900080804000F00F200080806000B1
:1032B00080C220000080400090407800F0C2B3003F
:1032C00080CF500011003400516980001E00900032
:1032D00080804000F00F20008080600080C22000CD
:1032E000008040009040780090C3B30080CF500031
:1032F000D8FF340005003700100020006069880006
:103300000000EB00200798000A0037005169800098
:103310001E009000008040005069880051698000C4
:10332000F00F200000806000506988001E007800C7
:10333000200798002E0090000080FA000000060090
:103340000400FA00506980008000E800F00F2000BF
:103350008080600080C220000080400090407800A3
:10336000A0C3B30080CF500013003A005069800022
:103370000080E8005069880051698000F00F20004B
:10338000008060005069880048FE0700000F780048
:10339000506980000000E900506988005169800090
:1033A000F00F200000806000506988001E00780047
:1033B0001007980002003700100020001007980046
:1033C0001E0090000080FA00000006000400FA00D1
:1033D000506980008000E800F00F200080806000CD
:1033E00080C220000080400090407800B0C3B3004D
:1033F00080CF500013003A00506980000080E80040
:103400005069880051698000F00F20000080600042
:103410005069880025FE0700000F78005069800081
:103420000000E9005069880051698000F00F200019
:1034300000806000506988001E0078001007980026
:10344000020037000000EB00100798001E009000FB
:103450000080FA00000006000000FA0007003700B4
:10346000506980000000E8005069880051698000C0
:10347000F00F2000008060005069880051698000D2
:1034800080C22000008040009040780000C2B3005D
:1034900080CF5000F2FF32000080FA0000000600EA
:1034A0000400FA000000EB00000F78005069800073
:1034B0000000E8005069880051698000F00F20008A
:1034C0000080600050698800E3FF0700F7FD0700F7
:1034D000000F78001E00E0004D003A000000EB00F5
:1034E00010079800130037001E0090000040E8000D
:1034F0006E6F02000000000020972800D66C0200CA
:10350000000000009E009000E00220000088B9004A
:103510006102200080804000E09320000080400095
:10352000026D0200000000001E0090000000E80094
:10353000100798001E009000E80F5000EAFF3400CA
:103540007101200040702000789A02000000000005
:103550000000EB006069880013002000920020004A
:103560001100200010002000F6000700000FE90005
:10357000E0FF2F009E0F1000030032000080EB00E0
:103580009E0F100005003A00E1002000B0712000FD
:10359000789A02000000000042003700A14080003D
:1035A000E00220000088B900010220008080400075
:1035B000E09320000080400010007800000001002F
:1035C000BE950200000000001E007800A0408800A8
:1035D000A1408000E00220000088B900FE00400009
:1035E000E0932000008040001000780000000100FF
:1035F0001E00E00001003200CA82A8005100200035
:10360000305A2000789A02000000000025003700A0
:103610001E0FE900800020009E0F10001D003C00DE
:10362000A1408000E00220000088B90001022000D3
:1036300080804000E093200000804000100078006F
:1036400000000100BE950200000000001E0078008E
:10365000A0408800A1408000E00220000088B9005E
:10366000FE004000E0932000008040001000780041
:10367000000001001E00E00001003200CA82A80024
:1036800051002000305A2000789A0200000000000B
:10369000040037005101200090722000789A020047
:1036A00000000000406980008000E900F00F200069
:1036B00000806000506988000080FA000000060069
:1036C0002600FA00100020002007980050698000B2
:1036D0000000E900100798009E009000F00F200005
:1036E0000080600010079800430037009E009000A3
:1036F00080C2200000804000104078000004E000FC
:1037000036003A001E0090008000E800F00F200014
:103710008080600080C2200000804000104078005F
:103720000004E0002D0032002E0090006E6F0200B9
:103730000000000020972800D66C02000000000066
:1037400010002000000F78000A0037001E009000D3
:103750009E004000F00F20008080600080C22000AA
:10376000008040001040780032710200000000002C
:103770001E0FE8001E0090009E004000F00F200089
:103780008080600080C220000080400010407800EF
:103790000004E000EDFF3A00AE0190001E00900032
:1037A0008000E800F00F200000816000E600470084
:1037B0000380410002B078002E0090000000E80075
:1037C000200798002E009000EF0F50000E003200EE
:1037D00070942800026D0200000000001E0090009E
:1037E0000000E900100798009E009000F00F2000F4
:1037F00000806000100798009E00900050698000D3
:10380000808F5000B9FF3A0071002000E073200063
:10381000789A020000000000130020002E019000A2
:10382000110020000000EB00460007001007980080
:103830001E009000E10F400003003A00100020003D
:10384000201798003C0037000000EB00200798008C
:1038500016003700416980002E00900080804000F3
:10386000F00F2000008160001E009000E60047007D
:1038700000004000E08078002E0090008080400032
:10388000F00F20008080600080C220000080400097
:103890009040780080C2200000004100014878007C
:1038A0002E0090000000E800200798001E00900005
:1038B000E600470000004000E08078002E00900005
:1038C00080804000F00F20008080600080C22000D7
:1038D00000804000104078000004E000DDFF3A0066
:1038E000406980008000E900F00F20000080600047
:1038F00050698800516980002E00900000804000CF
:103900008080E800F00F200000806000406988009F
:10391000406980008000E900F00F20008080600096
:1039200080C22000808040000040EB00804878008A
:103930000000EB00201798002E1090000080FA0085
:10394000000006001E00FA00100F9800210F9800DA
:10395000320F9800430F98000000EB0040079800DA
:103960000000EB00200798000000EB001007980013
:103970000000EB00000F780050972800D66C020082
:10398000000000001E0890006E6F020000000000A2
:1039900090972800D66C02000000000067003700F6
:1039A0002071020000000000204F98002E48900077
:1039B0000000FB00600F98006E089000ED0F5000B3
:1039C00029003200EE089000ED8F500007003C0007
:1039D0006E099000E80F51000D0032006E08900053
:1039E000EA0F50002000320035003700D0022000DE
:1039F000EE089000808F50001E00320080072000EB
:103A00006E099000800F5100270032002C00370013
:103A10004E0090000000E000070032004E009000D1
:103A20000000E9004007980030942800D66C02009E
:103A300000000000410037001E00E00006003200D8
:103A40000000EB00000F780030942800D66C0200D4
:103A5000000000003900370070C0B300327102006E
:103A600000000000350037001000200020079800FB
:103A7000320037004E0090000000E00006003A00DF
:103A8000D0C2B3003271020000000000100020001C
:103A9000000F78002900370070C0B30032710200B7
:103AA00000000000250037004E0890000000E000F4
:103AB000030032000080EB00500F98005D003700DB
:103AC000AE489000F0C2B30080CF50001800340020
:103AD000AE48900090C3B30080CF500014003C006B
:103AE0004E009000E30F50000600340070C0B30099
:103AF00032710200000000004000200040079800E2
:103B00000E0037002E4890003271020000000000C5
:103B1000CE0090006B0047002E4990008270780024
:103B20004E0090000000E8004007980003003700B6
:103B300070C0B30032710200000000002E0090003F
:103B40000000E00096FF320070942800026D020031
:103B5000000000004E0090000000E00003003A006A
:103B60001E089000500F9800320037000000EB0054
:103B7000100798004E0090000000E90040079800F0
:103B8000CE00900031079800110037001E00900011
:103B90006A00B90010079800BE0090004E00900027
:103BA000808050006B004700614078008000FB007F
:103BB0001E0090008080400000FD2F00008040002B
:103BC000100798004E0090000000E90040079800A0
:103BD0004E0090000000E000ECFF3D009E009000D1
:103BE0002E089000808F50000D0035009E00900040
:103BF0003E089000808F500009003C001E00E0004D
:103C0000040032001E0090000000EA00500F9800EF
:103C1000080037001E019000520F98000500370081
:103C2000B1012000E0EA2000789A020000000000C4
:103C300049FF37005E0890000080FA00000006008F
:103C40000400FA00D0972800026D02000000000076
:103C5000C0982800D66C020000000000D1002000AF
:103C600070802000EE99020000000000A1BF2A0031
:103C70000000EB004A72020000000000000F780014
:103C80001E0078004800DE006E6F02000000000099
:103C9000E0C2B30032710200000000001E00780094
:103CA0006E6F02000000000070942800026D020098
:103CB000000000006100200000762000EE99020064
:103CC00000000000B04080002870020000000000EA
:103CD0007100200070EA2000EE9902000000000050
:103CE000C04080002870020000000000209A2800D8
:103CF000D66C020000000000C04080001007980051
:103D0000200423009E009000808F50001600320097
:103D1000200423009E009000808F500005003E008C
:103D2000300023009E009000808F50000A00320077
:103D300019003700300423009E009000808F50004F
:103D40000D003200600423009E009000808F500020
:103D50000D00320010003700509A2800D66C020087
:103D6000000000000F003700809A2800D66C020087
:103D7000000000000B003700B09A2800D66C02004B
:103D80000000000007003700E09A2800D66C02000F
:103D90000000000003003700109B2800D66C0200D2
:103DA00000000000509B2800026D0200000000008F
:103DB000E101200060762000789A020000000000F7
:103DC0000080FA00000006000000FA005100200008
:103DD00020922000EE99020000000000C1BF2A00DE
:103DE0000000EB004A720200000000002870020090
:103DF000000000006100200070922000EE99020097
:103E000000000000E1BF2A000000EB004A7202003F
:103E100000000000287002000000000070942800DC
:103E2000026D020000000000C10020004078200068
:103E3000789A0200000000005D000700CAC2BF00BF
:103E40000042B2000004E000050032001101200031
:103E500080652000EE990200000000000400370099
:103E60002101200090662000EE9902000000000071
:103E7000C0C2B300327102000000000000C2B300F3
:103E8000327102000000000080B82000104078006D
:103E9000684060000004E0000500320021022000BC
:103EA00000792000789A020000000000040037002A
:103EB000E1012000207B2000789A02000000000031
:103EC00080B8200010407800644060000004E000EA
:103ED00005003A00B1012000007D2000EE990200AB
:103EE0000000000004003700C1012000B07E200067
:103EF000EE99020000000000C0C2B300327102005F
:103F00000000000000C2B300327102000000000097
:103F1000B1012000C0202100EE9902000000000045
:103F200070B72000104078006E6F020000000000A3
:103F300070942800026D02000000000080B820008C
:103F400010407800614060000004E000050032008D
:103F500051012000E05B2000789A02000000000080
:103F60000400370061012000805A2000789A020086
:103F700000000000A1408000E00220000088B9009D
:103F80004102200080804000E0932000008040003B
:103F90001000780000000100C100200040782000DF
:103FA000789A0200000000000080FA00000006007D
:103FB0000000FA00A1002000A0052100789A02006C
:103FC0000000000061042000200B2100789A02000C
:103FD00000000000A101200040062100EE9902002F
:103FE00000000000A1408000E00220000088B9002D
:103FF0002102200080804000E093200000804000EB
:104000001000780000000100A1002000E00721005E
:10401000EE99020000000000004020005000070060
:10402000001020004E000700002020004C00070078
:10403000000420004A000700000820004800070094
:1040400070942800026D0200000000004100200072
:10405000800F2100EE9902000000000021E3A8007B
:10406000A0C0B3000E9602000000000072700200B3
:104070000000000011002000903A2000EE9902009C
:104080000000000090C0B300327102000000000088
:1040900090C0B3000E960200000000007270020093
:1040A0000000000011002000903A2000EE9902006C
:1040B0000000000090C0B300327102000000000058
:1040C000C0C0B3000E960200000000007270020033
:1040D0000000000011002000903A2000EE9902003C
:1040E0000000000090C0B300327102000000000028
:1040F000B0C0B3000E960200000000007270020013
:104100000000000011002000903A2000EE9902000B
:104110000000000090C0B3003271020000000000F7
:1041200021E3A900004020001C000700001020002F
:104130001A000700002020001800070000042000DB
:1041400016000700000820001400070070942800E3
:10415000026D0200000000000080FA00000006006E
:104160000200FA00000F7800401680001E00600078
:104170000000E00004003200709B2800D66C0200B2
:104180000000000003003700A09B2800D66C02004E
:10419000000000000080FA00000006000200FA00A3
:1041A000000F7800501680001E0060000000E00044
:1041B00004003200D09B2800D66C020000000000F2
:1041C00003003700009C2800D66C020000000000AD
:1041D0000080FA00000006000200FA00506980002A
:1041E0000000E8005069880051698000F00F20004D
:1041F000008060005069880097FC0700ABFA070058
:10420000000F78001E00E00006003400400020008F
:104210009E0F100003003C001E00E9009040880043
:104220000D0037000000EB006069880021022000CB
:1042300040812000789A0200000000008001EB001D
:10424000420020001100200010002000BDFD0700EA
:104250000000E900904088002101200060832000D8
:10426000789A0200000000000080FA0000000600BA
:104270000200FA00506980000000E80050698800E0
:1042800051698000F00F20000080600050698800B4
:1042900071FC070085FA0700104798001E40900047
:1042A0000004E000090032001E409000EA4F500078
:1042B00006003E001E4090000040E900804078006B
:1042C00000812000014878000F0037000000EB005B
:1042D00060698800D108200030872000789A0200A9
:1042E000000000008001EB00A2002000110020006F
:1042F0009000200093FD07000040E9008040780016
:1043000000812000014878000081200010407800E2
:10431000E94F500010003A004FFC070063FA070015
:10432000004F78001E04E0000B003A000000EB0094
:1043300060698800309C2800026D020000000000C7
:104340008001EB00F2FF27008000EB00200220003C
:104350007CFD0700004F7800410120000090200004
:10436000789A02000000000011012000B01F210017
:10437000789A02000000000023C2BF006140600084
:104380000004E000FCFF32000081200010407800B3
:10439000E94F500003003A001E40780050710200BF
:1043A00000000000989602000000000000003700A6
:1043B00014710200000000000004E000FCFF320065
:1043C00020710200000000008040780000C2B300AD
:1043D00080CF500001003200F5FF37000080FA0066
:1043E000000006000000FA004173800000E7200092
:1043F000008040009040780030C8B30080CF50006B
:104400000E003A00407380000000E800407388000E
:1044100003003700407380000000E800407388000C
:104420004173800000E72000008040009040780049
:1044300000CEB30080CF5000F6FF36000080FA00B7
:10444000000006000A00FA00300798000000EB00A8
:1044500020079800AE00900000E720000080400098
:104460009040780000CEB30080CF500003003E00A3
:104470000080EB004007980023003700AE0090005A
:1044800000E7200000804000104078008080FB00A2
:1044900000F22F0000804000100798002E009000CE
:1044A0008000E80000E72000008040001040780015
:1044B0000080FB004801DD002E0090008080E800B5
:1044C00000E7200000804000104078000080FB00E2
:1044D000000F41009E0078003E009000808F500049
:1044E00003003A002E0090004007980006003700B5
:1044F0009E0090002E00900000804000630040006D
:1045000020079800D3FF37004E0090000080FA008B
:10451000000006000600FA00881F78000000EB008B
:10452000000F78004173800000E720000080400009
:104530009040780080C2B30080CF500010003A0055
:10454000407380000000E800407388001D010700F0
:10455000000F78004173800000E7200000804000D9
:104560009040780090C2B30080CF5000AA003A007B
:10457000407380000000E80040738800A600370008
:104580004173800000E720000080400090407800E8
:1045900000C4B30080CF5000160036004173800085
:1045A00000E720000080400090407800A0C5B300E4
:1045B00080CF50000F003E004273800000E72000D3
:1045C00000004100104078008080FB00F0FB2F00CD
:1045D000008040008000400080E02000008040001B
:1045E00010007800200798000200E800407388005F
:1045F0008B0037004173800000E7200000804000FE
:104600009040780000C8B30080CF5000740036009E
:104610004173800000E720000080400010407800D7
:104620000080FB00100798000100E800407388003C
:10463000700920009E009000808F500041003200E1
:10464000700920009E009000808F50000D003C00FB
:10465000400920009E009000808F5000160032001C
:10466000600920009E009000808F50002B003200D7
:10467000300920009E009000808F5000180032000A
:1046800046003700900920009E009000808F500067
:104690001E003200900920009E009000808F500084
:1046A00039003500A00920009E009000808F500046
:1046B0002E00320039003700A1408000E0022000C7
:1046C0000088B900EA004000E0932000008040002C
:1046D0001000780000000100000F78004E00370045
:1046E000A1408000E00220000088B900E8004000FE
:1046F000E093200000804000100478008200070052
:1047000008000100000F7800430037000276020025
:1047100000000000000F78003F003700A14080003B
:10472000E00220000088B900F4004000E09320007F
:10473000008040001000780000000100000F7800A9
:1047400035003700A1408000E00220000088B90059
:10475000F8004000E0932000008040001000780046
:1047600000000100000F78002B003700CAC2BF0014
:104770000080FB004500DE00614060000080FB001F
:10478000000F780024003700C0C0B3000E9602006E
:1047900000000000000F78001F0037000000EB0051
:1047A000000F78001C0037001E0078006A00B90076
:1047B000000F78004173800000E720000080400077
:1047C000104078000080FB009E00400000FD2F009C
:1047D000008F4000407380000000E80040738800B4
:1047E0004173800000E72000008040009040780086
:1047F000F0C2B30080CF5000070036004173800044
:1048000000E72000008040009040780090C3B30093
:1048100080CF5000E4FF36001E007800200798008B
:104820002E0090004F0478000080FA00000006007F
:104830000600FA0037FF0700000F7800000037007D
:104840004173800000E72000008040009040780025
:10485000A0C2B30080CF50000A0032004173800034
:1048600000E720000080400090407800F0C2B300D4
:1048700080CF5000030032001E007800200798000F
:104880001E0037004173800000E7200000804000D8
:10489000104078000080FB00100798000100E8003D
:1048A00040738800A00220009E009000808F50007E
:1048B00005003200F00220009E009000808F500022
:1048C00007003200DEFF370012FF0700800078008B
:1048D0001E0078000180B900000F7800D8FF370073
:1048E0000CFF0700000178001E007800110009008D
:1048F0000200D800000F7800D1FF37002E00900092
:104900000080FA00000006000600FA00C8FF070059
:10491000000F7800000037004173800000E720009E
:104920000080400090407800D0C2B30080CF50009B
:104930000A0032004173800000E720000080400040
:1049400090407800B0C2B30080CF50000300320026
:104950001E00780020079800170037004173800080
:1049600000E7200000804000104078000080FB003D
:10497000100798000100E80040738800B002200092
:104980009E009000808F500008003200D00220006E
:104990009E009000808F500001003200DEFF370043
:1049A000A3FF07001E0F1000DBFF3700A0FF07006A
:1049B0001E0F4000D8FF37002E0090000080FA0044
:1049C000000006000C00FA004273800000E720009F
:1049D00000004100104078008080FB00F0FB2F00B9
:1049E000008040008000400080E020000080400007
:1049F00090007800210798000200E80040738800CA
:104A00000000EB00000F78000B0037009E017800DB
:104A10004273800000E72000000041001040780051
:104A20008040780066004700817178000200E8004D
:104A3000407388001E0FE8004173800000E72000EB
:104A4000008040009040780000C4B30080CF500048
:104A5000070036004173800000E72000008040001E
:104A600090407800A0C5B30080CF50000E00360003
:104A70004173800000E720000080400090407800F3
:104A8000F0C2B30080CF5000E0FF360041738000D9
:104A900000E72000008040009040780090C3B30001
:104AA00080CF5000D9FF3E0097FF07001007980005
:104AB00066004700104078000000FB005007980097
:104AC000C0032000DE009000808F500032003200D2
:104AD000C0032000DE009000808F500005003C00E5
:104AE00010022000DE009000808F50004100320054
:104AF0004E003700D0032000DE009000808F500071
:104B000005003200E0032000DE009000808F50009E
:104B10000A003200450037000000EB004007980013
:104B2000AE0090001E009000808F500041003A00BF
:104B300011002000410798003E0037006600470042
:104B400090409000D0C3B30080CF500009003A00DD
:104B50000000EB0040079800AE0090001E0090009F
:104B6000808F50003300350011002000410798006D
:104B7000300037000000EB0040079800AE009000C6
:104B80001E009000808F50002A0034001100200089
:104B900041079800270037006600470090409000CA
:104BA000D0C3B30080CF500009003A000000EB00F2
:104BB00040079800AE0090001E009000808F5000CB
:104BC0001C003C001100200041079800190037002C
:104BD0000000EB0040079800AE0090001E0090001F
:104BE000808F500013003D00110020004107980005
:104BF000100037006600470090409000D0C3B3001B
:104C000080CF500009003A000000EB0040079800F8
:104C1000AE0090001E009000808F50000500320012
:104C20001100200041079800020037000000EB004F
:104C3000400798004E0090000080FA000000060037
:104C40001C00FA00881F78000000EB004073880009
:104C50000000EB00300798000000EB0020079800F0
:104C60000000EB00100798000000EB005073880074
:104C70000000EB00607388000000EB007073880098
:104C80000000EB0050079800D04080000080A0009A
:104C9000D04088000000EB00400798000900370072
:104CA0004E0090008000400080E0200080804000A6
:104CB0000000EB00800878004E0090000000E80043
:104CC000400798004E009000F90F5000F4FF3400A8
:104CD000330437001E0090000000E00021003A007D
:104CE0004173800000E72000008040009040780081
:104CF000F0CDB30080CF500003003E002000200024
:104D000030079800290437004173800000E7200035
:104D100000804000104078008080FB0000F22F00EF
:104D20000080400060079800407380008000E80029
:104D300000E7200000804000104078000080FB0069
:104D40004801DD00407380008080E80000E720001B
:104D500000804000104078000080FB0000007100DF
:104D6000500798000000EB00100798004073800087
:104D7000E300400000E72000008040001040780081
:104D80000080FB006101B90000F82F00F1FF2F0047
:104D90000201400083814800420F9800530F9800A1
:104DA00010022000010020004E099000DE09900052
:104DB000800F5100818F5900ED033E004E08900096
:104DC000DE08900000600100210037003500370048
:104DD000E7033700E6033700710037008100370032
:104DE000A3003700B7003700BE0037003B01370093
:104DF00088013700DE033700EE0137003502370047
:104E000099023700A0023700AE023700BC0237001B
:104E1000CA023700D8023700D50337007A033700BB
:104E20005E033700D2033700D1033700E2023700B8
:104E3000F0023700A1033700AC033700000337004E
:104E40001403370034033700B4033700C5033700B9
:104E5000100020002007980040738000660040008A
:104E600040738800407380008080E90000E72000E4
:104E700000804000104078008080FB00F0FB2F0095
:104E800000844000A0FE0700000178008800440074
:104E900080E02000008040000208780051FD0700FB
:104EA000B5033700100020002007980040738000F1
:104EB0006400400040738800C2FE07000000E0006C
:104EC0001C00320041738000310F980000E7200081
:104ED0003E09900000004100904078008041EB00C6
:104EE0004357980020C8B30080CF500002003A001A
:104EF00010C0B30040579800BE0890000100E800C1
:104F0000407388004E5190000204E0009A03320082
:104F100010002000100798004073800063005000CC
:104F20004073880094033700407380000000E8005D
:104F3000407388004173800000E72000008040003B
:104F40009040780030C8B30080CF50000700320096
:104F50004173800000E7200000804000904078000E
:104F600000CEB30080CF5000EFFF360041738000C9
:104F700000E72000008040009040780030C8B30077
:104F800080CF50007C033A001000200010079800EA
:104F9000407380000080E90040738800760337008A
:104FA000100020002007980040738000640040003B
:104FB0004073880054FE070022FD0700000F7800B0
:104FC0008081EB009E8F1100030032001E007800EC
:104FD00040738800680337006000200030079800A5
:104FE0006503370010002000200798004073800000
:104FF000640040004073880060738000E90F500037
:1050000018003C0062738000417380006E009000C5
:10501000008040008001E90082004100C0E32000E0
:105020000080400003087800607380000000E80002
:105030006073880034FE070002FD0700000F78004F
:105040008080EB009E8F1000030032001E0178006C
:105050004273880048033700600020003007980042
:1050600045033700700020003007980042033700E6
:1050700000892800D66C020000000000100020000B
:1050800020079800607380000000E0000A003200F2
:10509000607380000000E900607388006073800026
:1050A00080004000C0E32000008040001000780035
:1050B00040738800300337008000200030079800DC
:1050C0002D03370010002000200798004173800056
:1050D0006E00900000804000630040004073880034
:1050E000250337001000200020079800407380003F
:1050F000640040004073880057003700417380000F
:1051000000E72000008040009040780020C2B300FB
:1051100080CF50001F003A00407380000000E8007C
:105120004073880010003700D04080000080A1004C
:10513000D04088004173800000E7200000804000DC
:1051400010407800004178000100E80040738800BA
:10515000024078003271020000000000D040800060
:105160000080A000D04088004173800000E720004C
:10517000008040009040780020C2B30080CF5000F3
:10518000E9FF3A00407380000000E80040738800A7
:10519000310037004173800000E7200000804000AC
:1051A0009040780000C4B30080CF50000700360064
:1051B0004173800000E720000080400090407800AC
:1051C000A0C5B30080CF50000D00360041738000B1
:1051D00000E7200000804000104078000004E0005C
:1051E00013003D004173800000E720000080400074
:1051F00090407800F0CDB30080CF50000C003E000E
:10520000C1FD0700000F7800D04080000080A100A1
:10521000D04088001E007800106F020000000000DF
:10522000D04080000080A000D04088000A003700F5
:105230004173800000E7200000804000904078002B
:10524000B0C3B30080CF500003003A004073800029
:105250000000E800407388004173800000E72000F0
:105260000080400090407800F0CDB30080CF500027
:1052700007003E004173800000E7200000804000EE
:105280009040780030C8B30080CF50009BFF3A00B8
:10529000407380008000E90000E7200000804000AB
:1052A00090407800B0C3B30080CF500009003200B6
:1052B000D04080000080A100D0408800609228008B
:1052C000026D020000000000D04080000080A000BD
:1052D000D040880043FC0700A702370010002000E0
:1052E00020079800D04080000080A100D0408800B6
:1052F0004073800064004000407388004173800068
:1053000000E72000008040009040780020C2B300F9
:1053100080CF500018003A00407380000000E80081
:10532000407388000A0037004173800000E72000C6
:105330000080400010407800004178000100E80043
:1053400040738800024078003271020000000000C3
:105350004173800000E7200000804000904078000A
:1053600020C2B30080CF5000EFFF3A0040738000AE
:105370000000E800407388004173800000E72000CF
:105380000080400090407800C0C2B30080CF500041
:1053900004003A00407380000000E8004073880079
:1053A0000200370030002000300798004173800071
:1053B00000E7200000804000104078008080FB0063
:1053C000F0FB2F00008440008001EB00F2FF27007B
:1053D0008000EB000000EB00A21C020000000000B7
:1053E000000178008800440080E020000080400038
:1053F00002087800407380000000E80040738800D5
:10540000F8FB0700D04080000080A000D04088005A
:1054100059023700100020002007980040738000D8
:10542000640040004073880050738000E30F500018
:1054300004003C00507380000000E80050738800B6
:1054400002003700400020003007980052738000AF
:105450004373800000E72000008041001040780086
:105460008080FB0000FC2F00008240006610B90025
:105470008080E80000E520000080400004087800FB
:105480000300E800407388004173800000E72000BB
:105490000080400090407800D0C3B30080CF50001F
:1054A00011003A00407380000000E800407388005B
:1054B000507380006600B9008080E80000E520009D
:1054C00000804000100078000004E9000EFD070095
:1054D000000178008800440080E020000080400047
:1054E00002087800020037003000200030079800E2
:1054F00043738000130F980000E720009E0890007F
:1055000000804000904078000041EB000257980076
:10551000B0C8B30080CF500002003A0013C0B300FF
:10552000035798009E0890000100E800407388002F
:105530000E5190000204E000090032005873800010
:10554000F1FC0700000178006640B900E40040006B
:1055500000E52000008040000208780002003700CB
:1055600030002000300798004173800000E72000E1
:105570000080400090407800F0CDB30080CF500014
:105580000800360050738000427380006600B90046
:105590008000780000E520000080400002087800CC
:1055A0000200370030002000300798008DFB070014
:1055B000F1013700100020002007980040738000A0
:1055C00064004000407388004273800000E72000C0
:1055D00000004100104078008080FB0000FC2F009C
:1055E000008F40000200E800407388005000200057
:1055F000300798000000EB00400798002F003700AC
:105600004E0090006600B9008080E80000E52000B0
:1056100000804000100078009E0F500024003A00E7
:105620001E00E9008000400080E020000080400073
:10563000100178004E0090006600B900E4004000C0
:1056400000E520000080400010007800800F51002D
:1056500012003D009E00E9000181400080E0200032
:1056600000004100100078000001E8008180400047
:1056700080E0200000804000020878004E0090008A
:105680006600B9008000780000E52000008040003E
:1056900010007800407388000300370050738000CA
:1056A0000000E900507388000000EB00300798000C
:1056B0004E0090000000E800400798005173800001
:1056C0004E009000810F5000CDFF340045FB0700D5
:1056D000A9013700100020002007980040738000C7
:1056E0006400400040738800707380000000E00098
:1056F00027003A000000EB00400798000A0037003E
:10570000CE00900000E720000080400010407800AC
:105710008080FB004E0090008080400030F22F001F
:1057200000804000400798004E009000E3004000D9
:1057300000E720000080400090407800E0C8B300FF
:1057400080CF500006003200CE00900000E720001D
:1057500000804000104078000004E000E8FF3A00BC
:10576000CE00900000E7200000804000104078004C
:105770000004E000040032004E009000640040008D
:1057800070738800020037009000200030079800F6
:1057900043738000030F78007073800040738800AB
:1057A0009E00780000E72000008040001040780054
:1057B0008080FB00F0FB2F000084400055FB0700B9
:1057C000000178008800440080E020000080400054
:1057D0000208780040738000707388001E00E800A3
:1057E000407388007173800000E720000080400053
:1057F00090407800C0C2B30080CF500003003A0050
:10580000707380000000E80070738800717380007E
:1058100000E72000008040009040780000CEB300F8
:1058200080CF50000E00360070738000E30040000F
:1058300000E720000080400090407800E0C8B300FE
:1058400080CF5000030032000000EB00707388002E
:10585000030037007073800064004000707388009C
:10586000E0FA0700440137001000200020079800EC
:10587000417380006E009000008040006300400093
:10588000407388003C01370010002000200798007A
:10589000407380006400400040738800A140800095
:1058A000E00220000088B90080007800E09320002A
:1058B000008040001000780000000100C9FA0700D5
:1058C0002D01370010002000200798004073800051
:1058D0006400400040738800A1408000E002200086
:1058E0000088B9008080E800E0932000008040003C
:1058F0001000780000000100BAFA07001E0137000E
:1059000010002000200798004073800064004000D1
:1059100040738800A1408000E00220000088B900A8
:10592000E4004000E0932000008040001000780078
:1059300000000100ABFA07000F0137001000200043
:105940002007980040738000640040004073880086
:10595000A1408000E00220000088B900E60040007D
:10596000E09320000080400010007800000001005B
:105970009CFA070000013700100020002007980063
:10598000407380006400400040738800A1408000A4
:10599000E00220000088B900E8004000E093200009
:1059A0000080400010047800D7FB070008000100C9
:1059B0008CFA0700F0003700100020002007980044
:1059C000407380006400400040738800CEFB0700F5
:1059D0000000E00003003200BE750200000000007D
:1059E00002003700E0750200000000007DFA0700A9
:1059F000E10037001000200020079800407380006D
:105A00006400400040738800BFFB07000000E00016
:105A100005003200C082A900C282A800C8A2A90065
:105A2000CAA2A80004003700C082A900C282A9004F
:105A3000C8A2A900CAA2A9006AFA0700CE003700CE
:105A40001000200020079800407380006400400090
:105A500040738800ACFB07000000E0000600320045
:105A600080B82000104078000000A00081B820001D
:105A7000804878000500370080B82000104078008A
:105A80000000A00081B820008048780055FA070087
:105A9000B9003700100020002007980040738000F4
:105AA000640040004073880097FB07002061880075
:105AB000206180000000E00002003D000000EB00DB
:105AC000206188002161800000FA2000808F500052
:105AD0000200340000FA200020618800306180005C
:105AE000E10F500002003C002000200030618800DF
:105AF0003161800030062000808F500002003400A9
:105B0000300620003061880064720200000000004E
:105B100034FA070098003700100020002007980092
:105B200040738000640040004073880076FB0700EB
:105B300030618800206180000000E00002003D002C
:105B40000000EB00206188002161800000FA200045
:105B5000808F50000200340000FA2000206188008D
:105B600030618000E10F500002003C002000200066
:105B7000306188003161800030062000808F500045
:105B80000200340030062000306188006472020098
:105B90000000000013FA0700770037001000200013
:105BA0002007980040738000640040004073880024
:105BB00055FB07000000E00009003200A140800012
:105BC000E00220000088B900F0004000E0932000CF
:105BD000008040001000780000000100080037003D
:105BE000A1408000E00220000088B900F2004000DF
:105BF000E0932000008040001000780000000100C9
:105C0000F8F907005C00370010002000200798001A
:105C10004073800064004000407388003AFB070036
:105C2000700798007E009000E10F500010003200D5
:105C3000FE009000E28F5000160032007E019000BE
:105C40000200E000010032001A003700A14080008D
:105C5000E00220000088B900EE004000E093200040
:105C600000804000100078000000010011003700A3
:105C7000A1408000E00220000088B900EC00400054
:105C8000E093200000804000100078000000010038
:105C900008003700A1408000E00220000088B90021
:105CA000F6004000E09320000080400010007800E3
:105CB00000000100CBF907002F0037001000200082
:105CC0002007980040738000640040004073880003
:105CD000417380006E009000008040000000E900E9
:105CE00040738800BFF90700230037001000200030
:105CF00020079800407380006400400040738800D3
:105D000001FB0700000F78001E0078004C9702008E
:105D100000000000B3F90700170037001000200052
:105D200020079800407380006400400040738800A2
:105D3000F5FA0700000F7800A1408000E002200083
:105D40000088B900FC004000E09320000080400083
:105D5000900078001E00780001000100A1F9070002
:105D600005003700100020003007980002003700BF
:105D700030002000300798002E0090000000E00066
:105D800005003A00417380006E00900000804000E2
:105D900063004000407388000000EB00200798007B
:105DA0003E0090000000E000CAFB3200D0408000BE
:105DB0000080A100D04088003E009000E10F50001C
:105DC0001800320061002000A03A2000EE99020085
:105DD000000000003E009000106F02000000000074
:105DE00081002000003B2000EE990200000000002E
:105DF0005E009000106F020000000000B100200063
:105E0000803B2000EE9902000000000040738000FB
:105E1000106F02000000000060922800026D020076
:105E2000000000004F0478000080FA000000060027
:105E30000200FA00000F780000C2B30032710200C5
:105E4000000000001E007800D66C02000000000078
:105E500000C2B30032710200000000000080FA00AE
:105E6000000006000400FA000000EB004073880008
:105E70003F0037004173800000E7200000804000B1
:105E800090407800214798002E4090000004E000E8
:105E9000040035002E409000327102000000000026
:105EA00030003700AE40900000CEB30080CF5000ED
:105EB0001C00360060922800026D02000000000005
:105EC000407380008000E80000E720000080400070
:105ED000104078000080FB004801DD004073800026
:105EE0008080E80000E7200000804000104078003B
:105EF0000080FB0000004100000F7800407380002C
:105F00000080E800407388001E007800106F0200D7
:105F10000000000000C2B300327102000000000067
:105F20001000370000C2B300327102000000000010
:105F30002E4090008080FB0000F82F000080400081
:105F40008000400020B32000008040001000780056
:105F5000D66C02000000000000C2B30032710200E3
:105F600000000000407380000000E80040738800DB
:105F70004173800000E7200000804000104078005E
:105F80000004E000BBFF3A0060922800026D0200AE
:105F900000000000407380000000E900106F020064
:105FA0000000000071002000303C2000789A0200C0
:105FB000000000000080FA00000006000600FA0061
:105FC0001007980050698000000F78001700370014
:105FD0001E009000104178005169800080C22000AE
:105FE0000080400010407800804F510005003200D2
:105FF0001E007800506988000000EB002007980020
:1060000010003700506980000000E80050698800E7
:1060100051698000F00F2000008060005069880006
:106020001E0090000000E800100798001E0090007D
:10603000104078000004E000E5FF3A001000200066
:10604000200798002E0090000080FA000000060053
:106050000400FA000000EB00000F78001000370089
:106060001E0078008000400020B320000080400027
:1060700010007800D1FF07000000E00007003200A8
:106080001E0078008040780000C8B30000C04000C7
:106090000080FB0010079800060037001E0FE80084
:1060A000000220009E0F1000EDFF34000000EB0006
:1060B000100798001E0090000080FA000000060003
:1060C0003200FA0050698000600798001F00370016
:1060D000EE00900080C220000080400090407800D8
:1060E00000C6B30080CF500011003400EE009000D5
:1060F00080C220000080400090407800A0C7B3001C
:1061000080CF50000A003C006E019000EE0090002D
:1061100080C220000080400090407800F0CDB300A5
:1061200080C0600080C2200000004100014878006B
:106130006E0090000000E80060079800EE009000FC
:10614000F00F20000080600060079800EE009000D3
:1061500040698000808F5000DDFF3A000000EB00B6
:10616000600798005169800080C2200000804000D4
:1061700090407800F0C2B30080CF50001F0134007F
:106180005169800080C2200000804000904078006B
:1061900090C3B30080CF500018013C000000EB001A
:1061A00060079800070037006E019000EE0047007E
:1061B0000040EB0000F178006E0090000000E80065
:1061C00060079800EE00900020022000808F5000B1
:1061D000F5FF34005616020000000000400798004A
:1061E0004E0090004880DE00804078006E0047003E
:1061F000114098004E0090008040780000C0EB00F5
:1062000080C060006E004700214098004E00900062
:106210008CF80700300798003E009000E10F400026
:106220002B003200BE00900000E7200000804000FC
:10623000104078008080FB0030F22F00008040008A
:10624000100798003E009000600798000D0037008E
:106250006E019000EE0090001E00900080804000D3
:1062600000E72000008040009040780000E7200018
:1062700000004100014878006E0090000000E80036
:1062800060079800014020001E00900080805000B0
:106290006E009000808F5000EDFF3C00080037003A
:1062A000EE00900000E72000808040000040EB00FE
:1062B000804878006E0090000000E80060079800B9
:1062C000EE009000F03F2000808F5000F4FF34007B
:1062D00030002000600798000000EB00000F7800FD
:1062E0002C1A0200000000003E0037001E00E000F3
:1062F00002003A002C1A0200000000001E00E0001C
:1063000004003A0052FF07000080FB00400798009D
:10631000020037000000EB00400798004E0090009C
:106320000000E0000C0032006E0190004E00900072
:10633000804078006E00470001717800CE00900028
:1063400070082000808F50001A003A0010002000D2
:10635000000F7800170037005169800080C22000CC
:10636000008040009040780020C2B30080CF5000F1
:1063700001003A001E00A2006E01900051698000E9
:1063800080C22000008040001040780080407800EB
:106390006E00470001717800506980000000E8003D
:1063A0005069880051698000F00F20000080600073
:1063B000506988006E0090000000E80060079800B7
:1063C000EE00900030022000808F50000500340065
:1063D00091002000A03C2000789A020000000000FC
:1063E000E50037005169800040698000808F5000CF
:1063F000BEFF3A006E009000E30F5000DE00320056
:106400006E009000E40F5000DB0032006E00900040
:1064100080407800C0CDB30000C0400080407800CC
:106420006E004700014878000000EB00600798000C
:106430000000EB00200798000000EB0030079800F8
:106440003D003700EE00900000E720000080400093
:106450009040780000CEB30080CF50002500360079
:10646000EE00900000E7200000804000104078001F
:106470008080FB0000F22F00008040001007980091
:106480006E0090008000E80000E7200000804000DF
:10649000904078006E0047001040900080CF500080
:1064A0000E003E006E0090008080E80000E72000B3
:1064B00000804000904078006E004700204090002F
:1064C00080CF500005003100EE0090001E009000CB
:1064D0000080400063004000300798009E0090005C
:1064E0006E0090000080400063004000600798004C
:1064F000020037006E009000200798006E009000A8
:106500008000E80000E72000008040001040780094
:106510000080FB004801DD006E0090008080E800F4
:1065200000E7200000804000104078000080FB0061
:1065300000004100400798002E0090000000E0009D
:10654000C0FF32006E004700104078008080FB00E2
:1065500030F22F0000804000400798002E0090008D
:10656000600798000D003700EE0090004E0090008C
:1065700000814000EE00900000E720000080400015
:106580009040780000E720000000410001487800BA
:106590006E0090000000E90060079800EE00900097
:1065A0003E009000808F5000EFFF3D000000EB00A8
:1065B000600798000C003700BE0090006E0090004D
:1065C00000814000EE0090006E004700E14078003E
:1065D00000E7200000004100014878006E009000B4
:1065E0000000E80060079800EE0090004E00900068
:1065F000808F5000F0FF35005F0037007092280058
:106600006EFE07000000E000050032008CF9070074
:1066100060922800026D0200000000005600370062
:10662000B092280065FE07000000E0000200320082
:106630000CFE070050003700009328005FFE0700A3
:106640000000E00004003200D04080000090A10073
:10665000D0408800480037005093280057FE0700BC
:106660000000E000200032000000EB00600798000E
:10667000180037000000EB00500798000F003700AB
:10668000EE0090005E0090008080400000E7200057
:1066900000804000104078000080FB00D06F0200B6
:1066A0000000000000C2B3003271020000000000D0
:1066B0005E0090000000E800500798005E00900027
:1066C000EF0F5000EEFF34006E00900070004000AD
:1066D00060079800EE009000F03F2000808F50008F
:1066E000E4FF340024003700B093280033FE070095
:1066F0000000E0001C0032000000EB006007980082
:1067000008003700EE00900000E720008080400085
:106710000040EB00804878006E0090000000E80028
:1067200060079800EE009000F03F2000808F50003E
:10673000F4FF340011CEB30000E7200001487800D8
:1067400080C0EB0010E720000148780080C0EB001B
:1067500020E720000148780011CAB30030E720008C
:106760000148780004003700C1002000303D2000BF
:10677000789A0200000000000080FA000000060085
:106780005752490054452000424954003A20200005
:106790002A6E650078742000636C6F00636B2000C4
:1067A000285E2900207769006C6C200075736500F5
:1067B000207468006973200076616C007565310093
:1067C00057495200452072006F757400696E65006C
:1067D00073202800432920003230300030204D0043
:1067E0006963680061656C00205065006172630038
:1067F000652047004E55200047504C004E6F20004A
:1068000064657600696365002C207400727920004D
:1068100028414C0041524D0029205300454152006F
:10682000434820006D616300726F2000666972004A
:10683000737441004444520045535300204D4100BD
:1068400043524F00202030002E4D610063726F00D4
:10685000206D65006E754D00616372006F20200031
:106860002020200031574900524520006164640017
:1068700072657300730D0A00202020002A31570032
:106880004952450020524F004D2043004F4D4D00CE
:10689000414E4400204D410043524F00733A0D00D9
:1068A0000A203500312E52004541440020524F004D
:1068B0004D20280030783300332920002A666F00ED
:1068C00072207300696E67006C6520006465760055
:1068D0006963650020627500730D0A002038350079
:1068E0002E4D41005443480020524F004D202800B7
:1068F00030783500352920002A666F006C6C6F00F7
:106900007765640020627900203634006269740083
:10691000206164006472650073730D000A20320008
:1069200030342E00534B4900502052004F4D200070
:106930002830780043432900202A66006F6C6C00E1
:106940006F77650064206200792063006F6D6D00D1
:10695000616E64000D0A2000323336002E414C0077
:1069600041524D0020534500415243004820280029
:106970003078450043290D000A20320034302E00C3
:10698000534541005243480020524F004D202800FB
:1069900030784600302941004C4152004D205300D0
:1069A00045415200434820002830780045432900E3
:1069B00053454100524348002028300078463000BB
:1069C000294465007669630065204900447320000E
:1069D000617265002061760061696C0061626C0023
:1069E0006520620079204D00414352004F2C200069
:1069F0007365650020283000292E5200454144006F
:106A000020524F004D2028003078330033293A00BF
:106A1000204D41005443480020524F004D20280093
:106A200030783500352953004B49500020524F0033
:106A30004D20280030784300432955006E6B6E00CE
:106A40006F776E00206D610063726F002C20740000
:106A5000727920003F206F0072202800302920002A
:106A6000666F7200206865006C704200555320000C
:106A70005245530045542000576172006E696E0004
:106A8000673A20002A5368006F727400206F72000A
:106A9000206E6F00207075006C6C2D0075702000EA
:106AA0002A4E6F00206465007669630065206400EB
:106AB00065746500637465006420440053313800D8
:106AC000533230002048690067682000507265002A
:106AD000732044006967200054686500726D4400AB
:106AE0005331380042323000205072006F6720006E
:106AF0005265730020446900672054006865720085
:106B00006D4453003138320032204500636F6E000F
:106B10002044690067205400686572006D4453008A
:106B20003234300034204500636F6E0072616D00B6
:106B3000207469006D65200043686900704453004B
:106B400032343300312031004B2045004550520093
:106B50004F4D55006E6B6E006F776E0020646500C0
:106B600076696300655057004D20640069736100C9
:106B7000626C650064314B00487A2D00342C300083
:106B800030304B00487A200050574D004672650067
:106B9000717565006E63790020696E00204B4800B6
:106BA0007A2050007265730063616C00653A500092
:106BB00052323A00447574007920630079636C00A6
:106BC000652069006E202500205057004D2061008F
:106BD000637469007665450052524F00523A2000B6
:106BE00050574D002061630074697600652C2000C9
:106BF000672074006F20640069736100626C650037
:106C0000415558002046720065717500656E63003D
:106C1000793A20004155580020494E005055540003
:106C20002F4849002D5A4100555820004849470037
:106C30004841550058204C004F5756004F4C5400C7
:106C40004D455400455220004D4F440045564F00DD
:106C50004C5441004745200050524F0042453A00F5
:106C60002056450072726F007228290020406C0087
:106C7000696E65003A20400070676D0073706100B6
:106C800063653A0020627900746573002E546F00CA
:106C90006F206C006F6E6700215379006E74610085
:106CA0007820650072726F00724E6F0020454500BB
:106CB00050524F004D457200617369006E67640069
:106CC0006F6E650053617600696E670020746F0017
:106CD00020736C006F742000496E7600616C69004F
:106CE000642073006C6F74004C6F610064696E0007
:106CF00067206600726F6D0020736C006F74200057
:106D0000455252004F523A0020636F006D6D610092
:106D10006E64200068617300206E6F00206566005D
:106D200066656300742068006572650041434B002E
:106D30004E4143004B49320043205300544152001E
:106D400054204200495449003243200053544F001C
:106D50005020420049544900324320006D6F6400C6
:106D6000653A0D000A2031002E2053006F66740032
:106D700077617200650D0A0020322E002048610004
:106D8000726477006172650053657400207370004F
:106D9000656564003A0D0A0020312E00207E350022
:106DA0004B487A000D0A2000322E20007E3530003C
:106DB0004B487A000D0A2000332E20007E3130002F
:106DC000304B48007A0D0A0020342E00207E34001B
:106DD00030304B00487A570041524E00494E470030
:106DE0003A20480041524400574152004520490092
:106DF000324320006973200062726F006B656E0081
:106E0000206F6E00207468006973200050494300B1
:106E100021202800524556002041330029536500A7
:106E20007420730070656500643A0D000A2031001B
:106E30002E20310030304B00487A0D000A203200FD
:106E40002E20340030304B00487A0D000A203300E9
:106E50002E2031004D487A004932430020286D0031
:106E60006F64200073706400293D280020203000EA
:106E70002E4D610063726F00206D65006E750D0010
:106E80000A2031002E3762006974200061646400BA
:106E900072657300732073006561720063680D0092
:106EA0000A2032002E493200432073006E696600CA
:106EB000666572005365610072636800696E670001
:106EC00020493200432061006464720065737300DE
:106ED00020737000616365002E2046006F756E00A0
:106EE0006420640065766900636573002061740046
:106EF0003A536E006966660065722800424153008D
:106F00004943290052656100647961002F412F00D7
:106F1000402063006F6E7400726F6C00732041003C
:106F20005558200070696E00612F41002F402000ED
:106F3000636F6E0074726F006C7320004353200007
:106F400070696E00436F6D006D616E0064206E00AD
:106F50006F74200075736500642069006E207400F2
:106F600068697300206D6F0064655000756C6C007B
:106F70002D7570002072650073697300746F720064
:106F800073204F0046465000756C6C002D757000E4
:106F90002072650073697300746F720073204F0074
:106FA0004E5365006C662D00746573007420690093
:106FB0006E204800695A20006D6F640065206F00E4
:106FC0006E6C790052455300455442004F4F5400B7
:106FD0004C4F4100444552004155580020494E0055
:106FE000505554002F4849002D5A2C00205245007E
:106FF00041443A0020506F0077657200207375009D
:1070000070706C0069657300204F4E00506F770000
:107010006572200073757000706C690065732000E4
:107020004F4646004441540041205300544154000F
:10703000453A200044454C004159200075735700E3
:1070400052495400453A200052454100443A20003C
:10705000434C4F00434B2C00203143004C4F430026
:107060004B2C200030444100544120004F55540027
:10707000505554002C2031004441540041204F0011
:107080005554500055542C00203020002A706900BF
:107090006E20690073206E006F77200048695A00E7
:1070A000434C4F00434B2000544943004B533A009C
:1070B0002052450041442000424954003A205300E8
:1070C000796E740061782000657272006F72200022
:1070D0006174200063686100722078002E206500D2
:1070E000786974002877690074686F0075742000EF
:1070F000636861006E676500296E6F00206D6F0028
:1071000064652000636861006E6765004E6F6E0005
:1071100065786900737465006E74200070726F008A
:10712000746F63006F6C2100782E20006578690011
:10713000740D0A00496E7600616C6900642063007A
:10714000686F690063652C0020747200792061000B
:10715000676169006E444500564944003A6874000E
:1071600074703A002F2F6400616E670065726F00C3
:1071700075737000726F74006F74790070657300BE
:107180002E636F006D2A2D002D2D2D002D2D2D002D
:107190002D2D2D002A4F7000656E20006472610055
:1071A000696E20006F75740070757400732028007C
:1071B000483D4800692D5A002C204C003D474E00A8
:1071C00044294E006F726D00616C20006F75740071
:1071D0007075740073202800483D33002E3376000C
:1071E0002C204C003D474E0044294D0053422000C6
:1071F000736574003A204D004F53540020736900AA
:1072000067206200697420006669720073744C0024
:1072100053422000736574003A204C0045415300EE
:107220005420730069672000626974002066690059
:107230007273740020426F006F746C006F616400A1
:1072400065722000762031002E20480045580D0040
:107250000A2032002E20440045430D000A2033004E
:107260002E204200494E0D000A2034002E205200EC
:1072700041574400697370006C61790020666F00AB
:10728000726D610074207300657456006F6C740039
:1072900061676500206D6F006E6974006F72730026
:1072A0003A203500563A2000207C2000332E33004F
:1072B000563A2000207C2000565055004C4C55007A
:1072C000503A2000536574002073650072696100B4
:1072D0006C2070006F72740020737000656564002C
:1072E0003A20280062707300290D0A0020312E0018
:1072F00020333000300D0A0020322E0020313200C1
:1073000030300D000A2033002E203200343030009F
:107310000D0A2000342E200034383000300D0A00D1
:1073200020352E002039360030300D000A2036007E
:107330002E20310039323000300D0A0020372E0067
:1073400020333800343030000D0A2000382E200061
:107350003537360030300D000A2039002E2031003C
:107360003135320030300D000A3130002E2042001D
:107370005247200072617700207661006C756500CD
:1073800041646A007573740020796F007572200083
:10739000746572006D696E00616C41007265200059
:1073A000796F75002073750072653F0020434600B9
:1073B00047313A002043460047323A00285C2D000E
:1073C0002F5F5C002D2928005C5F2F002D295300C2
:1073D000656C6500637420006F75740070757400CF
:1073E0002074790070653A000D0A2000312E2000CB
:1073F0004F7065006E206400726169006E20280085
:10740000483D4800692D5A002C204C003D474E0055
:1074100044290D000A2032002E204E006F726D00AC
:10742000616C200028483D00332E3300562C20008C
:107430004C3D47004E44290052325700202873002B
:107440007064200068697A00293D280020203000FF
:107450002E4D610063726F00206D65006E750D002A
:107460000A2031002E4953004F37380031362D00A5
:107470003320410054520D000A2032002E4953009F
:107480004F37380031362D003320700061727300A1
:1074900065206F006E6C790049534F00203738002B
:1074A00031362D003320410054522000285245002F
:1074B00053455400206F6E0020435300290D0A00ED
:1074C000524553004554200048494700482C2000AD
:1074D000434C4F00434B2000544943004B2C2000A9
:1074E00052455300455420004C4F570049534F001C
:1074F0002037380031362D003320720065706C0063
:10750000792028007573650073206300757272001E
:10751000656E7400204C5300422073006574740043
:10752000696E6700293A200050726F00746F630023
:107530006F6C3A0020736500726961006C33200043
:1075400077697200653220007769720065524600E3
:1075500055756E006B6E6F00776E5200656164004A
:107560002074790070653A0020746F0020656E0009
:107570006476610072696100626C6500206C650070
:107580006E6774006844610074612000756E690064
:1075900074733A00206E6F0020696E0064696300A6
:1075A000617469006F6E44006174610020756E0043
:1075B000697420006C656E006774680020286200A2
:1075C00069747300293A200043532000454E41005E
:1075D000424C45004443530020444900534142007B
:1075E0004C4544005233570020287300706420003B
:1075F00063736C00206869007A293D002820290007
:107600000D0A4400697363006F6E6E006563740059
:1076100020616E00792064006576690063657300FF
:107620000D0A43006F6E6E006563740020285600DB
:1076300070752000746F20002B35560029206100E2
:107640006E64200028414400432074006F202B000A
:10765000332E33005629430074726C004155580094
:107660004D4F440045204C0045445000554C4C00C3
:1076700055502000485055004C4C550050204800B3
:107680005652450047414400432061006E6420008B
:1076900073757000706C7900355656005055330084
:1076A0002E33560041444300427573002068690040
:1076B000676842007573200048692D005A20300029
:1076C00042757300204869002D5A2000314D4F004B
:1076D00044452000616E640020565200454720005A
:1076E0004C45440073207300686F75006C64200083
:1076F000626520006F6E2100466F75006E64200089
:1077000020657200726F7200732E4D004F53490056
:10771000434C4B004D4953004F435300204F4B0007
:1077200020464100494C5300657420007370650089
:1077300065643A000D0A2000312E200033304B00E2
:10774000487A0D000A2032002E20310032354B00DD
:10775000487A0D000A2033002E20320035304B00CD
:10776000487A0D000A2034002E2031004D487A005E
:10777000436C6F00636B2000706F6C006172690076
:1077800074793A000D0A2000312E200049646C0003
:1077900065206C006F7720002A64650066617500C3
:1077A0006C740D000A2032002E204900646C6500C4
:1077B0002068690067684F00757470007574200058
:1077C000636C6F00636B200065646700653A0D00B1
:1077D0000A2031002E204900646C650020746F007F
:1077E0002061630074697600650D0A0020322E0066
:1077F0002041630074697600652074006F20690081
:10780000646C6500202A640065666100756C740014
:10781000496E70007574200073616D00706C6500B6
:1078200020706800617365003A0D0A0020312E0057
:10783000204D690064646C0065202A006465660060
:1078400061756C00740D0A0020322E0020456E0018
:1078500064535000492028007370640020636B005B
:10786000702073006B652000736D700020637300DF
:107870006C206800697A29003D28200020302E0005
:107880004D616300726F20006D656E00750D0A001A
:1078900020312E00536E690066662000435320009D
:1078A0006C6F77000D0A2000322E53006E6966005F
:1078B000662061006C6C200074726100666669006D
:1078C000632D7000202D6600202A42007974650027
:1078D00073206400726F7000706564002A46410076
:1078E000494C4500442C20004E4F20004441540098
:1078F000414461007461200062697400732061007A
:107900006E64200070617200697479003A0D0A009B
:1079100020312E0020382C00204E4F004E452000F4
:107920002A646500666175006C7420000D0A2000F1
:10793000322E2000382C2000455645004E200D00E8
:107940000A2033002E2038002C204F004444200011
:107950000D0A2000342E2000392C20004E4F4E00FE
:10796000455374006F70200062697400733A0D0013
:107970000A2031002E203100202A64006566610053
:10798000756C74000D0A2000322E20003252650002
:107990006365690076652000706F6C006172690034
:1079A00074793A000D0A2000312E200049646C00E1
:1079B00065203100202A640065666100756C7400E2
:1079C0000D0A2000322E200049646C006520300032
:1079D00055415200542028007370640020627200E8
:1079E000672064006270200073622000727870006B
:1079F000206869007A293D0028202000302E4D00A3
:107A0000616372006F206D00656E75000D0A2000C5
:107A1000312E540072616E007370610072656E00E9
:107A2000742062007269640067650D000A203200EC
:107A30002E204C0069766500206D6F006E69740021
:107A40006F720D000A2033002E42720069646700D5
:107A5000652077006974680020666C006F772000ED
:107A6000636F6E0074726F006C55410052542000B9
:107A70006272690064676500526573006574200076
:107A8000746F20006578690074526100772055009A
:107A90004152540020696E007075740055415200C7
:107AA00054204C00495645002044490053504C0096
:107AB00041592C00207D2000544F200053544F008A
:107AC000504C49005645200044495300504C410059
:107AD00059205300544F5000504544005741520024
:107AE0004E494E00473A200070696E0073206E00C8
:107AF0006F7420006F7065006E2064007261690011
:107B00006E20280048695A00292052004556490035
:107B1000443A0D000A496E0076616C0069642000E9
:107B200063686F00696365002C207400727920001F
:107B300061676100696E6D0073525300204C4F0005
:107B4000572C2000434F4D004D414E0044204D0026
:107B50004F4445005253200048494700482C20001C
:107B60004441540041204D004F44450041646400AD
:107B70007265730073206F00662050004346380022
:107B8000353734003F546800697320006D6F64001E
:107B9000652072006571750069726500732061006F
:107BA0006E20610064617000746572004C43440093
:107BB0002074790070653A000D0A2000312E2000F3
:107BC0004844340034373800302028007573690089
:107BD0006E67200050434600383537003420490096
:107BE0004F206500787061006E64650072294C005A
:107BF000434420002874790070206100646472009E
:107C000029203D002028200020302E004D616300F7
:107C1000726F20006D656E00750D0A0020312E0018
:107C20004C43440020526500736574000D0A200027
:107C3000322E49006E697400204C4300440D0A0046
:107C400020332E00436C6500617220004C434400D9
:107C50000D0A2000342E4300757273006F722000ED
:107C6000706F7300697469006F6E200065783A0068
:107C70002834290020300D000A2036002E577200CB
:107C80006974650020746500737420006E756D0062
:107C90006265720073206500783A2800362920005A
:107CA00038300D000A2037002E57720069746500C5
:107CB0002074650073742000636861007261630062
:107CC0007465720073206500783A28003729200017
:107CD00038304400697370006C617900206C690071
:107CE0006E6573003A0D0A0020312E00203120000D
:107CF0000D0A2000322E20004D756C007469700052
:107D00006C6549004E495400434C450041524300C4
:107D1000555253004F522000534554004E6F2000DF
:107D200041434B002C206300686563006B206100B9
:107D30006461700074657200434C4B00094D4F0044
:107D400053490900435309004D4953004F506900FE
:107D50006E73740061746500733A47004E44090005
:107D6000332E3300560935002E30560009414400A9
:107D70004309560050550900415558000950090063
:107D8000500950000949090049092D00094F5700C1
:107D900044092D00092D2D000954780044092D00B7
:107DA00009527800445343004C09530044410900F0
:107DB0002D092D00504743000950470044092D006C
:107DC000092D31002E28420052290900322E2800A8
:107DD0005244290009332E00284F5200290934004B
:107DE0002E28590057290900352E2800474E290012
:107DF00009362E0028424C00290937002E28500051
:107E000055290900382E28004752290009392E002B
:107E100028575400290930002E2842006C6B290095
:107E2000474E440009474E004409410044430900BD
:107E3000352E3000560933002E33560009565000B7
:107E4000550941005558090065786500637574004F
:107E500065203A0020205400494D45004F555400FC
:107E600020302E00204D610063726F00206D650090
:107E70006E750D000A2031002E204C0069766500D9
:107E800020696E0070757400206D6F006E6974005B
:107E90006F7249006E70750074206D006F6E69001E
:107EA000746F7200202A730074617200746269003A
:107EB0007420650072726F0072202A007061720077
:107EC0006974790020657200726F7200202A730055
:107ED000746F70006269740020657200726F7200C6
:107EE000204E4F004E452000554E4B004E4F570040
:107EF0004E20450052524F005220610075746F00B1
:107F000072616E00676520002B4D48007A292B00B6
:107F10006B487A002952610077207600616C750009
:107F2000652066006F7220004252470020284D00F5
:107F3000494449003D3132003729570041524E0033
:107F4000494E47003A2050006F73730069626C001D
:107F5000652062007566660065726F007665720066
:107F6000666C6F0077416E0079206B0065792000A8
:107F7000746F200065786900745370006163650058
:107F800020746F0020636F006E7469006E75650069
:107F90004E756D0062657200206F66002062690098
:107FA0007473200072656100642F77007269740039
:107FB000653A200043533A000D0A2000312E20007C
:107FC00043530D000A2032002E202F00435320007F
:107FD0002A646500666175006C7450006F736900F7
:107FE00074696F006E2069006E206400656772001E
:107FF0006565730053657200766F200061637400DD
:108000006976650047656E00657261006C0909005C
:108010000909090050726F00746F63006F6C2000D3
:10802000696E740065726100637469006F6E2D0083
:108030002D2D2D002D2D2D002D2D2D002D2D2D0024
:108040002D2D2D002D2D2D002D2D2D002D2D2D0014
:108050002D2D2D002D2D2D002D2D2D002D2D2D0004
:108060002D2D2D002D2D2D002D2D2D002D2D2D00F4
:108070002D2D2D002D2D2D002D2D2D002D2D2D00E4
:108080002D2D2D002D2D2D002D2D2D002D2D2D00D4
:108090002D2D3F00095468006973200068656C004D
:1080A000700909000928300029094C00697374001F
:1080B00020637500727265006E7420006D6163004C
:1080C000726F73003D582F007C580900436F6E009B
:1080D0007665720074732000582F72006576650013
:1080E00072736500205809000928780029094D009D
:1080F000616372006F2078007E095300656C660032
:108100007465730074090900095B09005374610008
:10811000727423000952650073657400090909002F
:10812000095D090053746F00702409004A756D00E1
:10813000702074006F2062006F6F74006C6F6100BC
:108140006465720009097B00095374006172740050
:1081500020776900746820007265610064262F0032
:1081600025094400656C6100792031002075730099
:108170002F6D7300090909007D095300746F7000A9
:10818000612F41002F4009004155580050494E00D1
:1081900020286C006F772F0048492F00524541007E
:1081A0004429090009226100626322000953650025
:1081B0006E64200073747200696E67006209530078
:1081C0006574200062617500647261007465090065
:1081D00009093100323363002F430900415558002B
:1081E00020617300736967006E6D65006E74200016
:1081F00028617500782F4300532909000930780061
:1082000031323300642F4400094D650061737500FD
:10821000726520004144430020286F006E636500B2
:108220002F434F004E542E00290930006231310097
:1082300030095300656E6400207661006C7565003E
:1082400066094D00656173007572650020667200F5
:1082500065717500656E6300790909007209520045
:1082600065616400672F5300094765006E65720001
:1082700061746500205057004D2F530065727600E1
:108280006F0909002F0943004C4B20006869680002
:1082900009436F006D6D61006E646800697374005E
:1082A0006F727900090909005C0943004C4B2000FA
:1082B0006C6F690009566500727369006F6E690022
:1082C0006E666F002F7374006174750073696E00C1
:1082D000666F0900095E0900434C4B002074690079
:1082E000636B6C002F4C0900426974006F7264006C
:1082F00065722000286D7300622F4C0053422900E4
:1083000009092D000944410054206800696D0900E5
:10831000436861006E676500206D6F006465090049
:1083200009095F000944410054206C006F6F090087
:1083300053657400206F75007470750074207400AC
:1083400079706500090909002E0944004154200094
:108350007265610064702F0050095000756C6C00EC
:108360007570200072657300697374006F7273001A
:1083700020286F0066662F004F4E29000921090052
:1083800042697400207265006164730009536300E0
:1083900072697000742065006E6769006E6509007F
:1083A00009093A0009526500706561007420650092
:1083B0002E672E0020723A00313076000953680093
:1083C0006F772000766F6C0074732F0073746100F8
:1083D0007465730009093B00094269007473200049
:1083E000746F200072656100642F770072697400F9
:1083F000652065002E672E002030780035353B0063
:1084000032772F005709500053552000286F66001F
:10841000662F4F004E290900093C78003E2F3C0092
:10842000783D20003E2F3C00303E0900557365002A
:10843000726D610063726F0020782F0061737300AA
:1084400069676E0020782F006C69730074206100EA
:108450006C6C00000000FA0080B920001040780029
:108460000030A00081B920008048780080B9200049
:1084700010407800704060000004E000020032000C
:10848000CAC2A90001003700CAC2A80080B92000F2
:1084900010407800704060000004E00003003200EB
:1084A000F0C2B3003271020000000000A100200001
:1084B00060AB2000789A0200000000000080FA0003
:1084C000000006000000FA0080B92000104078008B
:1084D0000030A10081B920008048780080B92000D8
:1084E00010407800704060000004E000020032009C
:1084F000CAC2A90001003700CAC2A80080B9200082
:1085000010407800704060000004E000030032007A
:10851000F0C2B3003271020000000000A100200090
:1085200060AB2000789A0200000000000080FA0092
:10853000000006000000FA0080B92000104078001A
:10854000704060000004E00002003200CAC2A800CF
:1085500001003700CAC2A90080B92000104078008D
:10856000704060000004E00003003200F0C2B3007D
:108570003271020000000000B100200000AC2000B9
:10858000789A0200000000000080FA000000060057
:108590000000FA0000C0EB00270207000080FB008B
:1085A0000080FA00000006000600FA00100798009C
:1085B0001E00900020020700004F780080B92000C4
:1085C00010407800684060000004E00003003200C2
:1085D0001E80FB00200798000200370000102000DA
:1085E000200798002E0090000080FA00000006008E
:1085F0000000FA0001022000D0C92000EE9902001C
:108600000000000060B72000104078006E6F02008C
:108610000000000000C2B300327102000000000040
:1086200080B9200010407800614060006E6F020049
:108630000000000000C2B300327102000000000020
:1086400080B92000104078000080FB000000D100BD
:10865000614060006E6F02000000000000C2B300C5
:10866000327102000000000080B920001040780044
:108670000080FB004200DE00614060006E6F02007F
:108680000000000000C2B3003271020000000000D0
:1086900080B92000104078000080FB004400DE001C
:1086A000614060006E6F02000000000000C2B30075
:1086B000327102000000000080B8200010407800F5
:1086C0000080FB004300DE00614060006E6F02002E
:1086D0000000000000C2B300327102000000000080
:1086E00031002000F0AD2000EE99020000000000F3
:1086F0000080FA00000006000C00FA002C1A0200AC
:10870000000000005616020000000000500798000C
:108710002C1A0200000000005616020000000000A3
:10872000400798002C1A02000000000056160200B4
:1087300000000000300798002C1A02000000000022
:108740005616020000000000200798002C1A0200B4
:10875000000000005616020000000000000F780024
:108760002C1A020000000000561602000000000053
:10877000100798005E0090000000E000090034003F
:108780005E009000E40F500006003C005E00900088
:108790000040E9008040780060B720000148780080
:1087A000020037000000EB00500798004E009000D8
:1087B0000000E0000F0034004E009000E20F500077
:1087C0000C003C004E0090000040E900E1406000D9
:1087D00080B920001040780061C16000E1CFB30093
:1087E000014060000240700081B92000804878009C
:1087F000020037000000EB00500798003E00900098
:108800000000E000100034003E009000E20F500035
:108810000D003C003E0090000040E9006141600016
:1088200080B9200090407800614061000041400024
:10883000D0CFB30080C0600082C0700080B920003B
:1088400001487800020037000000EB005007980054
:108850002E0090000000E000100034002E00900078
:10886000E20F50000D003C002E0090000040E90097
:108870006141600080B92000904078006140610053
:108880004201DD00B0CFB30080C0600082C0700044
:1088900080B9200001487800020037000000EB009A
:1088A000500798001E00E000100034002000200057
:1088B0009E0F10000D003C001E0078000040E900F3
:1088C0006141600080B92000904078006140610003
:1088D0004401DD00F0CEB30080C0600082C07000B3
:1088E00080B9200001487800020037000000EB004A
:1088F000500798001E0090000000E00010003400B7
:108900001E009000E20F50000D003C001E00900081
:108910000040EA006141600080B82000904078008B
:10892000614061004301DD0070CFB30080C0600092
:1089300082C0700080B82000014878000200370033
:108940000000EB00500798005E0090000000E0007F
:1089500079003A000000EB00606988007103200094
:10896000D0BB2000789A0200000000008001EB00DC
:10897000420020001100200010002000A21C020074
:10898000000000000040E9008040780060B720004F
:10899000014878005103200040BF2000789A02006F
:1089A000000000008001EB002200200011002000E8
:1089B00010002000A21C0200000000000040E9009E
:1089C000E140600080B920001040780061C1600083
:1089D000E1CFB300014060000240700081B9200087
:1089E000804878003104200090C22000789A02006C
:1089F000000000008001EB00220020001100200098
:108A000020002000A21C0200000000000040E9003D
:108A10006141600080B920009040780061406100B1
:108A200000414000D0CFB30080C0600082C0700021
:108A300080B920000148780011032000C0C6200042
:108A4000789A0200000000008001EB002200200064
:108A50001100200010002000A21C020000000000F5
:108A60000040E9006141600080B92000904078003A
:108A7000614061004201DD00B0CFB30080C0600002
:108A800082C0700080B9200001487800D101200028
:108A900070222100789A0200000000008001EB00A3
:108AA000220020001100200020002000A21C020053
:108AB000000000000040E9006141600080B9200032
:108AC00090407800614061004401DD00F0CEB300C9
:108AD00080C0600082C0700080B92000014878002A
:108AE000F1042000B0932000789A020000000000FA
:108AF0008001EB0022002000110020001000200067
:108B0000A21C0200000000000040EA006141600079
:108B100080B8200090407800614061004301DD0092
:108B200070CFB30080C0600082C0700080B82000A9
:108B30000148780001003700ADFE070080B9200031
:108B4000104078000030A10081B9200080487800F2
:108B500060B72000104078008080FB00E08120009A
:108B600000804000104078004B00070080B92000D2
:108B7000104078000080FB004400DE00614060008F
:108B8000614060004601DD00A12C2000914078008A
:108B9000F0CBB30000C0600002407000CAE2B70032
:108BA0000080FA00000006000000FA008E000700B6
:108BB0000080FA00000006000400FA00000F7800B0
:108BC0001E007800100798001E009000E10F500072
:108BD0000C0032001E009000E10F5000040039002C
:108BE0001E009000E20F5000120032001D003700FE
:108BF00041032000D0CB2000789A02000000000042
:108C00001C0037007100200050592000789A0200A3
:108C100000000000F1002000C01E2100789A020030
:108C20000000000011C0B3000040EB0090000700FE
:108C3000100037007100200050592000789A02007F
:108C400000000000F1002000C01E2100789A020000
:108C50000000000011C0B30010C0B3008400070082
:108C60000400370041022000C0202000789A020052
:108C7000000000000080FA00000006000000FA007A
:108C800001012000A0042100789A020000000000E9
:108C90000080FA00000006000200FA00004F780091
:108CA00041E2A90080B820001040780068406000D0
:108CB0000004E00004003200CEE2A800CF02A800C9
:108CC000CEC2A80003003700CEE2A900CF02A9005F
:108CD000CEC2A900816A20009140780000CEB30086
:108CE00000C060007040B300A8E6B700916C20009F
:108CF0009140780000CEB30000C060007040B30027
:108D0000C9E6B700816C20009140780000CEB30026
:108D100000C060000034A000C8E6B700CAC2A800C6
:108D2000C8C2A900C902A900C8E2A800C922A900B6
:108D30001E80FB001012880042A2A80080B920000B
:108D40001040780061406000614060004601DD0035
:108D50002124200091407800F0CBB30000C06000D7
:108D60000240700042E2B70080B920001040780055
:108D70000080FB000000D1006140600061416000A4
:108D80003124200091407800E0CFB30000C06000A3
:108D90000240700043E2B70080B920001040780024
:108DA0000080FB004200DE00614060006140600026
:108DB000004140003124200091407800D0CFB30022
:108DC00000C060000240700043E2B7000000EB000A
:108DD000201288000000EB000012880041E2A80089
:108DE0000080FA00000006000000FA0041E2A9003D
:108DF000A8C6BF00F041B300A8E6B700916C200000
:108E00009140780000CEB30000C06000C9E6B70012
:108E1000816C20009140780000CEB30000C060005B
:108E2000C8E6B700CEE2A900CF02A900CEC2A900D1
:108E30000080FA00000006000200FA00004F7800EF
:108E40001E80FB004012880085C0BF0064406000A7
:108E50000004E000FCFF320040128000004F780068
:108E60008540A9001E80FB000080FA00000006007B
:108E70000400FA00204798003147980010C0B30062
:108E8000004F7800DA71020000000000D6FF0700F2
:108E90007B0007002E4090000004E00002003A0032
:108EA00042E2A80062E2A8002E409000E14F50008C
:108EB00003003E0041E2A80061E2A8000000370084
:108EC0001E04E00009003A00CAC2BF000044B2001C
:108ED0000004E00005003200D0C5B300E8710200D4
:108EE0000000000010C0B300004F780040C2BF0077
:108EF0000042B2000004E0002F003A0060C2BF0050
:108F00000042B2000004E0002B003A004012800052
:108F10001047980010C0B3009E4F100005003A00A3
:108F2000B0C5B300E8710200000000000040EB0093
:108F3000004F78003E4090000004E0000500320041
:108F40001E4090000080FB00FA6F0200000000004D
:108F500006003700C0C5B300E87102000000000041
:108F60001E409000E87102000000000040138000E5
:108F7000104798003E4090000004E0000B003200D3
:108F800080C2B300E8710200000000001E409000A3
:108F90000080FB00FA6F02000000000090C2B300E6
:108FA000E871020000000000030037001E4090003E
:108FB000E87102000000000040C2BF000044B2009F
:108FC0000004E00004003A0060C2BF000044B200A8
:108FD0000004E0000A003200CA82A9003E4090006E
:108FE0000004E00003003200A09F2800026D020090
:108FF0000000000040C2A90060C2A90013003700B1
:10900000187202000000000022C2BF006140600030
:109010000004E000AAFF3200311180002007200088
:10902000808F500003003A0041E2A90061E2A900EC
:10903000A3FF37003E4090000004E0000300320030
:10904000B0A02800026D0200000000008B000700A5
:1090500081C6BF00F041B30081E6B70060B72000D1
:10906000104078008080FB00E081200000804000FC
:109070001040780008FF07000080FA00000006009A
:109080000000FA00C8C2A800C902A800C8E2A800EF
:10909000C922A800A16A20009140780000CEB30048
:1090A00000C060006040B300AAE6B700E16A20009B
:1090B0009140780000CEB30000C060006040B30073
:1090C000AEE6B700816A20009140780000CEB30080
:1090D00000C060009040B300A8E6B700916A20008D
:1090E0009140780000CEB30000C060000034A000C2
:1090F000A9E6B700C16A20009140780000CEB30015
:1091000000C060007040B300ACE6B700D16A200038
:109110009140780000CEB30000C060000034A00091
:10912000ADE6B70060B72000104078008080FB00FB
:10913000E081200000804000104078000080FB00AB
:109140001012880080B92000104078006140600053
:10915000614060004601DD0021242000914078003C
:10916000F0CBB30000C060000240700042E2B700E4
:1091700080B92000104078000080FB000000D10082
:10918000614060006141600031242000914078001E
:10919000E0CFB30000C060000240700043E2B700BF
:1091A0000000EB00201288000000EB000012880095
:1091B00060B72000104078008080FB00E081200034
:1091C00000804000104078000080FB0010138800F1
:1091D00080B920001040780061406000614060006C
:1091E0004601DD002126200091407800F0CBB3003D
:1091F00000C060000240700062E2B70080B9200049
:10920000104078000080FB000000D1006140600049
:10921000614160003126200091407800E0CFB3002A
:1092200000C060000240700063E2B7000000EB0085
:10923000201388000000EB00001388000000EB0002
:10924000401288000000EB00401388004322A90070
:109250006322A9004362A80042A2A9006362A80099
:1092600062A2A90040C2A90060C2A9004402A800ED
:109270006402A8000080FA00000006000000FA0066
:1092800041E2A9004362A90061E2A9006362A9006A
:10929000AAC6BF00F041B300AAE6B700AEC6BF0041
:1092A000F041B300AEE6B700A8C6BF00F041B3007E
:1092B000A8E6B700A9C6BF00F041B300A9E6B70011
:1092C000ACC6BF00F041B300ACE6B700ADC6BF000E
:1092D000F041B300ADE6B7000080FA0000000600E0
:1092E0000000FA00C0A02800D66C020000000000B8
:1092F0000080FA00000006000A00FA00881F7800CB
:1093000011C0B30060B720000148780080B9200088
:10931000104078000000A10081B92000804878004A
:1093200080B92000104078000010A00081B9200012
:109330008048780080B92000104078000020A1000B
:1093400081B920008048780080B820001040780063
:109350000030A00081B820008048780060B720006D
:10936000104078008080FB002082200000804000B8
:109370001040780048FE0700D9FF070000003700C2
:1093800022C2BF00614060000004E000FCFF320028
:10939000301180008040780060B9200001487800DA
:1093A00060B92000104078000080FB004400DE001F
:1093B0008040780050B920000148780050B9200062
:1093C000104078000080FB00400798004E0090009D
:1093D000E40F5000FA0032004E009000E40F5000FD
:1093E00007003C004E0090000000E0000B0032003F
:1093F0004E009000E10F5000CB0032005C013700BE
:109400004E009000E60F5000F50032004E00900034
:10941000E80F5000070132005501370060B9200005
:10942000104078000080FB00300798003E0090005C
:10943000E30F50002A0032003E009000E30F50007E
:109440000A003C003E009000E10F50001A0032007C
:109450003E009000E10F500019003C003E009000DB
:109460000000E00012003200AB0037003E00900028
:10947000ED0F5000220032003E009000ED0F500032
:1094800004003C003E009000E40F50003100320028
:10949000A10037003E009000EE0F50001F00320088
:1094A0003E009000EF0F5000230032009A0037007A
:1094B0004DFE07003201370089FF0700B0FF37007B
:1094C00060168000F1FB2F0001006000601688002C
:1094D00010C0B3003271020000000000A8FF370086
:1094E00060168000010420000100700060168800F2
:1094F00010C0B3003271020000000000A0FF37006E
:109500008040EB0020C0B30059FE070010C0B3003C
:10951000327102000000000099FF37008040EB002C
:109520000040EB0052FE070010C0B3003271020091
:109530000000000092FF37008040EB0010C0B30035
:109540004BFE070010C0B3003271020000000000A3
:109550008BFF370022C2BF00614060000004E000C2
:10956000FCFF320030118000100798001E009000B0
:109570004800DD001007980022C2BF006140600073
:109580000004E000FCFF3200301180009E009000DB
:10959000008070001007980022C2BF006140600088
:1095A0000004E000FCFF320030118000000F780062
:1095B0001E0078004800DD00000F780022C2BF00C6
:1095C000614060000004E000FCFF320030118000C8
:1095D0001E0F70009E009000F0FF2000808F500052
:1095E00003003E00F0FF20009E0F10000400360034
:1095F0000040EB00327102000000000060FF370005
:109600000000EB00200798000C00370022C2BF00CA
:10961000614060000004E000FCFF32007140800007
:109620002E0090008080400030118000804878003B
:109630002E0090000000E80020079800AE00900087
:109640001E009000808F5000F0FF3900CAC2A900B0
:109650000000EB00200798000800370071408000F0
:109660002E0090000080400010407800F2FD0700BE
:109670002E0090000000E80020079800AE00900047
:109680001E009000808F5000F4FF39000000EB00B6
:109690002007980009003700714080002E009000DC
:1096A0000084400000C0EB00E3FD0700004C7800A0
:1096B0002E0090000000E800200798002E00900087
:1096C0009E0F5000F4FF3900CAC2A80010C0B300BA
:1096D00032710200000000000000EB00200798003B
:1096E00009003700714080002E009000008040008B
:1096F0001040780032710200000000002E0090003F
:109700000000E800200798002E0090009E0F5000F7
:10971000F4FF39001AFF37000040EB0032710200FD
:109720000000000016FF370060B92000904078006C
:10973000F0C0B30080C0600060B92000014878002C
:1097400060B92000104078008040E80060B9200037
:109750000148780010C0B300327102000000000020
:109760008040EB0040B92000014878000D00370030
:1097700022C2BF00614060000004E000FCFF320034
:1097800030118000ACFD07003271020000000000C3
:1097900040B92000104078008040E80040B9200027
:1097A0000148780040B920009040780060B920005E
:1097B0001040780080CF5000EDFF3900F0FE3700F8
:1097C00060B9200010407800D09C0200000000002A
:1097D00010C0B3003271020000000000E8FE370044
:1097E00060B920009040780070C0B30080C0600075
:1097F00060B920000148780060B9200090407800EE
:1098000060B720000148780060B720001040780061
:109810008080FB0020822000008040001040780003
:109820001DFD070010C0B3003271020000000000EF
:10983000D3FE370080B92000104078000000A1005E
:1098400081B920008048780080B92000104078005D
:109850000010A10081B920008048780080B9200064
:10986000104078000020A10081B9200080487800D5
:1098700080B82000104078000030A10081B820009E
:109880008048780060B92000104078000080FB001C
:109890004200DE00610060000004E00005003200CC
:1098A00080B92000104078000000A00081B920009D
:1098B0008048780060B92000104078000080FB00EC
:1098C0000000D100610060000004E00005003200EB
:1098D00080B92000104078000010A00081B920005D
:1098E0008048780060B92000104078000080FB00BC
:1098F000610060000004E0000500320080B9200033
:10990000104078000020A00081B920008048780035
:1099100060B92000104078000080FB004300DE00AA
:109920000000A200610060000004E00005003200B9
:1099300080B82000104078000030A00081B82000DE
:109940008048780060B72000104078008080FB00DD
:10995000208220000080400010407800CEFC0700EC
:1099600010C0B300327102000000000084FE370016
:109970000040EB00327102000000000080FE370062
:109980004F0478000080FA00000006000400FA008E
:109990002E9C0200000000000004E00022003200C3
:1099A00032C2BF00684060000004E00004003200E2
:1099B0003100200010CF2000EE99020000000000CE
:1099C00032C2BF00644060000004E00004003200C6
:1099D0003100200040CF2000EE990200000000007E
:1099E0001C9C020000000000004F780032C2BF0043
:1099F000624060000004E00008003200F100200036
:109A000070CF2000EE99020000000000901180004D
:109A1000D1FF2F0001006000901188001E80FB0024
:109A20001007980006003700F100200060D02000E9
:109A3000EE990200000000000000EB001007980003
:109A40001E0090000080FA00000006000200FA00EC
:109A5000000F78001E007800089C02000000000043
:109A6000001020000080FA00000006000000FA004C
:109A700001022000C0DB2000EE990200000000007F
:109A800060B72000104078006E6F020000000000F8
:109A900000C2B300327102000000000060B7200075
:109AA00010407800E94F500007003A00C0118000D4
:109AB000106F02000000000000C2B300327102000B
:109AC000000000000C00370060B720001040780054
:109AD0000080FB0080004000A0B02000008040001B
:109AE00010007800106F02000000000000C2B300F8
:109AF0003271020000000000A0DD2000104078005C
:109B0000634060006E6F02000000000000C2B300FE
:109B10003271020000000000A0DD2000104078003B
:109B20000080FB004200DE00614060006E6F0200BA
:109B30000000000000C2B30032710200000000000B
:109B4000A0DD2000104078000080FB004300DE0014
:109B5000614060006E6F02000000000000C2B300B0
:109B6000327102000000000080B820001040780030
:109B70000080FB004300DE00614060006E6F020069
:109B80000000000000C2B3003271020000000000BB
:109B900031002000F0AD2000EE990200000000002E
:109BA0000080FA00000006000C00FA002C1A0200E7
:109BB0000000000056160200000000005007980048
:109BC0005E009000EA0F500005003A002C1A0200D7
:109BD000000000005616020000000000000F780090
:109BE0002C1A0200000000005616020000000000BF
:109BF000400798002C1A02000000000056160200D0
:109C000000000000300798002C1A0200000000003D
:109C10005616020000000000200798002C1A0200CF
:109C20000000000056160200000000001007980017
:109C30005E0090000000E000090034005E0090002B
:109C4000EA0F500006003C005E0090000040E90072
:109C50008040780060B7200001487800020037009B
:109C60000000EB00500798004E0090000000E0005C
:109C70000F0034004E009000E40F50000C003C0038
:109C80004E0090000040E900E3406000A0DD2000AD
:109C90001040780063C16000C1CFB3000140600094
:109CA00002407000A1DD20008048780002003700EB
:109CB0000000EB00500798003E0090000000E0001C
:109CC000100034003E009000E20F50000D003C00F8
:109CD0003E0090000040E90061416000A0DD2000EE
:109CE00090407800614061004201DD00B0CFB300D8
:109CF00080C0600082C07000A0DD200001487800B4
:109D0000020037000000EB00500798002E00900082
:109D10000000E000100034002E009000E20F500020
:109D20000D003C002E0090000040E9006141600001
:109D3000A0DD200090407800614061004301DD001B
:109D400070CFB30080C0600082C07000A0DD200032
:109D500001487800020037000000EB00500798002F
:109D60001E0090000000E000100034001E00900073
:109D7000E20F50000D003C001E0090000040EA0081
:109D80006141600080B8200090407800614061002F
:109D90004301DD0070CFB30080C0600082C070005E
:109DA00080B8200001487800020037000000EB0076
:109DB000500798005E0090000000E00073003A0039
:109DC0000000EB0060698800D10820003087200087
:109DD000789A0200000000008001EB00A200200041
:109DE0001100200010002000A21C02000000000052
:109DF0000040E9008040780060B72000014878000A
:109E000060B7200010407800E94F50000B003A0086
:109E1000C1012000001B2100789A02000000000010
:109E20008001EB00F2FF270011002000200220003B
:109E3000A21C020000000000000F78004105200075
:109E400050D12000EE990200000000008001EB00DC
:109E5000420020001100200010002000A21C02007F
:109E6000000000000040E900E3406000A0DD2000A9
:109E70001040780063C16000C1CFB30001406000B2
:109E800002407000A1DD200080487800110220000F
:109E900090D62000EE990200000000008001EB0047
:109EA000220020001100200010002000A21C02004F
:109EB000000000000040E90061416000A0DD2000DA
:109EC00090407800614061004201DD00B0CFB300F6
:109ED00080C0600082C07000A0DD200001487800D2
:109EE00021032000A0D82000EE990200000000000D
:109EF0008001EB0022002000110020001000200053
:109F0000A21C0200000000000040E9006141600066
:109F1000A0DD200090407800614061004301DD0039
:109F200070CFB30080C0600082C07000A0DD200050
:109F300001487800F1042000B0932000789A0200D4
:109F4000000000008001EB00220020001100200032
:109F500010002000A21C0200000000000040EA00E7
:109F60006141600080B8200090407800614061004D
:109F70004301DD0070CFB30080C0600082C070007C
:109F800080B820000148780001003700B7FE0700C4
:109F900060B7200010407800E94F50001C003A00E4
:109FA000A0DD2000104078000080FB004200DE00B1
:109FB0006140600080417800A0DD20001040780002
:109FC0006340600080427800A0DD200010407800EF
:109FD0000080FB004300DE0061406000004178002B
:109FE00080B82000104078000080FB004300DE00B5
:109FF00061406000804078001E00780003427800D5
:10A00000854178005C9B02000000000022003700C0
:10A01000A0DD2000104078000080FB004200DE0040
:10A020006140600000417800A0DD20001040780011
:10A030006340600080417800A0DD2000104078007F
:10A040000080FB004300DE00614060008042780039
:10A0500080B82000104078000080FB004300DE0044
:10A06000614060000043780060B720001040780035
:10A070000080FB0080004000A0B020000080400075
:10A080001000780002427800054178008640780090
:10A090005C9B020000000000E09B0200000000004A
:10A0A000C111800040118000808F500004003100F9
:10A0B00001022000C01C2100789A0200000000006C
:10A0C0000080FA00000006000000FA00EC9B02008D
:10A0D000000000000080FA00000006000400FA0002
:10A0E000000F78001E007800100798001E009000F6
:10A0F000E10F50000C0032001E009000E10F5000F4
:10A10000040039001E009000E20F50003D003200B4
:10A110005900370031052000C0DD2000EE99020013
:10A120000000000058003700B1002000F0E22000DD
:10A13000789A020000000000D1002000A0E3200077
:10A14000789A0200000000001E9B02000000000040
:10A150000000E0004C00320090118000D1FF2F0081
:10A1600001006000901188000000370032C2BF007B
:10A17000614060000004E0000600320023C2BF001E
:10A18000624060000004E00002003A00B01180006C
:10A190002011880022C2BF00614060000004E0007E
:10A1A0000600320033C2BF00624060000004E000DD
:10A1B00002003A0030118000A011880032C2BF00B6
:10A1C000624060000004E00004003A0022C2BF00C8
:10A1D000624060000004E000E4FF32009111800062
:10A1E000D0FF2F00008060009011880011118000C6
:10A1F000D0FF2F000080600010118800CA82A900E3
:10A20000DAFF3700E100200070E42000789A0200B5
:10A2100000000000F1002000C01E2100789A02001A
:10A220000000000090118000D1FF2F0001006000AD
:10A230009011880032C2BF00614060000004E0005D
:10A240000600320023C2BF00624060000004E0004C
:10A2500002003A00B01180002011880022C2BF0025
:10A26000614060000004E000F2FF32003011800025
:10A27000000F78000400370041022000C0202000B9
:10A28000789A0200000000000080FA00000006003A
:10A290000000FA0091118000D0FF2F0000806000C4
:10A2A00090118800A0DD2000104078000040A00040
:10A2B000A1DD20008048780080B8200010407800A0
:10A2C0000010A00081B8200080487800C101200063
:10A2D00050E52000789A0200000000000080FA009B
:10A2E000000006000000FA00A0DD20001040780009
:10A2F0000040A100A1DD20008048780080B8200047
:10A30000104078000010A10081B82000804878003B
:10A310004101200010E72000789A020000000000B0
:10A320000080FA00000006000200FA000000EB00C6
:10A33000000F780035003700A0DD200010407800C5
:10A34000704060000004E0002C003200A0A3280050
:10A35000026D020000000000610020006069200022
:10A36000EE9902000000000032C2BF0068406000A9
:10A370000004E000040032003100200010CF200073
:10A38000EE9902000000000032C2BF00644060008D
:10A390000004E000040032003100200040CF200023
:10A3A000EE990200000000001C9C0200000000006A
:10A3B0000080FB00C69602000000000032C2BF0011
:10A3C000624060000004E00008003200F10020005C
:10A3D00070CF2000EE990200000000009011800074
:10A3E000D1FF2F000100600090118800A0A3280079
:10A3F000026D020000000000020037001C9C0200F9
:10A400000000000010002000000F78002E9C0200C9
:10A41000000000000004E000C7FF3A001E007800C2
:10A420000080FA00000006000000FA00B1002000E1
:10A4300010092100789A0200000000000080FA0054
:10A44000000006000000FA00B0A32800D66C02004D
:10A45000000000000080FA00000006000400FA007E
:10A46000A0DD2000104078000000A1000010A10035
:10A47000A1DD200080487800A0DD20001040780099
:10A480000020A100A1DD200080487800A0DD200090
:10A49000104078000030A100A1DD20008048780045
:10A4A00080B82000104078000030A00081B8200063
:10A4B00080487800F0588000A06E8800A0DD200061
:10A4C000104078000040A100A1DD20008048780005
:10A4D000A0DD2000104078000080FB004200DE007C
:10A4E0006140600080417800A0DD200010407800CD
:10A4F0006340600080427800A0DD200010407800BA
:10A500000080FB004300DE006140600000417800F5
:10A5100080B82000104078000080FB004300DE007F
:10A520006140600080407800A06E800003427800A7
:10A53000854178005C9B020000000000E09B020067
:10A5400000000000BFFF0700000037002E9C020043
:10A55000000000000004E0000C003200A0DD20003C
:10A5600010407800704060000004E00005003200F8
:10A570001C9C02000000000032710200000000007C
:10A58000020037001C9C02000000000032C2BF0025
:10A59000624060000004E00004003200901180007E
:10A5A000D1FF2F00010060009011880022C2BF007F
:10A5B000614060000004E000E4FF320030118000E0
:10A5C0008040780080DD20000148780080DD200098
:10A5D000104078000080FB004400DE0080407800DE
:10A5E00070DD20000148780070DD20001040780008
:10A5F0000080FB00100798001E009000E40F500040
:10A60000D00032009E009000E48F500007003C0014
:10A610001E0090000000E0000F0032009E0090003D
:10A62000E18F50009F0032008A0137001E00900029
:10A63000E60F5000CB0032009E009000E68F5000E5
:10A64000840135009E00900068805000E10F5000AA
:10A6500080013E00FB00370080DD200010407800C4
:10A660000080FB00000F78001E007800E20F500011
:10A67000190032009E007800E28F500007003C0075
:10A680001E0078000000E0000E0032009E007800FE
:10A69000E18F50000E0032007E0037001E0078006F
:10A6A000E70F5000260032009E007800EF8F500028
:10A6B0005B0032001E007800E30F500017003200EC
:10A6C00074003700EC9B02000000000065013700B9
:10A6D0005CFF07009DFF370010C0B300327102001D
:10A6E0000000000032C2BF00624060000004E000D1
:10A6F0000400320090118000D1FF2F0001006000A3
:10A7000090118800A0DD2000104078000040A000DB
:10A71000A1DD2000804878008CFF3700A0DD2000FC
:10A72000104078000040A100A1DD200080487800A2
:10A7300010C0B300327102000000000083FF370038
:10A7400010C0B3003271020000000000EC9B020058
:10A750000000000022C2BF00614060000004E00071
:10A76000FCFF3200301180004800DD00A06E880040
:10A7700010C0B300327102000000000022C2BF000E
:10A78000614060000004E000FCFF3200A16E800028
:10A790003011800000807000A06E8800A0DD2000D5
:10A7A000104078000080FB004200DE006140600045
:10A7B00080417800A0DD20001040780063406000F8
:10A7C00080427800A0DD2000104078000080FB006F
:10A7D0004300DE00614060000041780080B8200046
:10A7E000104078000080FB004300DE006140600004
:10A7F00080407800A06E8000034278008541780098
:10A800005C9B020000000000E09B020000000000D2
:10A8100010C0B30032710200000000004BFF37008F
:10A8200010C0B300327102000000000090118000DF
:10A83000D1FF2F0001006000901188000000370058
:10A8400032C2BF00614060000004E0000600320038
:10A8500023C2BF00624060000004E00002003A0032
:10A86000B01180002011880022C2BF00614060004A
:10A870000004E000F2FF320033C2BF00624060001B
:10A880000004E000EEFF3A0030118000A0118800C3
:10A89000EBFF37000040EB003271020000000000C7
:10A8A0002AFF370080DD200090407800F0C0B30020
:10A8B00080C0600080DD20000148780080DD20003D
:10A8C000104078008040E80080DD200001487800DA
:10A8D00010C0B30032710200000000008040EB00A5
:10A8E00060DD2000014878000F00370022C2BF0061
:10A8F000614060000004E000FCFF32003011800085
:10A90000089C02000000000010C0B3003271020079
:10A910000000000060DD2000104078008040E8006A
:10A9200060DD20000148780060DD20009040780064
:10A9300080DD20001040780080CF5000EBFF390010
:10A9400002FF370080DD200010407800D09C02001C
:10A950000000000010C0B3003271020000000000CF
:10A96000FAFE370080DD200090407800F0C0B30090
:10A9700080C0600080DD20000148780080DD20007C
:10A9800010407800EA4F500003003600A1C0B30029
:10A9900080DD20000148780080DD20001040780034
:10A9A0000080FB0080004000E0B1200000804000FB
:10A9B00010007800A06E8800EC9B020000000000F0
:10A9C000A0DD2000104078000080FB004200DE0087
:10A9D0006140600080417800A0DD200010407800D8
:10A9E0006340600080427800A0DD200010407800C5
:10A9F0000080FB004300DE00614060000041780001
:10AA000080B82000104078000080FB004300DE008A
:10AA10006140600080407800A06E800003427800B2
:10AA2000854178005C9B020000000000E09B020072
:10AA30000000000010C0B3003271020000000000EE
:10AA4000C2FE3700A0DD2000104078000000A10009
:10AA50000010A100A1DD200080487800A0DD2000CA
:10AA6000104078000020A100A1DD2000804878007F
:10AA7000A0DD2000104078000030A100A1DD200002
:10AA80008048780080B82000104078000030A10095
:10AA900081B820008048780080DD200010407800D8
:10AAA0000080FB004300DE00610060000004E00065
:10AAB0000D003200A0DD20001040780063406000EF
:10AAC0000014A000E3406000A0DD200010407800EA
:10AAD00063C16000C1CFB30001406000024070005C
:10AAE000A1DD20008048780080DD20001040780043
:10AAF0000080FB004200DE00610060000004E00016
:10AB00000D003200A0DD200010407800634060009E
:10AB10000004A000E3406000A0DD200010407800A9
:10AB200063C16000C1CFB30001406000024070000B
:10AB3000A1DD20008048780080DD200010407800F2
:10AB40000080FB000000D100610060000004E00014
:10AB500005003200A0DD2000104078000020A00099
:10AB6000A1DD20008048780080DD200010407800C2
:10AB70000080FB00610060000004E000050032007E
:10AB8000A0DD2000104078000030A000A1DD2000F2
:10AB90008048780080DD2000104078000080FB00B5
:10ABA0004400DE000000A200610060000004E0003C
:10ABB0000500320080B82000104078000030A0006E
:10ABC00081B8200080487800EC9B02000000000063
:10ABD000A0DD2000104078000080FB004200DE0075
:10ABE0006140600080417800A0DD200010407800C6
:10ABF0006340600080427800A0DD200010407800B3
:10AC00000080FB004300DE006140600000417800EE
:10AC100080B82000104078000080FB004300DE0078
:10AC20006140600080407800A06E800003427800A0
:10AC3000854178005C9B020000000000E09B020060
:10AC40000000000010C0B3003271020000000000DC
:10AC50003EFE37000040EB003271020000000000B1
:10AC60003AFE37000080FA00000006000000FA00FB
:10AC700018990200000000000080FB000080FA002C
:10AC8000000006000200FA00000F78001E007800A5
:10AC90008098020000000000001020000080FA00F0
:10ACA000000006000000FA007E990200000000008B
:10ACB0000080FB000080FA00000006000000FA009F
:10ACC00060BA200010407800DE980200000000000A
:10ACD0000080FA00000006000000FA0060BA2000C0
:10ACE000104078000080FB000080FA0000000600A1
:10ACF0000000FA008040EB0060BA200001487800B4
:10AD000041022000B0002000789A020000000000FC
:10AD10000080FA00000006000000FA0011C0B30035
:10AD200060BA20000148780041022000B0002000F5
:10AD3000789A0200000000000080FA00000006007F
:10AD40000000FA0080B82000104078000030A00019
:10AD500081B82000804878008040EB0080BB200054
:10AD600001487800C922A800CB22A900E1022000F6
:10AD7000F0022000789A0200000000000080FA0033
:10AD8000000006000400FA00881F7800000F780019
:10AD90001E00E00044003200200320009E0F10003F
:10ADA00041003E001E0FE90080BB200010407800EB
:10ADB0000080FB009E0F500005003E009102200025
:10ADC000D0052000789A02000000000063013700DF
:10ADD000E100200060082000EE9902000000000061
:10ADE0001E0078000040E8006E6F020000000000C6
:10ADF00000A22800D66C0200000000008040EB009A
:10AE000020BB2000014878001F0037001E01780099
:10AE100020BB2000104078008080FB004310DD0044
:10AE20008100400090BB200000804000104078006E
:10AE30000080FB00C69602000000000000C2B300C4
:10AE400032710200000000001E01780020BB2000CB
:10AE5000104078008080FB004310DD00810040003E
:10AE600090BB2000008040001040780080980200D5
:10AE70000000000020BB2000104078008040E80067
:10AE800020BB20000148780020BB20001040780043
:10AE9000E74F5000DDFF360030A22800026D0200AF
:10AEA000000000002D0137001E00780010079800F8
:10AEB000500520009E009000808F5000110132004C
:10AEC000500520009E009000808F500008003E003A
:10AED0001E0090000000E00012003200300320004D
:10AEE0009E009000808F5000DD0032001701370077
:10AEF000C00E20009E009000808F50006300320042
:10AF0000000F20009E009000808F50005F003200F4
:10AF1000C00C20009E009000808F50000201320083
:10AF20000A013700D100200040092000789A020071
:10AF30000000000071012000100A2000789A020031
:10AF40000000000080BB2000104078000004E000FA
:10AF500005003A0091022000D0052000789A0200F6
:10AF600000000000440037008040EB0030BB2000B0
:10AF7000014878003A00370000C2B3003271020085
:10AF80000000000030BB2000104078000040E800C6
:10AF90006E6F02000000000040A22800D66C020084
:10AFA000000000008040EB0020BB2000014878003A
:10AFB0001600370030BB2000104078000081FB00F5
:10AFC00020BB2000104078008080FB004310DD0093
:10AFD0008100400090BB20000080400010407800BD
:10AFE0000080FB00C69602000000000000C2B30013
:10AFF000327102000000000020BB200010407800E9
:10B000008040E80020BB20000148780020BB2000E1
:10B0100010407800E74F5000E6FF36006100200046
:10B02000800B2000EE9902000000000030BB2000E1
:10B03000104078000080FB00C300DD0090BB2000C2
:10B040000080400010407800F700070030BB20006F
:10B05000104078008040E80030BB200001487800B4
:10B0600080BB20009040780030BB2000104078006A
:10B0700080CF5000C0FF3E00310D2000E00B2000CB
:10B08000789A020000000000B40037001E0078002B
:10B0900080407800C083200001487800C00E200066
:10B0A0009E0F100005003A00310120001019200009
:10B0B000789A02000000000004003700D100200050
:10B0C000401A2000789A0200000000007101200060
:10B0D000100A2000789A0200000000008040EB0077
:10B0E00020BB2000014878000A010700804078005A
:10B0F00030BB2000014878008040EB0080BB20007E
:10B10000014878004D00370000C2B30032710200E0
:10B110000000000020BB2000104078000040E80044
:10B120006E6F02000000000040A22800D66C0200F2
:10B13000000000000000EB00805D88000D0037007B
:10B14000815D800090C020000080400010407800A9
:10B150000080FB00C69602000000000000C2B300A1
:10B160003271020000000000805D80000000E800F5
:10B17000805D8800805D8000E70F5000F0FF3600A2
:10B1800061002000800B2000EE990200000000000A
:10B1900090C0200010407800A300070020BB2000D2
:10B1A00010407800E94F50001B003E000000EB000B
:10B1B000805D88001000370080BB200010407800C0
:10B1C0008081FB00845D8000815D800090C0200054
:10B1D00000804000104178004318DD0084004000EA
:10B1E00090BB20000080400002487800805D800015
:10B1F0000000E800805D8800805D8000E70F50005F
:10B20000EDFF360080BB2000104078008040E80051
:10B2100080BB20000148780020BB2000104078004F
:10B220008040E80020BB200001487800C7000700EC
:10B230008040780030BB20000148780030BB2000FF
:10B24000104078000004E000AFFF3A00B102200097
:10B25000101B2000789A0200000000003F00370019
:10B260004800070011012000C01D2000EE990200D7
:10B270000000000030C3B30080980200000000000E
:10B280000000EB00805D880014003700885D8000BE
:10B2900018990200000000008040780070BA200079
:10B2A0000000440001487800815D800070BA2000F1
:10B2B00000804000104078000080FB00C69602002D
:10B2C0000000000000C2B300327102000000000064
:10B2D000805D80000000E800805D8800805D800067
:10B2E000E70F5000E9FF360030A22800026D02008F
:10B2F0000000000070BA2000104078004A000700EB
:10B30000160037001F00070001012000D01E20009A
:10B31000789A02000000000050C5B3008098020037
:10B32000000000000D00370016000700F1002000AB
:10B33000D01F2000789A020000000000C0CCB300AB
:10B340008098020000000000040037004102200045
:10B35000C0202000789A0200000000004F0478000E
:10B360000080FA00000006000000FA0091002000B2
:10B3700080082100789A0200000000000080FA0096
:10B38000000006000200FA00FA9702000000000028
:10B39000004F7800A100200000232000EE99020059
:10B3A000000000001E04E00005003A00310020000B
:10B3B00050BB2000789A02000000000018003700FF
:10B3C00091002000A0232000EE9902000000000060
:10B3D0001E80FB00610060000004E00004003200F9
:10B3E0005101200030242000EE99020000000000EE
:10B3F0001E80FB000000D100610060000004E0003E
:10B40000040032004101200080252000EE99020056
:10B410000000000030A22800026D020000000000C1
:10B420000080FA00000006000400FA00004F7800D7
:10B430001E80FB0010079800200220009E00900054
:10B44000808F50001E003200200220009E009000DD
:10B45000808F500007003C001E009000E40F500059
:10B460001C0032009E009000F08F50000A00320055
:10B4700022003700800220009E009000808F500044
:10B480000A003200D00220009E009000808F500001
:10B490001500320019003700B1012000C02620003D
:10B4A000789A02000000000018003700A101200077
:10B4B00070282000789A0200000000001300370076
:10B4C00051012000102A2000789A0200000000009C
:10B4D0000E00370081012000602B2000789A0200C6
:10B4E000000000000900370001012000E02C2000CE
:10B4F000789A02000000000004003700E1002000FC
:10B50000E02D2000EE990200000000000080FA000B
:10B51000000006000000FA008040EB0010C120008F
:10B52000014878008040EB0030C1200001487800DD
:10B530008040EB0020C1200001487800080007008F
:10B540000080FB000080FA00000006000000FA0006
:10B55000030007000080FB000080FA0000000600E6
:10B560000A00FA0010C0B300704798000040EB00DA
:10B57000604798000040EB005047980010C0B300AF
:10B58000104798000040EB00404798008040EB00D7
:10B5900040C120000148780030C1200010407800F0
:10B5A0000004E0009C003A00FA970200000000004E
:10B5B0000004E0000C0032008040EB0010C12000CD
:10B5C000014878008040EB0030C12000014878003D
:10B5D0008040EB0020C12000014878000000EB0013
:10B5E00040079800A1003700C08320001040780079
:10B5F00080980200000000007E9902000000000018
:10B60000304798007E990200000000002047980013
:10B610003E409000E14F500003003A002E40900061
:10B62000E14F500068003200BE4090002E40900074
:10B6300080CF500003003200BE409000014F7800E0
:10B640002600370010C12000904078007E40900016
:10B65000814F50000E0031005E4090008080FB0062
:10B6600090C0200000804000904078001E40900074
:10B6700080C060000040EB00004F78000104E00053
:10B680000C00320010C0B300004F780009003700F2
:10B6900010C12000904078000040EB00004F78007F
:10B6A0007E409000814F500002003A0010C0B3006D
:10B6B000004F78001E04E00008003A007E40900031
:10B6C000604798006E409000E84F500003003E0035
:10B6D00020C12000EE4090000148780010C0B30067
:10B6E0009E4F10000D003A005E4090000081FB006C
:10B6F0005E4090008080FB0090C0200000804000F1
:10B70000904078001E40900080C0700090C02000E3
:10B710000000410001487800110037005E409000B1
:10B720000082FB005E4090008080FB0090C0200003
:10B730000080400010407800804178001E41900059
:10B74000024078000080EA008180EA0000C06100C9
:10B750008040780090C0200000004200014878003E
:10B760001E407800DE980200000000007E4090003D
:10B770000040E800704798001E40900000404000E4
:10B78000104798001E4090000004E0000B003A00B3
:10B790005E4090008080FB0090C020000080400050
:10B7A00010407800920007005E4090000040E800E2
:10B7B0005047980010C0B300104798005E409000BA
:10B7C000E74F50008CFF3600FE40900000C4B300ED
:10B7D00080CF50001000360040C12000104078009B
:10B7E0000004E0000C003A0010C12000EE40900080
:10B7F0000148780010C12000104078000004E000EB
:10B8000003003A0011C0B30030C1200001487800A5
:10B8100010C0B300404798004E4090000004E00084
:10B820000400320090C02000104078000004E000C6
:10B830000B003A008040EB0010C120000148780066
:10B840008040EB0030C12000014878008040EB00D0
:10B8500020C12000014878000040EB0040479800DC
:10B860004E4090000080FB00400798004E00900082
:10B870000080FA00000006000E00FA000040EB0015
:10B88000404798000C0037004E4090000081FB00BC
:10B890004E4090008080FB0090C02000008040005F
:10B8A0009040780065004700017178004E4090009C
:10B8B0000040E800404798004E409000E74F50009D
:10B8C000F1FF360010C12000904078002147980019
:10B8D00030C12000904078001147980020C120001E
:10B8E000104F780001C4B30010C120000148780057
:10B8F0008040EB0030C120000148780018FF0700AD
:10B900000004E0001A00320010C0B3003047980075
:10B910000040EB0040479800110037004E40900077
:10B920008080FB0065004700614178004E40900038
:10B930008080FB0090C02000008040001040780014
:10B94000804F5100030032000040EB003047980068
:10B95000090037004E4090000040E8004047980042
:10B960004E409000E74F5000ECFF360002003700D9
:10B970000040EB00304798000040EB004047980043
:10B980000C0037004E4090000081FB004E409000BC
:10B990008080FB0065004700E140780090C02000F7
:10B9A00000004100014878004E4090000040E8004F
:10B9B000404798004E409000E74F5000F1FF36009E
:10B9C00010C12000AE4090000148780030C1200036
:10B9D0009E4090000148780020C120001E48780059
:10B9E0003E4090000080FB000080FA00000006004E
:10B9F0000200FA00004F780040C12000104078009B
:10BA00001E4068008080FB00D08320000080400042
:10BA10009040780040C120000148780040C12000DB
:10BA2000104078000080FB000080FA000000060053
:10BA30000000FA0060A22800D66C0200000000009E
:10BA40000080FA00000006000400FA00C922A800E5
:10BA5000CB22A900C8C2A90080B8200010407800FD
:10BA60000030A00081B820008048780080B8200015
:10BA7000104078000020A10081B8200080487800A4
:10BA8000EBFF07000000370022C2BF0061406000EA
:10BA90000004E000FCFF320030118000804078009C
:10BAA00070BB20000148780070BB20001040780077
:10BAB0000080FB004400DE008040780060BB200076
:10BAC0000148780060BB2000104078000080FB0037
:10BAD000100798001E009000E10F5000780032001F
:10BAE0009E009000E48F50009D0032001E009000E8
:10BAF0000000E00001003200A100370070BB200010
:10BB0000104078000080FB00000F78009E00780055
:10BB1000E28F5000170032001E007800E20F500044
:10BB200007003C009E0078000100E0009800320011
:10BB30001E007800E10F50000C0032005C0037005E
:10BB40009E007800E48F5000130032001E00780041
:10BB5000E40F5000560035009E00780068805000C9
:10BB6000E10F500052003E0010003700B0FF070008
:10BB7000C5FF3700FA9702000000000080407800FF
:10BB800040BB20000148780010C0B30032710200B1
:10BB900000000000BCFF3700189902000000000000
:10BBA0003271020000000000B7FF370010C0B30080
:10BBB000327102000000000070BB200010407800CD
:10BBC000E94F500004003A00C1CEB300C08320000A
:10BBD000014878000300370001CFB300C083200084
:10BBE000014878004BFE07008040780040BB2000F1
:10BBF00001487800190037008040EB0050BB20005E
:10BC0000014878000D00370050BB2000104078003C
:10BC10008080FB0090C02000008040001040780031
:10BC2000327102000000000050BB2000104078007C
:10BC30008040E80050BB20000148780050BB200045
:10BC400010407800E74F5000EFFF36003FFE07003E
:10BC50008040780040BB20000148780040BB2000B5
:10BC6000104078000004E000E3FF3A008040EB0061
:10BC700050BB2000014878000800370000C0EB00EE
:10BC8000327102000000000050BB2000104078001C
:10BC90008040E80050BB20000148780050BB2000E5
:10BCA00010407800E74F5000F4FF360076FF370071
:10BCB0000040EB00327102000000000072FF37000C
:10BCC00070BB200090407800F0C0B30080C06000DE
:10BCD00070BB20000148780070BB20001040780045
:10BCE0008040E80070BB20000148780010C0B3001D
:10BCF00032710200000000008040EB0050BB2000C9
:10BD0000014878000F00370022C2BF006140600088
:10BD10000004E000FCFF3200301180008098020037
:10BD20000000000010C0B3003271020000000000EB
:10BD300050BB2000104078008040E80050BB20003D
:10BD40000148780050BB20009040780070BB200074
:10BD50001040780080CF5000EBFF39004AFF3700D9
:10BD600070BB200010407800D09C02000000000052
:10BD700010C0B300327102000000000042FF370023
:10BD80000040EB0032710200000000003EFF37006F
:10BD90000080FA00000006000000FA0060A42800FD
:10BDA000D66C0200000000000080FA0000000600CF
:10BDB0000000FA000040EB00A48102000000000037
:10BDC0000040EB00A4810200000000000040EB00F6
:10BDD000A4810200000000000040EB00A4810200EA
:10BDE000000000000000EB00E08002000000000006
:10BDF0000000EB00E0800200000000000000EB000B
:10BE0000E0800200000000000080FA000000060050
:10BE10000C00FA0080B82000104078000030A0002C
:10BE200081B820008048780080B820001040780059
:10BE30000020A10081B820008048780011C0B30024
:10BE400060B720000148780081C0B30070B72000BF
:10BE50000148780021C0B300D0DE200001487800FE
:10BE600080C0EB0020C0B300807F02000000000013
:10BE7000C922A900C902A900C8E2A80010C0B300E5
:10BE80001082020000000000C3FF0700000037001E
:10BE900022C2BF00614060000004E000FCFF3200ED
:10BEA000301180008040780010DF200001487800C9
:10BEB00010DF2000104078000080FB004400DE000E
:10BEC0008040780000DF20000148780000DF20007B
:10BED000104078000080FB00300798003E00900082
:10BEE000E30F500014013200BE009000E38F5000B9
:10BEF0000A003C003E019000E10F5100A400320016
:10BF0000BE019000E18F5100F8003C003E0090001F
:10BF10000000E00012003200E5023700BE00900091
:10BF2000E68F50008E0232003E019000E60F510075
:10BF300004003C00BE019000E48F510080023200FA
:10BF4000DB0237003E009000E80F50009B023200F9
:10BF5000BE009000EA8F500031013200D402370059
:10BF600010DF2000104078000080FB006101B90064
:10BF70004207980053079800D000200001002000DD
:10BF80004E019000DE019000800F5100818F59001A
:10BF90007B003E004E009000DE009000006001003B
:10BFA000C70237000C0037000D00370012003700C1
:10BFB000170037001D00370023003700430037000B
:10BFC000470037004B00370051003700570037005B
:10BFD0005D003700630037006FFF0700ACFF3700DC
:10BFE0000E8002000000000010C0B3003271020099
:10BFF00000000000A6FF37004E8002000000000095
:10C0000010C0B3003271020000000000A0FF370032
:10C010000040EB00108202000000000010C0B300DE
:10C02000327102000000000099FF370010C0B30019
:10C03000108202000000000010C0B3003271020044
:10C040000000000092FF3700D0DE20001040780092
:10C05000E24F500006003A00348102000000000068
:10C0600080407800F0DE20000148780006003700AC
:10C07000F00F20006E800200000000008040780079
:10C08000F0DE20000148780080B8200010407800E1
:10C09000644060000004E00007003200F0DE200091
:10C0A00010407800AE970200000000008040780049
:10C0B000F0DE200001487800F0DE2000104078001B
:10C0C000327102000000000071FF3700828102001F
:10C0D0000000000032710200000000006CFF370019
:10C0E0002282020000000000327102000000000005
:10C0F00067FF370010C0B300C681020000000000D7
:10C1000010C0B300327102000000000060FF370071
:10C110000040EB00FE8102000000000010C0B300F0
:10C12000327102000000000059FF370010C0B30058
:10C13000FE8102000000000010C0B3003271020056
:10C140000000000052FF37000040EB00EC810200CD
:10C150000000000010C0B3003271020000000000B7
:10C160004BFF370010C0B300EC810200000000005C
:10C1700010C0B300327102000000000044FF37001D
:10C180000040EB00327102000000000040FF370069
:10C1900010DF200090407800F0C0B30080C0600045
:10C1A00010DF20000148780010DF200010407800E8
:10C1B0008040E80010DF20000148780010C0B30084
:10C1C00032710200000000008040EB00F0DE200031
:10C1D000014878003E00370022C2BF006140600085
:10C1E0000004E000FCFF3200301180008040780045
:10C1F000E0DE20000148780080B820001040780080
:10C20000644060000004E00007003200E0DE20002F
:10C2100010407800AE9702000000000080407800D7
:10C22000E0DE200001487800D0DE200010407800D9
:10C23000E24F500009003A00E0DE20001040780094
:10C240000080FB00E08002000000000010C0B3008E
:10C25000327102000000000018003700E0DE20000C
:10C26000104078000080FB006E800200000000009B
:10C2700080407800E0DE20000148780080B820008F
:10C2800010407800644060000004E00007003200C5
:10C29000E0DE200010407800AE97020000000000B1
:10C2A00080407800E0DE200001487800E0DE2000D9
:10C2B000104078003271020000000000F0DE200023
:10C2C000104078008040E800F0DE2000014878004F
:10C2D000F0DE20009040780010DF20001040780051
:10C2E00080CF5000BCFF3900E9FE370010DF20008E
:10C2F00090407800F0C0B30080C0600010DF2000E4
:10C300000148780010DF2000104078008040E800ED
:10C3100010DF20000148780010DF20001040780076
:10C32000C68102000000000010C0B300327102009C
:10C3300000000000D6FE370010DF2000904078009B
:10C34000F0C0B30080C0600010DF2000014878001A
:10C3500010DF2000104078008040E80010DF20004F
:10C360000148780010C0B3003271020000000000E4
:10C3700022C2BF00614060000004E000FCFF320008
:10C38000301180008040780000DF200001487800F4
:10C390008040EB00F0DE20000148780016003700F6
:10C3A00000DF2000104078000004E00004003D00A1
:10C3B00010C0B300A4810200000000000300370099
:10C3C0000040EB00A48102000000000000DF20001C
:10C3D00010407800004040008040780000DF2000DE
:10C3E00001487800F0DE2000104078008040E8002E
:10C3F000F0DE200001487800F0DE20009040780058
:10C4000010DF20001040780080CF5000E4FF39009A
:10C4100010C0B30032710200000000009CFE370023
:10C4200010DF2000104078000080FB0020079800FB
:10C43000400A2000AE009000808F500015003200AE
:10C44000500A20002E019000800F5100C5003200DC
:10C45000000A2000AE019000808F510001003200E0
:10C460003301370022C2BF00614060000004E000D9
:10C47000FCFF32003011800080407800C0DE2000D8
:10C480000148780010C0B3003271020000000000C3
:10C490007FFE3700C0DE2000104078000080FB00E7
:10C4A000100798001E009000E10F500004003200B9
:10C4B0009E009000E28F50003B003200A500370044
:10C4C00022C2BF00614060000004E000FCFF3200B7
:10C4D00030118000506F8800506F80006300B900F9
:10C4E000506F88000000EB00406F88000C003700A0
:10C4F00022C2BF00614060000004E000FCFF320087
:10C5000071408000406F80008080400030118000CA
:10C5100080487800406F80000000E800406F88008D
:10C52000416F8000506F8000808F5000F0FF390015
:10C530000000EB00406F880013003700714080005E
:10C54000406F8000008040000080E80010417800CB
:10C5500071408000406F8000008040000000E800D3
:10C560009041780071408000406F80000080400062
:10C57000104078008340780053010700406F80002E
:10C5800063004000406F8800416F8000506F800062
:10C59000808F5000E9FF390010C0B30032710200F3
:10C5A000000000003AFE370022C2BF006140600078
:10C5B0000004E000FCFF320030118000506F880062
:10C5C000506F80004200DD00506F88000000EB00DB
:10C5D000406F88000C00370022C2BF00614060003D
:10C5E0000004E000FCFF320071408000406F8000DA
:10C5F000808040003011800080487800406F8000CB
:10C600000000E800406F8800416F8000506F80009C
:10C61000808F5000F0FF39000000EB00406F880071
:10C62000440037000040EB00A4810200000000003D
:10C630000040EB00A4810200000000000040EB007D
:10C64000A4810200000000000040EB00A481020071
:10C650000000000071408000406F800000804000BA
:10C66000104078000080FB00E08002000000000025
:10C6700071408000406F8000008040000000E800B2
:10C68000104078000080FB00E08002000000000005
:10C6900071408000406F8000008040000080E80012
:10C6A000104078000080FB00E080020000000000E5
:10C6B00071408000406F80000080400063014000B6
:10C6C00071408000406F80000080400063004000A7
:10C6D000104078006F406000004978008040EB0017
:10C6E000F0DE20000148780006003700B0FD0700AA
:10C6F000F0DE2000104078008040E800F0DE2000EE
:10C700000148780071408000406F80000080400048
:10C710006300400090407800F0DE20001040780078
:10C7200080CF5000F1FF3E00406F80006400400069
:10C73000406F8800416F8000506F8000808F5000F4
:10C74000B8FF390010C0B3003271020000000000D1
:10C75000CFFD37000040EB00327102000000000006
:10C76000CBFD3700C0DE2000104078000080FB00C9
:10C77000000F78001E017800E10F51000400320024
:10C780009E017800E28F510045003200C0FD370065
:10C7900022C2BF00614060000004E000FCFF3200E4
:10C7A00030118000506F880022C2BF0061406000DD
:10C7B0000004E000FCFF320030118000804078006F
:10C7C00000DF2000014878000000EB00406F880087
:10C7D0002E00370000DF200090407800E0DE2000CF
:10C7E000014878008040EB00F0DE2000014878002E
:10C7F00019003700E0DE2000104078000080FB00C8
:10C80000610060000004E0000400320010C0B300CA
:10C81000A481020000000000030037000040EB008C
:10C82000A481020000000000E0DE2000104078003B
:10C830000080FB000000D10080407800E0DE200096
:10C8400001487800F0DE2000104078008040E800C9
:10C85000F0DE200001487800F0DE20001040780073
:10C86000E34F5000E3FF3600348102000000000077
:10C87000348102000000000032710200000000005C
:10C88000406F80000000E800406F8800416F80002A
:10C89000506F8000808F5000CEFF39007CFD370044
:10C8A00022C2BF00614060000004E000FCFF3200D3
:10C8B00030118000506F88000000EB00406F88004E
:10C8C0001600370022C0B30060B92000A10B200081
:10C8D000B7000700ED00070022C0B30060BB2D00C9
:10C8E000A10B2000B200070022C0B300603D2D0064
:10C8F000A10B2000AE000700E400070022C0B30037
:10C9000060BB2000A10B2000A9000700DF0007008A
:10C91000406F80000000E800406F8800416F800099
:10C92000506F8000808F5000E6FF390058FD3700BF
:10C930000040EB00327102000000000054FD37009F
:10C9400010DF200010407800D09C020000000000A2
:10C9500010C0B30032710200000000004CFD37002F
:10C9600010DF20009040780030C0B30080C060002D
:10C9700010DF20000148780010DF20009040780090
:10C9800060B720000148780060B720009040780030
:10C99000D0DE200010407800807F02000000000000
:10C9A00010C0B300108202000000000010C0B300ED
:10C9B000327102000000000035FD370080B8200011
:10C9C000104078000030A10081B820008048780035
:10C9D00010DF2000104078000080FB004300DE00E4
:10C9E0000000A200610060000004E00005003200C9
:10C9F00080B82000104078000030A00081B82000EE
:10CA00008048780021C0B300D0DE200001487800C3
:10CA100010DF2000104078000080FB004200DE00A4
:10CA2000610060000004E0000300320031C0B30088
:10CA3000D0DE20000148780080B820001040780047
:10CA40000020A10081B820008048780010DF20007D
:10CA5000104078000080FB000000D1006100600001
:10CA60000004E0000500320080B82000104078008B
:10CA70000020A00081B820008048780060B7200026
:10CA800090407800D0DE200010407800807F0200C7
:10CA90000000000010C0B30010820200000000007F
:10CAA00010C0B3003271020000000000F8FC370033
:10CAB0000040EB003271020000000000F4FC37007F
:10CAC0000080FA00000006000600FA0020479800E7
:10CAD00031479800424798002E4090000080FB00AC
:10CAE0004600DE00004F78000040EB001047980041
:10CAF000220037001E409000E34F50000C003A0027
:10CB00001E04E0000A00320010C0B300FE810200E3
:10CB1000000000001E80FB004C9702000000000097
:10CB20000040EB00FE810200000000001000370012
:10CB30002E4090000080FB00610060000004E000D7
:10CB40000400320010C0B300A48102000000000005
:10CB5000030037000040EB00A48102000000000049
:10CB60002E4090000080FB000000D100204798007C
:10CB70001E4090000040E800104798001E409000C2
:10CB8000E34F5000DBFF36003E4090000080FB008A
:10CB9000E0800200000000004E4090000080FB009A
:10CBA000E0800200000000000080FA0000000600A3
:10CBB0000800FA00100798002107980062479800C3
:10CBC0000040EB00A4810200000000000040EB00E8
:10CBD000A4810200000000000040EB00A4810200DC
:10CBE000000000000040EB00A481020000000000F3
:10CBF0001E009000AE970200000000000080FB00C5
:10CC0000E0800200000000001E009000AE009000D6
:10CC10004809DD004800DE0000007100C808DE00A1
:10CC2000AE970200000000000080FB00E0800200E0
:10CC3000000000001E009000AE0090004008DE00E2
:10CC400001002000AE970200000000000080FB0001
:10CC5000E0800200000000006E4090006F40600025
:10CC6000604798000040EB00004F7800020037005A
:10CC70004FFC07001E4FE8006E4090009E4F1000D2
:10CC8000FBFF39000080FA00000006000000FA00F7
:10CC900010C0B300A4810200000000000040EB00BF
:10CCA000A4810200000000000040EB00A48102000B
:10CCB000000000000040EB00A48102000000000022
:10CCC0000000EB00E0800200000000003481020060
:10CCD00000000000327102000000000034810200F8
:10CCE00000000000327102000000000030FC07006C
:10CCF0002FFC07000080FA00000006000200FA0086
:10CD0000005D80000000E0001200320000C2B300AD
:10CD100032710200000000003100200010442000A9
:10CD2000EE9902000000000000C2B3003271020060
:10CD300000000000F05C80000000E00003003A000A
:10CD40000040EB00A4810200000000000000EB00A6
:10CD5000005D8800F05C80000000E00003003A0005
:10CD60003481020000000000004F78001000200015
:10CD7000005D88001E80FB000080FA0000000600B5
:10CD80000400FA00000F7800005D80000000E00061
:10CD90001200320000C2B300327102000000000035
:10CDA0003100200010442000EE9902000000000035
:10CDB00000C2B3003271020000000000F05C80008D
:10CDC0000000E00003003A000040EB00A4810200F4
:10CDD000000000000000EB00005D8800F05C8000B7
:10CDE0000000E00007003A001E007800E08002002A
:10CDF0000000000082810200000000000080FB00B3
:10CE0000000F780000C2B300327102000000000081
:10CE10001E00E00007003A0031002000104420000E
:10CE2000EE9902000000000000302000100798007A
:10CE3000060037004100200040442000EE99020027
:10CE40000000000000102000100798001E00900055
:10CE50000080FA00000006000000FA00005D80007B
:10CE60000000E0000F00320041002000404420009C
:10CE7000EE9902000000000020A12800026D0200CF
:10CE800000000000F05C80000000E00003003A00B9
:10CE900010C0B300A4810200000000000000EB00FD
:10CEA000005D8800F05C80000000E0000F003A00A8
:10CEB0000E800200000000000000E0000B003200C5
:10CEC00091002000A0232000EE9902000000000045
:10CED0005101200030242000EE99020000000000E3
:10CEE00020A12800026D020000000000D1002000F7
:10CEF00080442000789A0200000000000080FA00C0
:10CF0000000006000000FA00005D80000000E00064
:10CF10000F0032004100200040442000EE99020042
:10CF20000000000020A12800026D020000000000A7
:10CF3000F05C80000000E00003003A0010C0B30085
:10CF4000A4810200000000000000EB00005D8800EA
:10CF5000F05C80000000E00002003A004E80020019
:10CF600000000000C100200050452000789A020017
:10CF7000000000000080FA00000006000000FA0037
:10CF80000101200020522000EE9902000000000064
:10CF90000040EB006E6F02000000000000C2B30012
:10CFA000327102000000000060B7200010407800DD
:10CFB0006E6F02000000000000C2B3003271020078
:10CFC0000000000030A12800026D020000000000F7
:10CFD0000080FA00000006000400FA000000EB00E8
:10CFE000100798000000EB00F05C88002C1A02008B
:10CFF000000000005616020000000000000F78003C
:10D000001E00E00009003400400020009E0F1000C8
:10D0100006003C001E0078000040E90080407800D7
:10D0200060B7200001487800020037000000EB00E4
:10D03000000F78001E00E0002D003A000000EB0019
:10D04000606988000000EB00F05C8800F05C800004
:10D050000000E0000F003A00B1032000604820000B
:10D06000789A0200000000008001EB0042002000DE
:10D070001100200010002000A21C0200000000008F
:10D080000040E9008040780060B720000148780047
:10D0900022003700C140800030002300808F500004
:10D0A00004003E0051032000104C2000EE990200C5
:10D0B00000000000C1022000604F2000EE99020035
:10D0C000000000008001EB00320020001100200071
:10D0D00010002000A21C0200000000000040E90037
:10D0E0008040780060B72000014878000B003700CE
:10D0F000C140800030002300808F500004003E00BB
:10D1000051032000104C2000EE99020000000000A6
:10D110009AFF07000000EB00005D880080B8200047
:10D12000104078000030A00081B8200080487800CE
:10D13000F05C80000000E00009003A00C922A8006D
:10D14000C902A800CB02A900CB22A90060B7200029
:10D150009040780020C0B300807F020000000000F3
:10D160000080FA00000006000000FA000000EB005A
:10D17000005D8800F05C8000E10F500001003A0083
:10D1800007E2A9000080FA00000006000600FA008D
:10D19000100798001E009000200798002E009000B5
:10D1A000E10F50000C0032002E009000E10F500003
:10D1B000040039002E009000E20F5000650032009C
:10D1C000730037005103200020532000EE99020025
:10D1D00000000000720037008040EB0000302000AB
:10D1E0002E82020000000000E102200070562000A4
:10D1F000789A020000000000CBC2BF0061406000CE
:10D200000004E00004003200CBC2BF0062406000B6
:10D210000004E0000C003A0091002000A023200050
:10D22000EE9902000000000051012000302420008F
:10D23000EE9902000000000020A12800026D02000B
:10D2400000000000560037000000EB00000F7800DF
:10D2500039003700F05C80000000E00009003A006F
:10D260000E800200000000001E007800E080020036
:10D270000000000082810200000000000080FB002E
:10D28000100798001E0090000000E00024003A0003
:10D290001E007800C69602000000000080C2B300A5
:10D2A00032710200000000001E0078000080D100F2
:10D2B000C6960200000000001E0078000000A200D8
:10D2C000610060000004E0000400320050A128006A
:10D2D000D66C0200000000000B003700F05C8000FC
:10D2E0000000E00005003A00348102000000000068
:10D2F00010C0B300A48102000000000080A128003B
:10D30000D66C02000000000030A12800D66C02009C
:10D310000000000000C2B3003271020000000000F3
:10D32000F05C80000000E00002003A004E80020045
:10D33000000000001E0FE800F00F20009E0F1000FC
:10D34000C4FF340020A12800026D0200000000008C
:10D3500013003700F05C8000E10F500001003A003C
:10D3600007E2A9007100200050592000789A0200BD
:10D3700000000000F1002000C01E2100789A020089
:10D380000000000010C0B3000E00070004003700CA
:10D3900041022000C0202000789A02000000000016
:10D3A0000080FA00000006000000FA00B100200032
:10D3B000C0092100789A0200000000000080FA00F5
:10D3C000000006000A00FA00004F98000040EB0041
:10D3D000204798000040EB00104798000040EB0009
:10D3E000004F7800DA71020000000000C922A80096
:10D3F000C902A800CB02A900CB22A90062A0A80004
:10D4000062C0A8008660A900CBC2BF000080FB00FC
:10D410000000D10061406000604798006E409000BD
:10D4200050479800CBC2BF00614060006047980041
:10D430006E409000304798000000370086C0BF0063
:10D44000684060000004E00012003A0023C2BF0000
:10D45000624060000004E0000E003A001872020012
:10D460000000000022C2BF00614060000004E00034
:10D47000F2FF320030118000004F780062A0A90056
:10D4800062C0A9000E4890000004E00061003A006C
:10D49000630037008660A900CBC2BF000080FB009C
:10D4A0000000D1006140600060479800CBC2BF001F
:10D4B00061406000404798002E4090000004E0006A
:10D4C0002E0032003E4090000004E0002B003A00A5
:10D4D0004E4090000004E000280032001E40900002
:10D4E000E74F50000B003E001E4078000040400017
:10D4F000004F78006E4090000004E0000100320010
:10D500001E04A0001E4090000040E8001047980054
:10D510003B0037000E4890000004E0000400320099
:10D520001E80FB00FA6F02000000000006003700BA
:10D53000C0C5B300E8710200000000001E40780082
:10D54000E8710200000000006E4090000004E0005E
:10D5500004003200D0C2B300E871020000000000F5
:10D5600003003700B0C2B300E87102000000000001
:10D570000040EB0010479800210037003E4090002B
:10D580000004E0001E0032004E4090000004E00065
:10D590001B0032005E4090000004E0000B003200EF
:10D5A0006E4090000004E00008003A0010C0B30094
:10D5B000204798000040EB0010479800B0C5B3002A
:10D5C000E8710200000000000D0037005E4090008E
:10D5D0000004E0000A003A006E4090000004E00001
:10D5E000070032000040EB00204798000040EB00AD
:10D5F00010479800D0C5B300E87102000000000099
:10D600006E409000504798004E4090003047980080
:10D610008AFF370020A12800026D020000000000F0
:10D620000080FA00000006000000FA00B0A1280007
:10D63000D66C0200000000000080FA000000060026
:10D640000400FA00C922A800C902A800CB02A90060
:10D65000CB22A900C8C2A90080B8200010407800E1
:10D660000030A00081B820008048780080B82000F9
:10D67000104078000020A10081B820008048780088
:10D6800080C0EB0020C0B300807F020000000000DB
:10D69000E5FF07000000370022C2BF0061406000C4
:10D6A0000004E000FCFF3200301180008040780070
:10D6B000C0B9200001487800C0B9200010407800AF
:10D6C0000080FB004400DE0080407800B0B92000FC
:10D6D00001487800B0B92000104078000080FB00BD
:10D6E000100798001E009000E10F50005E0032000D
:10D6F0001E009000E10F500004003C001E0090004E
:10D700000000E00008003200970037001E00900083
:10D71000E40F50008C0032001E009000E60F500015
:10D720007A00320090003700C0B920001040780025
:10D730000080FB00000F78001E007800E30F50000F
:10D74000260032001E007800E30F50000A003C0063
:10D750001E007800E10F5000180032001E00780013
:10D76000E10F500017003C001E0078000000E000B0
:10D7700081003200380037001E007800E60F5000AC
:10D78000210032001E007800E60F500004003C002B
:10D790001E007800E40F5000160032002E00370003
:10D7A0001E007800E70F50001E0032001E007800B7
:10D7B000EF0F500022003200270037009AFF0700C9
:10D7C000B5FF37000E8002000000000010C0B3005B
:10D7D0003271020000000000AFFF37004E800200EF
:10D7E0000000000010C0B300327102000000000011
:10D7F000A9FF3700348102000000000032710200EE
:10D8000000000000A4FF37000040EB00A4810200EC
:10D810000000000010C0B3003271020000000000E0
:10D820009DFF370010C0B300A4810200000000007B
:10D8300010C0B300327102000000000096FF3700F4
:10D840000040EB00DFFE070010C0B30032710200A1
:10D850000000000090FF37000040EB003271020032
:10D86000000000008CFF3700C0B920009040780015
:10D87000F0C0B30080C06000C0B92000014878004B
:10D88000C0B92000104078008040E800C0B92000F6
:10D890000148780010C0B30032710200000000009F
:10D8A0008040EB00A0B9200001487800100037004C
:10D8B00022C2BF00614060000004E000FCFF3200B3
:10D8C00030118000E0800200000000008281020030
:10D8D000000000003271020000000000A0B920002A
:10D8E000104078008040E800A0B92000014878008E
:10D8F000A0B9200090407800C0B920001040780006
:10D9000080CF5000EAFF390063FF3700C0B9200024
:10D910009040780030C0B30080C06000C0B92000E3
:10D9200001487800C0B920009040780020C0B300C2
:10D93000807F02000000000010C0B30032710200BE
:10D940000000000054FF3700C0B9200010407800EC
:10D95000D09C02000000000010C0B3003271020031
:10D96000000000004CFF37000040EB003271020065
:10D970000000000048FF37000080FA0000000600A9
:10D980000200FA00000F78001E00E00003003200E1
:10D9900010C3B300330207000200370000C3B30016
:10D9A000300207000080FA00000006000600FA00BE
:10D9B00010079800020037001E4078002902070077
:10D9C0001E009000104F78001E40780040479800DD
:10D9D0004E4090000004E0000200320010C0B3008E
:10D9E000404798004E4090009E0090008100E80063
:10D9F000110798000004E000EFFF3A000080FA00F1
:10DA0000000006000600FA00100798000200370028
:10DA10001E407800130207001E009000104F78008F
:10DA20001E407800404798004E4090000004E000FF
:10DA30000200320010C0B300404798004E409000F2
:10DA40009E0090008100E800110798000004E000AB
:10DA5000EFFF3A00D0C0B30002020700A0C0B3003D
:10DA6000000207000080FA00000006000400FA002F
:10DA70002047980000C8B300004F7800C09D2800E0
:10DA8000CAFF07000040EB00104798000F00370066
:10DA90002E4090001E4060000004E00003003200B1
:10DAA00010C3B300EF0107000200370000C3B3004A
:10DAB000EC0107001E80FB000000D100004F780041
:10DAC0001E4090000040E800104798001E40900063
:10DAD000E74F5000EEFF36000080FA00000006001D
:10DAE0000E00FA0050079800610798000040EB0014
:10DAF000004F780000102E00515F20003007980082
:10DB0000410798000040EB001047980032003700B2
:10DB10003E019000CE0190005E009000EE0090006B
:10DB2000300602000000000010079800210798004E
:10DB30001E04E00005003A001E009000AE009000B8
:10DB4000E00F5000E08F5800180032001E009000D7
:10DB50000043B000C30107009E0090003E0090000B
:10DB6000000AB8009E0090004E0090000088B900A6
:10DB70000501780000014100BE0090002E009000D9
:10DB80000088B90000014100820278005E00900028
:10DB9000EE00900004005000858058005007980067
:10DBA0006107980010C0B300004F78003E0090005D
:10DBB000CE009000A20020000300200030060200EA
:10DBC0000000000030079800410798001E409000B8
:10DBD0000040E800104798001E409000E74F5000BA
:10DBE000CBFF36005E0090000043B0009D010700AF
:10DBF0000080FA00000006000C00FA0040079800C0
:10DC0000510798000000EB00100798000000EB009F
:10DC1000000F78006000B8002007980031079800D6
:10DC20004E019000DE019000F0232400F10020005E
:10DC3000800F5100818F5900210036004E00900066
:10DC4000DE00900002242400F300200030060200D1
:10DC50000000000020079800310798002E00900077
:10DC60006F000700C0C2B3007E0107004E009000A5
:10DC7000DE00900002242400F30020005006020081
:10DC80000000000040079800510798004E019000E6
:10DC9000DE019000703E200001002000800F510046
:10DCA000818F590002003E00F09D28003FFF0700D1
:10DCB000100020001007980010002000000F7800CE
:10DCC0004E019000DE019000703E20000100200017
:10DCD000800F5100818F5900320036004E009000B5
:10DCE000DE009000823E200003002000300602008B
:10DCF0000000000020079800310798002E019000D6
:10DD0000BE0190004006200001002000800F51005D
:10DD1000818F5900030036002E009000400007005C
:10DD2000140037001E0090000000E0000F003200D9
:10DD30002E019000BE019000A000200001002000F4
:10DD4000800F5100818F59000300360000C3B300DB
:10DD50004401070002003700409E280013FF07001F
:10DD60002E0090002E000700020037002E009000C9
:10DD70002B000700C0C2B3003A0107004E0090001C
:10DD8000DE009000823E20000300200050060200CA
:10DD90000000000040079800510798001000200084
:10DDA000000F78004E019000DE0190004006200038
:10DDB00001002000800F5100818F590003003600C0
:10DDC0004E00900016000700130037001E00E00010
:10DDD0000F0032004E019000DE019000A0002000F4
:10DDE00001002000800F5100818F59000300360090
:10DDF00000C3B3001B01070002003700409E28004B
:10DE0000EAFE07004E009000050007000200370000
:10DE10004E009000020007000080FA00000006009B
:10DE20000800FA00300798000040EB00004F78002F
:10DE300000712200200798000040EB001047980076
:10DE40001E0037003E0090002E01900011000900D6
:10DE50000280D800100798001E04E00003003A007A
:10DE60001E0090000000E0000C0032001E00900038
:10DE70000043B000FB0007009E0090002E009000C1
:10DE80000088B900800078003E009000010050003A
:10DE90003007980010C0B300004F78002E009000AB
:10DEA000A2002000110009000280D800200798007D
:10DEB0001E4090000040E800104798001E4090006F
:10DEC000E34F5000DFFF36003E0090000043B000FB
:10DED000E40007000080FA00000006000600FA00D7
:10DEE000404798000040EB00004F780040C6B30068
:10DEF000304798000040EB00204798002000370092
:10DF00004E4090008080FB003E4090000081FB006E
:10DF1000110009008280D800104798001E04E0001C
:10DF200003003A001E4090000004E0000B003200A5
:10DF30001E4090000043B000CA0007004E41900010
:10DF40009E4090003E4090000088B9000040510083
:10DF50004047980010C0B300004F78003E4090004A
:10DF60000080FB00A2002000110009000280D80000
:10DF7000304798002E4090000040E800204798006D
:10DF80002E409000E14F5000DDFF36004E409000E3
:10DF90000043B000B30007000080FA000000060054
:10DFA0000400FA0010079800709F28007FFE070009
:10DFB0001E0090004400DE006F0F60009E0078009D
:10DFC000709E28000080400010407800A5000700E7
:10DFD0001E0090006F0F60009E007800709E280069
:10DFE00000804000104078009E0007000080FA008A
:10DFF000000006000400FA001007980000C3B300F8
:10E00000F300070080C7B300F10007001E00900076
:10E010004400DE006F0F60009E007800709E2800B4
:10E020000080400010407800E90007001E009000CA
:10E030006F0F60009E007800709E280000804000F6
:10E0400010407800E20007000080FA00000006009F
:10E050000400FA0010079800709F280053FE070084
:10E060001E0090004C00DE006F0F60009E007800E4
:10E07000709E280000804000104078007900070062
:10E080001E0090004800DE006F0F60009E007800C8
:10E09000709E28000080400010407800710007004A
:10E0A0001E0090004400DE006F0F60009E007800AC
:10E0B000709E280000804000104078006900070032
:10E0C0001E0090006F0F60009E007800709E280078
:10E0D0000080400010407800620007000080FA00D5
:10E0E000000006000800FA00300798003E0090008B
:10E0F000CF80DE00F403020000000000926C2200DA
:10E10000B331240052040200000000001007980000
:10E11000210798001E009000AE00900056060200F5
:10E1200000000000004F78001E4078006BFF0700E1
:10E13000E0C2B3004B0007001E009000AE0090004C
:10E140005606020000000000CF80DE00F40302004B
:10E15000000000000001BE001E009000AE00900014
:10E16000D604020000000000100798002107980064
:10E1700002002000031224001E009000AE00900058
:10E180009205020000000000100798002107980087
:10E190001E009000AE009000560602000000000035
:10E1A000004F78001E4078004CFF07001E009000D2
:10E1B000AE0090005606020000000000CF80DE0096
:10E1C000F4030200000000000001BE001E009000E9
:10E1D000AE009000D6040200000000001007980076
:10E1E0002107980002002000031224001E00900066
:10E1F000AE00900092050200000000001007980099
:10E20000210798001E009000AE0090005606020004
:10E2100000000000004F78001E4078002FFF07002C
:10E220000080FA00000006000000FA0022C2BF00D1
:10E23000614060000080FB000080FA0000000600E2
:10E240000000FA0022C2BF00614060000004E0004C
:10E25000FCFF3200301180000080FB000080FA00DB
:10E26000000006000200FA00004F7800D040800055
:10E2700001102000010060000000E00006003A00EC
:10E2800023C2BF00624060000004E000FCFF3A00CF
:10E290001E00FB00201188000080FA00000006002C
:10E2A0000200FA00004F78001E80FB004011880039
:10E2B0000080FA00000006000000FA0095C0BF00D0
:10E2C000704060000004E00010003A0051408000FF
:10E2D00040408000808F50000C00320023C2BF00FD
:10E2E000624060000004E000FCFF3A008580A90065
:10E2F0009580A800314080004040800000804000B0
:10E30000104078000080FB00201188000080FA0097
:10E3100000000600809FBE000000FA00014080005F
:10E3200020408000808040003011800080487800CC
:10E33000204080000000E80020408800214080004C
:10E3400010408000808F500001003A009560A900C5
:10E350008560A9000080FA004F00BE000040060062
:10E36000809FBE000000FA00404080000000E800EE
:10E37000404088004140800050408000808F500025
:10E3800002003A009580A900060037003140800065
:10E390004040800000804000104078000080FB007A
:10E3A000201188008580A9000080FA004F00BE007F
:10E3B000004006000000FA000000EB00906E8800AC
:10E3C00010002000806E88000080FA000000060027
:10E3D0000200FA00004F7800816E8000906E80008D
:10E3E000808F500002003A00CA82A9000E00370058
:10E3F00071408000806E8000808040001E40780068
:10E4000080487800806E80000000E800806E880000
:10E41000816E800000002100808F500002003A00D1
:10E420000000EB00806E88000080FA00000006000B
:10E430000200FA00906E8000000FE800000021004A
:10E440009E0F100002003A000000EB00000F780061
:10E45000806E80009E0F10000C00320023C2BF00AF
:10E46000624060000004E00008003A001E007800EE
:10E47000906E880071408000906E800000804000A7
:10E48000104078000080FB00201188000080FA0016
:10E49000000006000400FA00000F78001107980041
:10E4A0001E007800900188001E0090001080BA00C5
:10E4B000C800DD001E0090001000BA00008070004F
:10E4C0000080FA00000006000600FA000000EB00E1
:10E4D000800888000000EB00F00888000000EB00D6
:10E4E000E00C8800206180000000E00008003A0095
:10E4F000A16C20009140780000CEB30000C0600005
:10E50000CAE6B7000000EB00B06088003D003700AD
:10E5100020618000E30F500005003C00E003200074
:10E52000000F780010A1A8001081A8001500370086
:10E5300020618000FE0F500005003C00A00F20006D
:10E54000000F780010A1A8001081A9000D0037006D
:10E5500021618000400F2000808F500005003C00AA
:10E56000007D2000000F780010A1A9001081A800F4
:10E570000400370000E82300000F780010A1A90074
:10E580001081A90020618000000178001E00780041
:10E59000110009000280D8000000E900200798005F
:10E5A0002E009000600888003061800080007800B4
:10E5B0002E0090000088B9004206200011000900DA
:10E5C0000280D80010079800A16C200091407800CC
:10E5D00000CEB30000C060006041B300CAE6B700DF
:10E5E0001E009000D00C88001E009000C00C880017
:10E5F00060002000E00C880011E1A800200020004D
:10E60000B06088000080FA00000006001200FA00E6
:10E610000000EB00800888000000EB00F008880094
:10E620000000EB00E00C8800B0608000E20F5000BA
:10E6300014003A00A16C20009140780000CEB30095
:10E6400000C06000CAE6B700C1002000C02E200054
:10E65000789A0200000000000000EB00B060880023
:10E66000506980008000E800F00F2000808060008A
:10E6700080C2200000804000104078000004E000CC
:10E68000AE0032000000EB002007980050698000C7
:10E690000000E8005069880051698000F00F2000F8
:10E6A00000806000506988002C1A02000000000001
:10E6B0005616020000000000400798002C1A0200C5
:10E6C000000000005616020000000000CF80DE00AF
:10E6D000F403020000000000008FBE004E00900016
:10E6E0000000E00007003200CE009000F0F92000AA
:10E6F000808F500003003E002E0090000000E800D4
:10E70000200798006011B8001E00BE004A040200F5
:10E71000000000000000E00001003C000B0037009A
:10E7200002002000832C24001E00BE004E040200C4
:10E73000000000000000E000010035000300370089
:10E740002E0090000000E800200798002E009000A6
:10E75000E20F5000110032000000EB0060698800F9
:10E7600011012000802F2000789A02000000000094
:10E770001101200090302000EE99020000000000FE
:10E780008001EB0002FA200011002000200320008D
:10E79000A21C020000000000400798004E009000FC
:10E7A000E30F500005003E00E00320003007980012
:10E7B00010A1A8001081A800150037004E0090009D
:10E7C000FE0F500005003E00A00F2000300798000B
:10E7D00010A1A8001081A9000D003700CE00900004
:10E7E000400F2000808F500005003E00007D20007B
:10E7F0003007980010A1A9001081A800040037007C
:10E8000000E823003007980010A1A9001081A9009A
:10E810003E0090004E019000110009000280D800D7
:10E820000000E900600798002E009000E20F500001
:10E830000E0032000101200070322000EE9902002B
:10E84000000000008001EB00320620008000EB0099
:10E8500020032000A21C020000000000CF80DE0088
:10E86000F403020000000000008FBE000200200040
:10E87000832C24001E00BE00520402000000000091
:10E88000008FBE006E009000CF80DE00F403020017
:10E890000000000070079800010F98006E009000C3
:10E8A0000000E00008003D00020020000378240082
:10E8B0007E0090008E089000D80402000000000046
:10E8C00070079800010F98001E01BE007E009000A6
:10E8D0008E0890009205020000000000FA05020078
:10E8E0000000000050079800A16C200091407800C3
:10E8F00000CEB30000C060006041B300CAE6B700BC
:10E900005E009000D00C88005E009000C00C880073
:10E9100060002000E00C88006E0090006008880015
:10E9200011E1A800A100200070332000789A0200B5
:10E930000000000020002000B06088000080FA0085
:10E94000000006000000FA00B0608000E20F5000F6
:10E9500005003A00F101200010342000789A0200EE
:10E96000000000003E003700F100200000362000CB
:10E97000EE990200000000000000EB00F0088800A3
:10E980000000EB0080088800C942A80061682000F0
:10E990009140780000CEB30000C06000A040B300FA
:10E9A00086E6B700A0032000800888002E0007003C
:10E9B000C0608800D1608800C2608000D3608000A1
:10E9C000F00F200001002000800F5100818F5900BE
:10E9D00009003600C0608000D1608000C808DD00FA
:10E9E0000080FD00804078000040EB00C06088009F
:10E9F000D160880009003700B1002000B019210063
:10EA0000EE99020000000000A000200080088800AD
:10EA100015000700C0608800D1608800C0608000D9
:10EA2000D1608000FC6D02000000000040A32800BF
:10EA3000D66C02000000000080A32800026D0200D6
:10EA40000000000086C6BF00F041B30086E6B700B4
:10EA50000000EB00F00888000000EB008008880050
:10EA60000080FA00000006000000FA000080EB00C1
:10EA7000700888000080EB00600888000000EB0050
:10EA8000400888000000EB00300888000000EB0020
:10EA9000B00888000000EB00A0088800800020007B
:10EAA000F0088800400F2000E008880000402200A5
:10EAB000D00888008780A9001FE1A80011E1A80004
:10EAC00087C0BF00704060000004E000FCFF32001F
:10EAD00011E1A9001FE1A900300880001061880041
:10EAE0004008800000618800006180000100200073
:10EAF000E0608800F1608800E0608000F1608000E4
:10EB0000C000DD0000002000E0608800F1608800A7
:10EB1000106180006101B800E0608000F160800059
:10EB20000200400083804800E0608800F1608800B7
:10EB3000E0608000F16080000080FA0000000600C4
:10EB40000000FA0080B820001040780061406000AA
:10EB50000004E00002003A00C942A80001003700AA
:10EB6000C8C2A800E1002000F0362000EE990200A3
:10EB7000000000000080FA00000006000000FA001B
:10EB800080B8200010407800614060000004E00080
:10EB900003003A00C942A900CB42A8000200370096
:10EBA000C8C2A900CAC2A80081002000D037200036
:10EBB000789A0200000000000080FA0000000600C1
:10EBC0000000FA0080B8200010407800614060002A
:10EBD0000004E00003003A00C942A900CB42A900AA
:10EBE00002003700C8C2A900CAC2A90071002000F3
:10EBF00050382000789A0200000000000080FA00DF
:10EC0000000006000200FA0080B8200010407800E2
:10EC1000614060000004E00009003A00C942A80019
:10EC20000000000000000000CBC2BF000080FB001D
:10EC30004200DE0061406000004F780008003700AD
:10EC4000C8C2A8000000000000000000CAC2BF0047
:10EC50000080FB004600DE0061406000004F78004D
:10EC60001E80FB000080FA00000006000C00FA0085
:10EC70000000EB00800888000000EB00F00888002E
:10EC80000000EB00E00C8800B0608000E20F500054
:10EC900014003A00A16C20009140780000CEB3002F
:10ECA00000C06000CAE6B700C1002000C02E2000EE
:10ECB000789A0200000000000000EB00B0608800BD
:10ECC000506980008000E800F00F20008080600024
:10ECD00080C2200000804000104078000004E00066
:10ECE00066003200506980000000E800506988002A
:10ECF00051698000F00F200000806000506988009A
:10ED00002C1A02000000000056160200000000004D
:10ED1000CF80DE00F403020000000000008FBE0080
:10ED2000606980000000E00008003A000200200056
:10ED3000433324001E00BE004A040200000000000D
:10ED40000000E00001003C00100037000000EB0074
:10ED5000606988003101200040242100789A020077
:10ED6000000000008001EB00420B20008000EB005F
:10ED7000A0052000A21C020000000000CF80DE00E1
:10ED8000F403020000000000008FBE0010A1A800E4
:10ED90001081A800204E20003007980002002C00AF
:10EDA000A35524001E00BE00520402000000000013
:10EDB000008FBE003E009000CF80DE00F403020012
:10EDC0000000000040079800510798003E009000A6
:10EDD0000000E00008003D0002002000037824004D
:10EDE0004E009000DE009000D804020000000000F9
:10EDF00040079800510798001E01BE004E00900089
:10EE0000DE009000920502000000000002002000D9
:10EE100083272400D804020000000000FA05020045
:10EE20000000000020079800A16C200091407800AD
:10EE300000CEB30000C060006041B300CAE6B70076
:10EE40002E009000D00C88002E009000C00C88008E
:10EE500060002000E00C88003E0090006008880000
:10EE600011E1A800C100200070252100789A02005D
:10EE70000000000020002000B06088000080FA0040
:10EE8000000006000000FA0000A42800D66C020072
:10EE9000000000000080FA00000006000200FA00F6
:10EEA000CA82A800E0000700F6FF07000000370054
:10EEB000D40007008040780060DE20000148780020
:10EEC00060DE2000104078000004E000C70035003C
:10EED00060DE2000104078000004E00002003A00EC
:10EEE000E8FF0700F2FF370060DE200010407800E6
:10EEF000E14F500006003A00CB0007007C490200B9
:10EF000000000000C8000700DEFF0700E8FF370030
:10EF100060DE200010407800E24F500006003A000A
:10EF2000C1000700206B020000000000BE000700C7
:10EF3000D4FF0700DEFF370060DE200010407800BD
:10EF4000E34F500006003A00B70007002E520200BF
:10EF500000000000B4000700CAFF0700D4FF37001C
:10EF600060DE200010407800E44F500006003A00B8
:10EF7000AD000700245D020000000000AA000700A9
:10EF8000C0FF0700CAFF370060DE20001040780095
:10EF9000E54F500006003A00A3000700085F02009A
:10EFA00000000000A0000700B6FF0700C0FF370008
:10EFB00060DE200010407800E64F500006003A0066
:10EFC00099000700DE8C0200000000009600070098
:10EFD000ACFF0700B6FF370060DE2000104078006D
:10EFE000E74F500004003A008F0007008E00070032
:10EFF000A4FF0700AEFF370060DE2000104078005D
:10F00000EF4F50000A003A0010C0B3003271020006
:10F0100000000000CA82A90023C2BF006140600056
:10F020000004E000FCFF32000000FE00A0FF3700FB
:10F0300060DE200010407800F24F500035003A00AA
:10F040000000EB00800888000000EB00F00888005A
:10F050000000EB00E00C8800A16C200091407800DB
:10F0600000CEB30000C060006041B300CAE6B70044
:10F07000640007000080FB00000F78001E0078008D
:10F080000000D100610060000004E00001003200D7
:10F0900010A1A8009E007800618060000004E000DC
:10F0A000010032001081A800560007000080FB001C
:10F0B0004800DD00000F7800520007000080FB00D0
:10F0C0001E0F70001E007800D00C88009E00780093
:10F0D000C10C880060002000E00C88004900070097
:10F0E0000080FB004800DD00000F780045000700AD
:10F0F0000080FB001E0F70001E0078006008880072
:10F1000011E1A80010C0B30032710200000000003D
:10F1100067FF370060DE200010407800F34F50009A
:10F120000D003A000000EB00800888000000EB00B2
:10F13000E00C8800A16C20009140780000CEB30064
:10F1400000C06000CAE6B70010C0B3003271020010
:10F150000000000056FF370060DE200010407800FD
:10F16000F44F50000E003A0021E3A800C0C0B300E5
:10F170000E96020000000000000F780021E3A900B5
:10F180001E0078004800DE0032710200000000001E
:10F190001E007800327102000000000044FF3700BA
:10F1A00060DE2000104078000080FB004500DE009B
:10F1B0000080FB000000D100610060000004E0005E
:10F1C0000600320060DE2000104078001F000700BB
:10F1D000327102000000000035FF37000040EB00F4
:10F1E000327102000000000031FF370060DE2000B5
:10F1F00010407800A50007003271020000000000F6
:10F200002BFF37000000FA0022C2BF0061406000FF
:10F210000004E000FCFF3200301180000080FB00A1
:10F220000080FA00000006000000FA0000C0EB00B9
:10F23000060007000040EB0094000700C962A90027
:10F24000CB62A9000080FA00000006000400FA006A
:10F25000204798000040EB00004F78002E409000BF
:10F260000080FB004400DE00610060000004E0005C
:10F270000200320010C0B300004F78009E407800BA
:10F2800061C06000614060004201DD00912C2000FF
:10F2900091407800B0CFB30000C060000240700021
:10F2A000C9E2B7000040EB00004F78002E4090000C
:10F2B0000080FB004300DE00610060000004E0000D
:10F2C0000200320010C0B300004F78009E4078006A
:10F2D00061C060006140600000414000912C20004E
:10F2E00091407800D0CFB30000C0600002407000B1
:10F2F000C9E2B7000040EB00004F78002E409000BC
:10F300000080FB004200DE00610060000004E000BD
:10F310000200320010C0B300004F78009E40780019
:10F3200061C0600061416000912C20009140780034
:10F33000E0CFB30000C0600002407000C9E2B70037
:10F340000040EB00004F78002E4090000080FB0052
:10F350000000D100610060000004E0000200320003
:10F3600010C0B300004F78009E40780061C060007C
:10F37000C700DD00C8C2BF000074A10001407000DA
:10F38000C8E2B7000040EB00004F78002E4090002C
:10F390000080FB00610060000004E0000200320019
:10F3A00010C0B300004F78009E40780061C060003C
:10F3B000614060004601DD00812C20009140780012
:10F3C000F0CBB30000C0600002407000C8E2B7009C
:10F3D000500020007897020000000000AE4090002E
:10F3E00000CEB30000C0600020479800CBC2BF0031
:10F3F000644060000004E000030032002E409000F2
:10F400000044A00020479800CBC2BF0062406000CB
:10F410000004E000030032002E4090000034A00001
:10F4200020479800CBC2BF00614060000004E000AC
:10F43000030032002E4090000024A00020479800D6
:10F44000CAC2BF0001C8B300014060000004E00070
:10F45000030032002E4090000014A00020479800C6
:10F46000CAC2BF000044B2000004E0000300320042
:10F470002E4090000004A000204798002E409000ED
:10F480000080FB000080FA00000006000400FA0083
:10F49000204798002E4090000080FB004600DE00D0
:10F4A000610060000004E00005003200C082A90095
:10F4B000C282A800C8A2A900CAA2A80004003700FE
:10F4C000C082A900C282A900C8A2A900CAA2A9003C
:10F4D0000040EB00004F78002E4090000080FB00C1
:10F4E0004400DE00610060000004E0000200320021
:10F4F00010C0B300004F78009E40780061C06000EB
:10F50000614060004201DD00B12C20009140780094
:10F51000B0CFB30000C0600002407000CBE2B70083
:10F520000040EB00004F78002E4090000080FB0070
:10F530004300DE00610060000004E00002003200D1
:10F5400010C0B300004F78009E40780061C060009A
:10F550006140600000414000B12C200091407800E3
:10F56000D0CFB30000C0600002407000CBE2B70013
:10F570000040EB00004F78002E4090000080FB0020
:10F580004200DE00610060000004E0000200320082
:10F5900010C0B300004F78009E40780061C060004A
:10F5A00061416000B12C200091407800E0CFB300B1
:10F5B00000C0600002407000CBE2B7000040EB00EA
:10F5C000004F78002E4090000080FB000000D1002A
:10F5D000610060000004E0000200320010C0B300CF
:10F5E000004F78009E40780061C06000C700DD00D9
:10F5F000CAC2BF000074A10001407000CAE2B70097
:10F600000040EB00004F78002E4090000080FB008F
:10F61000610060000004E0000200320010C0B3008E
:10F62000004F78009E40780061C06000614060003B
:10F630004601DD00A12C200091407800F0CBB30002
:10F6400000C0600002407000CAE2B7005000200015
:10F650007897020000000000AE40900000CEB3009A
:10F6600000C0600020479800CBC2BF00644060002B
:10F670000004E000030032002E4090000044A0008F
:10F6800020479800CBC2BF00624060000004E00049
:10F69000030032002E4090000034A0002047980064
:10F6A000CBC2BF00614060000004E00003003200F4
:10F6B0002E4090000024A00020479800CAC2BF003E
:10F6C00001C8B300014060000004E0000300320004
:10F6D0002E4090000014A00020479800CAC2BF002E
:10F6E0000044B2000004E000030032002E4090000D
:10F6F0000004A000204798002E4090000080FB00EE
:10F700000080FA00000006000000FA0080B8200027
:10F71000104078000030A00081B8200080487800B8
:10F72000960007000080FA00000006000000FA00C2
:10F730003C010700530007003027210010407800EB
:10F740000080FB000080FA00000006000400FA00C0
:10F75000100798001E00900071010700004F78000C
:10F760001E04E00005003A00310020001044200093
:10F77000EE990200000000000C00370010C0B3003A
:10F780009E4F100005003A00410020004044200038
:10F79000EE99020000000000040037008100200004
:10F7A00000122100EE99020000000000001020006D
:10F7B0000080FA00000006000400FA00000F780044
:10F7C0001E007800100798001E0090000000E00066
:10F7D000040032001E009000E10F500006003200CD
:10F7E000220037006102200080122100789A020076
:10F7F0000000000021003700D1002000E0142100AB
:10F80000789A020000000000F1002000C01E2100D4
:10F81000789A020000000000020107000004E000E6
:10F8200008003A0030272100104078000080FB00DB
:10F83000C69602000000000000C2B3003271020050
:10F840000000000022C2BF00614060000004E00030
:10F85000F1FF320030118000000F780020A6280050
:10F86000026D020000000000040037004102200089
:10F87000C0202000789A0200000000000080FA00FA
:10F88000000006000400FA00004F78001E80FB0014
:10F89000100798009E009000E28F50001A0032007E
:10F8A0001E009000E20F500007003C009E009000F8
:10F8B0000100E0002F0032001E009000E10F500018
:10F8C0000C003200270037009E009000E48F5000AB
:10F8D000170032001E009000E40F50000F003500AA
:10F8E000F00F20009E009000808F50001800320022
:10F8F0001C00370001012000B0152100789A020099
:10F90000000000001B003700E1002000B0162100BD
:10F91000789A02000000000016003700F100200075
:10F9200090172100789A02000000000011003700B3
:10F9300000C2B3003271020000000000810020000C
:10F9400000122100EE9902000000000009003700BB
:10F950005100200080182100789A02000000000069
:10F9600004003700E1002000D0182100789A02003E
:10F97000000000000080FA00000006000000FA000D
:10F98000C922A800C902A900CB02A900CB22A90064
:10F990000080FA00000006000400FA000040EB00BE
:10F9A000410107000004E0000300320020002000B5
:10F9B000100798000E003700CBC2BF000080FB008C
:10F9C0000000D10061406000004F780010C0B3001B
:10F9D000350107000004E000030032002000200091
:10F9E00010079800020037001E80FB0010079800E7
:10F9F0001E0090000080FA00000006000600FA00D9
:10FA00000040EB00204798000040EB0010479800B2
:10FA1000CBC2BF000080FB000000D100E1406000CD
:10FA2000202721001040780061C16000E1CFB300C1
:10FA300001406000024070002127210080487800CA
:10FA40002027210010407800614060000004E000A1
:10FA50000300320010002000200798006E003700DD
:10FA600010C0B300100107000004E00003003200E2
:10FA70004100200021079800670037000040EB009C
:10FA800030479800190037001E4090000080FB00AE
:10FA90000000D10010479800BFFF0700004F78001A
:10FAA00020C0B3009E4F100003003A004100200028
:10FAB000210798005800370010C0B3009E4F100077
:10FAC00007003A009E40900000C8B30000C040000C
:10FAD000104798002E4090000004A2002047980094
:10FAE0003E4090000040E800304798003E409000C3
:10FAF000E74F5000E4FF3600302721009E40900081
:10FB000001487800A4FF0700004F780020C0B30030
:10FB10009E4F100003003A0041002000210798008A
:10FB20003D0037001E407800E14060004027210082
:10FB30001040780061C16000E1CFB3000140600077
:10FB400002407000412721008048780040272100B2
:10FB500010407800614060008080FB002E409000E3
:10FB60000080FB00808F500008003A0040272100F1
:10FB7000104078000020A000412721008048780034
:10FB80002100200021079800230037004027210092
:10FB9000104078000020A100412721008048780013
:10FBA0007DFF0700004F780020C0B3009E4F10007B
:10FBB00003003A004100200021079800160037009A
:10FBC0001E4078006141600040272100904078008D
:10FBD0006140610000414000D0CFB30080C06000B0
:10FBE00082C070004027210001487800C902A900A6
:10FBF0004027210010407800624060000004E000CF
:10FC000003003A003100200021079800020037006D
:10FC10000000EB00200798002E0090000080FA0002
:10FC2000000006000200FA0000C0EB00004F780060
:10FC3000C922A800C902A8000040EB0010479800A4
:10FC400011003700CBC2BF00614060000004E0003B
:10FC500007003A0069FF0700004F78001E04E0002B
:10FC60000C00320040C0B3009E4F1000090032006B
:10FC70005000200078970200000000001E40900015
:10FC80000040E800104798001E409000E14F4000FF
:10FC9000ECFF3A00C902A9001E80FB000080FA00B8
:10FCA000000006000400FA00004F780010C0B30006
:10FCB0007D0007000004E000030032002000200067
:10FCC00010079800130037009E40780061C0600064
:10FCD0006140600000414000912C2000914078007C
:10FCE000D0CFB30000C0600002407000C9E2B7008E
:10FCF0000040EB006C0007000004E000030032004D
:10FD00002000200010079800020037008000EB0060
:10FD1000110798001E0090000080FA000000060005
:10FD20000800FA00404798000040EB002047980088
:10FD3000C902A900CB02A900C003200078970200E5
:10FD400000000000CB22A900C922A900C902A80016
:10FD50001000200078970200000000000040EB0037
:10FD6000510007000004E0000300320040002000C2
:10FD700030079800490037000000EB00000F7800C2
:10FD80001C0037004E4090000080FB0061006000C6
:10FD90000004E0000B00320010C0B300C1FF0700F8
:10FDA0000004E0000300320040002000300798000B
:10FDB0003A0037002E4090000004A200204798002F
:10FDC000070037000040EB00B6FF07000004E0002A
:10FDD0000300320040002000300798002F00370059
:10FDE0004E4090000080FB000000D100404798008A
:10FDF0001E0FE800700020009E0F1000E1FF36008B
:10FE00002E4090000004A200204798002E40900051
:10FE1000A4FF07000004E0000300320040002000BF
:10FE2000300798001D003700C922A800CB22A90086
:10FE300010C0B3001C0007000004E0000300320003
:10FE4000400020003007980014003700D2FE070061
:10FE5000E24F500003003A004000200030079800B5
:10FE60000E003700CCFE07000080FB00000F78007A
:10FE7000200020009E0F100003003A0040002000E8
:10FE80003007980005003700C902A900CB02A9007D
:10FE90001E0078000080FB00300798003E009000B4
:10FEA0000080FA00000006000600FA0020479800D3
:10FEB0000080EB00000F7800CBC2BF006140600003
:10FEC0008080FB002E4090000080FB00808F50005F
:10FED00003003A000000EB002007980005003700FF
:10FEE0001E0FE9001E00E000F3FF3A0010002000A2
:10FEF000200798002E0090000080FA000000060005
:10FF00000400FA00004F780011479800C0DD20007F
:10FF10001E48780030C0B3009E4F100005003A0024
:10FF200000202000F06E880000082000006F88008C
:10FF30000400370000202000F06E88000020200020
:10FF4000006F88001E4090000080FB0010079800A2
:10FF50001E009000E10F5000110032001E009000C2
:10FF6000E20F5000180032001E0090000000E00078
:10FF7000010032001E00370041C1B30020DE200026
:10FF80000148780041C6B30030DE20000148780007
:10FF900021C3B30040DE2000014878001D00370077
:10FFA00021C0B30020DE200001487800A1C0B300CA
:10FFB00030DE20000148780051C0B30040DE200050
:10FFC000014878001300370011C0B30020DE200084
:10FFD0000148780051C0B30030DE200001487800AD
:10FFE00021C0B30040DE200001487800090037003E
:10FFF0008040EB0020DE2000014878008040EB00CC
:020000040001F9
:1000000030DE2000014878008040EB0040DE200018
:10001000014878000080FA00000006000200FA00A3
:100020000000EB00000F780030DE200090407800E8
:100030000030200009010700CBC2BF006140600012
:100040000004E00004003200CBC2BF006240600048
:100050000004E00002003A0010002000000F7800C9
:1000600030DE2000904078000020200017010700BB
:1000700030DE2000904078000010200013010700BF
:1000800030DE20009040780000202000F3000700C0
:100090001E0078000080FA00000006000000FA0050
:1000A00030DE20009040780000302000070107007B
:1000B00030DE20009040780000102000E7000700AC
:1000C00030DE20009040780000202000E300070090
:1000D0000000EB000080FA00000006000C00FA00AF
:1000E000500798000000EB00000F780070B7200068
:1000F000104078000080FB008000E9001000200024
:100100000100DD00300798005E0090002007980095
:100110000000EB00400798002000370020DE2000A0
:1001200010417800AE0090003E009000008060001A
:1001300001202000FC00070030DE20009040780005
:1001400000102000C500070000082000260107005D
:100150000080FB001007980030DE200090407800FF
:1001600000102000D90007002E0090000000400081
:10017000200798001E00780000004000000F780063
:100180001E0090000000E000010032001E0FE80099
:100190004E0090000000E8004007980070B7200073
:1001A000104078008080FB004E009000808F50004F
:1001B000DAFF3E001E0078000080FA000000060012
:1001C0000800FA003007980070B72000104078004F
:1001D0000080FB008000E900100020000100DD002D
:1001E000100798003E009000000F78000000EB0020
:1001F000200798001400370020DE2000104178000E
:100200001E0090001E00600001202000C6000700B4
:1002100030DE200090407800001020008F000700A2
:1002200030DE20009040780000102000A70007007A
:100230001E00780000004000000F78002E009000A3
:100240000000E8002007980070B7200010407800F8
:100250008080FB002E009000808F5000E6FF3E0063
:100260000080FA00000006000600FA000000EB0023
:10027000000F780000202000DB0007000000EB00EA
:10028000200798001600370030DE200090407800EC
:10029000001020007100070000202000D20007009D
:1002A0000080FB001007980030DE200090407800AE
:1002B00000102000850007001E00780000004000AC
:1002C000000F78001E0090000000E00001003200E6
:1002D0001E0FE8002E0090000000E80020079800A4
:1002E00070B72000104078008080FB002E00900046
:1002F000808F5000E4FF3E001E0078000080FA006E
:10030000000006000200FA00006F8000B60007003F
:1003100030DE200090407800001020004F000700E1
:10032000006F8000B0000700004F780030DE200032
:100330009040780000102000640007001E80FB0041
:100340000080FA00000006000200FA00004F78006A
:1003500020DE200010417800F16E80001E80FB003E
:100360007100070030DE200090407800001020006F
:100370003A00070030DE2000904078000010200096
:10038000520007000080FA00000006000400FA0096
:10039000204798000040EB00004F7800090037002C
:1003A00030DE200090407800001020002B00070075
:1003B00030DE20009040780000102000430007004D
:1003C0001E4FE8002E4090009E4F1000F4FF3900B1
:1003D0000080FA00000006000200FA00004F7800DA
:1003E00020DE200010417800F16E80001E80FB00AE
:1003F0004D0007000080FA00000006000200FA002D
:10040000004F780020DE2000104178001E80FB00A5
:1004100001102000440007000080FA0000000600E0
:100420000200FA00004F780020DE20001041780022
:100430001E80FB00010420003B0007000080FA0042
:10044000000006000000FA00006F80006600070050
:100450000080FB000080FA00000006000400FA00A3
:10046000000F78002147980080B8200010407800E5
:10047000684060000004E0000B003A006016800055
:100480001E007000601688001E0078000080EA00E0
:100490008180EA00800078004016800000806000C3
:1004A0004016880003003700401680001E007000D0
:1004B000401688002E4090000080FB0078970200D4
:1004C000000000000080FA00000006000400FA00AE
:1004D000000F7800214798001E0078000080EA0095
:1004E0008180EA0080007800601680000080600053
:1004F000601688001E0078000080EA008180EA0013
:10050000800078004016800000806000401688005F
:100510002E4090000080FB00789702000000000051
:100520000080FA00000006000600FA00000F7800C4
:1005300011079800424798001E00E0000F003A00A3
:100540001E0090000080EA008180EA0080007800B0
:100550006016800000806000601688001E00900019
:100560000080EA008180EA00800078004016800068
:1005700000806000401688001500370080B8200019
:1005800010407800684060000004E0000C003A0071
:10059000611680001E0090000080700060168800C8
:1005A0001E0090000080EA008180EA008000780050
:1005B000401680000080600040168800040037006C
:1005C000401680009E0090000100700040168800D8
:1005D0004E4090000080FB00789702000000000071
:1005E0000080FA00000006000400FA00000F780006
:1005F000401680001E0070004016880000000000B9
:100600000000000000000000501680001E00600086
:100610000000E000030032001000200010079800E6
:10062000020037000000EB00100798001E00900049
:100630000080FA00000006000000FA003481020089
:10064000000000000080FA00000006000200FA002E
:10065000000F78001E007800E0800200000000001B
:10066000001020000080FA00000006000000FA00E0
:100670000E8002000000000081002000D0922000C7
:10068000EE99020000000000D1002000804420000C
:10069000789A0200000000000080FA0000000600C6
:1006A0000000FA004E8002000000000061002000FF
:1006B00050932000EE99020000000000C1002000CD
:1006C00050452000789A0200000000000080FA00E7
:1006D000000006000000FA00828102000000000015
:1006E0000080FB000080FA00000006000000FA0015
:1006F00022820200000000000080FB000080FA005F
:10070000000006000000FA000040EB00FE8102003D
:10071000000000000080FA00000006000000FA005F
:1007200010C0B300FE810200000000000080FA004B
:10073000000006000000FA0010C0B300C6810200ED
:10074000000000000080FA00000006000000FA002F
:100750000040EB00EC810200000000000080FA0085
:10076000000006000000FA0010C0B300EC81020097
:10077000000000000080FA00000006000000FA00FF
:1007800001012000A0982000EE9902000000000066
:1007900060B72000104078006E6F0200000000007B
:1007A00000C2B300327102000000000080B82000D7
:1007B000104078000080FB004300DE0061406000D4
:1007C0006E6F02000000000000C2B3003271020030
:1007D0000000000031002000F0AD2000EE99020082
:1007E000000000000080FA00000006000400FA008B
:1007F0002C1A020000000000561602000000000043
:10080000100798002C1A0200000000005616020083
:1008100000000000000F78001E0090000000E000C3
:10082000090034001E009000E40F500006003C0058
:100830001E0090000040E9008040780060B7200072
:1008400001487800020037000000EB001007980014
:100850001E00E00010003400200020009E0F100059
:100860000D003C001E0078000040EA00614160007D
:1008700080B8200090407800614061004301DD00B5
:1008800070CFB30080C0600082C0700080B82000CC
:1008900001487800020037000000EB0010079800C4
:1008A0001E0090000000E00026003A000000EB006F
:1008B00060698800B103200060482000789A020037
:1008C000000000008001EB00420020001100200029
:1008D00010002000A21C0200000000000040E900FF
:1008E0008040780060B7200001487800F1042000C3
:1008F000B0932000789A0200000000008001EB0015
:10090000220020001100200010002000A21C020084
:10091000000000000040EA006141600080B8200053
:1009200090407800614061004301DD0070CFB3006A
:1009300080C0600082C0700080B82000014878004C
:10094000010037008DFF0700CB02A900CB22A900D0
:10095000C922A800C902A90060B720009040780011
:1009600020C0B300807F0200000000000080FA0079
:10097000000006000400FA00000F78001E00780056
:10098000100798001E009000E10F50000C0032008C
:100990001E009000E10F5000040039001E0090007E
:1009A000E20F5000070032000800370081032000EA
:1009B000A0992000EE990200000000000700370017
:1009C0001000070025000700040037004102200046
:1009D000C0202000789A0200000000000080FA0089
:1009E000000006000200FA00000F7800B1002000AD
:1009F000C0092100789A0200000000000080FA007F
:100A0000000006000000FA00F1032000209D2000F5
:100A1000789A0200000000000040EB001082020003
:100A200000000000F00F2000789702000000000096
:100A300010C0B300108202000000000010C0B3001C
:100A4000C6810200000000000040EB00108202009E
:100A5000000000000080FA00000006000A00FA0012
:100A6000881F7800D102200010A12000EE9902001A
:100A7000000000000000EB00000F780010003700BD
:100A80001E047800348102000000000080407800DD
:100A900063004700017478009E00780063004700FF
:100AA000614078000080FB00D06F02000000000071
:100AB00000C2B30032710200000000001E0FE80007
:100AC000300020009E0F1000EDFF3600A0A528008A
:100AD000026D020000000000A1002000E0A3200041
:100AE000EE9902000000000063004700104078000B
:100AF0000080FB004400DE000080FB0040079800FF
:100B00004E009000E90F5000130032004E0090009C
:100B1000E90F500004003C004E009000E80F500028
:100B2000080032001B0037004E009000EA0F500012
:100B30000E0032004E009000EF0F50001000320007
:100B4000140037006100200080A42000EE9902000C
:100B5000000000001300370061002000E0A4200026
:100B6000EE990200000000000E0037006100200036
:100B700040A52000EE9902000000000009003700A7
:100B800031002000A0A52000EE9902000000000026
:100B90000400370071002000D0A52000EE9902006B
:100BA00000000000A0A52800026D02000000000067
:100BB000B100200040A62000EE99020000000000D5
:100BC00063004700104090000080FB004700DE00FB
:100BD0000004E00005003A0061002000F0A62000BB
:100BE000EE9902000000000004003700F100200030
:100BF00050A72000EE99020000000000A0A52800E8
:100C0000026D020000000000C100200040A820008A
:100C1000EE990200000000006300470010409000C1
:100C20008080FB0080F72F00008060004380DE00A2
:100C3000204798002E4090000004E00005003A0094
:100C4000D100200000A92000EE9902000000000061
:100C50001E0037002E409000EF4F500005003A0074
:100C600031002000A0A52000EE9902000000000045
:100C70001600370000042000000F7800E300470052
:100C80000040EB0080487800080037001E00780024
:100C900000004000000F780063004700104078001B
:100CA0008040E80063004700014878006300470087
:100CB000904078002E40900080CF5000F3FF390024
:100CC0001E007800106F020000000000A0A52800A0
:100CD000026D02000000000091012000D0A9200058
:100CE000EE99020000000000630047009040900071
:100CF00070C0B30000C060002047980010002000C2
:100D0000000F7800E30047000040EB0080487800C7
:100D1000080037001E00780000004000000F780037
:100D200063004700104078008040E80063004700FF
:100D30000148780063004700904078002E40900002
:100D400080CF5000F3FF39001E0078006E6F020064
:100D500000000000A0A52800026D020000000000B5
:100D60004F0478000080FA00000006000000FA003E
:100D700040168000017C20000100700040168800B1
:100D80001100070020C0B3002D00070014710200FD
:100D9000000000000004E0000500320020710200A5
:100DA00000000000260007000004E00004003A00F4
:100DB000360107000004E00001003A00F3FF3700AD
:100DC0000080FA00000006000000FA00CA82A900B4
:100DD0000000EB00400388000000EB005003880097
:100DE0000000EB00000388000000EB001003880007
:100DF0000000EB00F0088800D10A20009140780044
:100E0000F0C8B30000C06000ADE0B7000000EB0028
:100E1000E008880000642000D0088800000021005D
:100E2000307088008040EB0040E0200001487800EE
:100E30000000EB00906F88000080FA0000000600C0
:100E40000A00FA00004F7800E06F80004007980029
:100E5000CE009000E18F5000440032004E0190001F
:100E6000E10F5100040039004E009000E20F5000E5
:100E70004F003200000137009E80FB0031079800D0
:100E80003E019000E20F5100150032003E0090003C
:100E9000E20F500007003C00BE0090000100E0009F
:100EA0000B0032003E019000E10F510010003200B3
:100EB000230037003E009000F10F5000EE0032009A
:100EC000BE009000F38F5000EB0032001C00370092
:100ED000BDFF07001200200022079800E80037003D
:100EE000C0A42800D66C020000000000E200370019
:100EF000CA82A8000000EB00F00888000000EB00A8
:100F0000B00888000000EB00A008880080002000E6
:100F1000F00888008660A9009660A900D10A200028
:100F200091407800F0C8B30000C060000044A00009
:100F3000ADE0B70010002000906F8800CE003700B1
:100F400040DF20001E48780041C0B30090DF200041
:100F5000014878008040EB00A0DF200001487800C5
:100F600010002000E06F8800C3003700A0DF2000E1
:100F7000104078008040E800A0DF200001487800A1
:100F8000A0DF2000104078008080FB0040DF2000C0
:100F9000008040001E487800A0DF200090407800CC
:100FA00090DF20001040780080CF5000B200390060
:100FB00040DF2000104078000080FB001007980000
:100FC000100820009E009000808F50003E003200EC
:100FD000000C20001E019000800F5100050032001F
:100FE000000820009E009000808F50004E003200CC
:100FF0009F00370050DF2000104078000080FB0089
:101000004400DE00610060000004E00003003200E4
:10101000100380000000A0001003880050DF2000B3
:10102000104078000080FB004300DE00610060009B
:101030000004E000040032001003800001022000E0
:10104000010070001003880050DF2000104078007D
:101050000080FB004200DE00610060000004E00050
:101060000400320010038000010420000100700021
:101070001003880050DF2000104078000080FB0043
:101080000000D100610060000004E00004003200B4
:101090001003800001082000010070001003880088
:1010A00050DF2000104078000080FB0061006000ED
:1010B0000004E00004003200100380000110200052
:1010C000010070001003880060DF200010407800ED
:1010D0000080FB0030708800307080004800DD0028
:1010E0003070880050DF2000104078008080FB00C6
:1010F0003070800000807000307088003070800098
:101100004200DD00640040003070880031708000D3
:1011100000002100808F50005500360000002100A3
:10112000307088005200370070DF200010407800D7
:101130000080FB0001002000F06F88000170880033
:10114000F06F800001708000C808DD000080FD00A5
:10115000804078000040EB00F06F8800017088004C
:1011600060DF2000104078000081FB0003002000B9
:10117000F06F8000017080000000710081807100BC
:10118000F06F880001708800F06F800001708000AF
:10119000C808DD000080FD00804078000040EB00C2
:1011A000F06F88000170880050DF20001040780048
:1011B0000081FB0003002000F06F800001708000C0
:1011C0000000710081807100F06F8800017088005C
:1011D000F06F8000017080004209DD00CE00DE006B
:1011E000810071004200DD0064004000E0804800A2
:1011F00092012000030020003006020000000000E1
:10120000F06F880001708800F26F8000037080002A
:101210000001200001002000800F5100818F590043
:1012200007003600F06F80000170800070005000F1
:10123000E0805800F06F88000170880004003700DB
:101240001000200001002000F06F8800017088006D
:10125000F06F8000017080004008DE000100200077
:10126000E0088800F06F800001708000D0088800DE
:101270000000EB00E06F88000000EB002007980002
:101280002E0090000080FA00000006000200FA0024
:10129000906F8000E10F50000100320036003700EF
:1012A00086C0BF00684060000004E00003003A0010
:1012B000100380000000E0002F003A001FE1A800AA
:1012C0008780A9000000EB00107088000E00370036
:1012D00071408000107080008080400050168000B7
:1012E0004600DE008048780087C0BF007040600084
:1012F0000004E000FCFF32008780A900107080002D
:101300000000E800107088001170800030708000CC
:10131000808F5000EEFF39000000EB0010038800C2
:101320000000EB00F008880030708000107088002A
:101330000A0037007140800010708000008040007B
:101340000000E90010407800327102000000000047
:10135000107080000000E90010708800107080009C
:101360000000E000F3FF3A0097FE070010002000A5
:10137000000F7800020037000000EB00000F78003B
:101380001E0078000080FA00000006000200FA004B
:10139000000F78001E0078008040780000272100B0
:1013A000104078000080FB000000D1006140600028
:1013B00046010700001020000080FA00000006002F
:1013C0000000FA0000272100104078000010A10062
:1013D000012721008048780041012000B0EC200066
:1013E000789A0200000000000080FA000000060069
:1013F0000000FA0000272100104078000010A00033
:10140000012721008048780021012000F0ED200014
:10141000789A0200000000000080FA000000060038
:101420000000FA0080B82000104078000030A000D2
:1014300081B8200080487800002721001040780003
:101440000010A0000127210080487800816A200058
:101450009140780000CEB30000C060007040B3003F
:10146000A8E6B700916C20009140780000CEB30050
:1014700000C060007040B300C9E6B700816C200076
:101480009140780000CEB30000C060000034A0009E
:10149000C8E6B700CAC2A900C8C2A900C902A9000B
:1014A000C8E2A800C922A900D013200010128800A9
:1014B0000000EB00201288000000EB000012880002
:1014C00041E2A800D101200040F02000789A0200FB
:1014D000000000000080FA00000006000800FA008A
:1014E00020079800506980000000E80050698800DB
:1014F00051698000F00F2000008060005069880072
:101500002C1A020000000000561602000000000025
:10151000100798000000EB00606988002E00900022
:10152000300798003E009000E30F50003C0032006E
:101530003E009000E30F500004003E003E0090008B
:101540000000E0000B0032000F0037003E0090006A
:10155000E60F5000480032003E009000E70F5000B8
:101560006A0032003E009000E40F50003700320065
:101570008B0037008109200060F62000789A020075
:10158000000000008A003700510020003063200076
:10159000789A020000000000AC0007002E009000C6
:1015A000E10F5000820032001E0090000000E000B9
:1015B000030034001E009000E20F500013003400BE
:1015C00041022000E0FF2000789A020000000000A5
:1015D0008001EB00220020001100200020002000EC
:1015E000A21C020000000000100798001E009000DE
:1015F000E10F500003003A000040EB0075000700C7
:101600000200370080C0B3007200070041002000D4
:1016100020022100789A02000000000064003700D8
:1016200011C0B3000040EB00A8000700F00020004C
:101630004C970200000000005100200060022100D1
:10164000789A020000000000590037001E00900048
:101650008040780000C8B30080C070000040EB00FC
:101660009A000700A1002000B0022100789A020031
:10167000000000004E00370011C0B3000040EB0036
:1016800092000700F00020004C97020000000000CC
:1016900000032000200798001E0090000000E000DA
:1016A00002003A0000052000100798000000EB003F
:1016B000000F780011003700AE009000900320006A
:1016C000808F5000020036000003200020079800A1
:1016D0002E0090008040780010C0B3007B0007000F
:1016E0002E00900032710200000000002E009000D9
:1016F0000000E800200798001E0FE8001E00900080
:101700009E0F1000ECFF35002900370011C0B30018
:101710000040EB006D000700F00020004C97020035
:101720000000000010022000200798001E0090001A
:101730000000E00002003A000005200010079800B9
:101740000000EB00000F780011003700AE009000A1
:10175000F0072000808F50000200360010022000A9
:10176000200798002E0090008040780010C0B30041
:10177000560007002E0090003271020000000000A9
:101780002E0090000000E800200798001E0FE800DF
:101790001E0090009E0F1000ECFF35000400370083
:1017A00041022000C0202000789A020000000000C2
:1017B0000080FA00000006000000FA00B1002000DE
:1017C000C0092100789A0200000000000080FA00A1
:1017D000000006000200FA00004F78001E4078006A
:1017E0000042B000804078000040EB003700070066
:1017F000F00020004C9702000000000081C0B30000
:101800000040EB0031000700F00020004C97020080
:101810000000000011C0B3000040EB002B000700E7
:10182000F00020004C97020000000000E1C0B3006F
:101830000040EB0025000700F00020004C9702005C
:10184000000000000080FA00000006000000FA001E
:101850000040EB004A000700F00020004C97020017
:101860000000000031C0B3000040EB00260007007C
:10187000500020004C9702000000000031C0B3006F
:101880000040EB0020000700000A200078970200CB
:101890000000000031C0B3000040EB001A00070058
:1018A000000A2000789702000000000021C0B30069
:1018B0000040EB0014000700000A200078970200A7
:1018C000000000000080FA00000006000200FA009C
:1018D000004F7800114798001E4090000080FB00E8
:1018E0004400DE00804078001E40780006000700BB
:1018F0001E409000EF4060001E407800020007008C
:101900000080FA00000006000200FA00004F780094
:10191000114798001E4090004400DD0010479800D9
:101920001E4090000004A0001047980010C0B300B3
:101930009E4F100003003A001E4090000014A000CB
:10194000104798001E4090000D0007001E409000B8
:101950000034A000104798001E40900008000700C7
:101960009E40900070CFB30000C060001047980008
:101970001E409000020007000080FA0000000600F0
:101980000200FA00004F78001E4078001C47020059
:1019900000000000CAC2A800CAC2A9000080FA0064
:1019A000000006000000FA0020A52800D66C020006
:1019B000000000000080FA00000006000A00FA00A3
:1019C000704080003007980010002000B09388001D
:1019D000F4FF070000003700207102000000000043
:1019E000104798001E4090000080FB0040079800C0
:1019F000CE009000E38F5000200032004E00900097
:101A0000E30F50000A003C00CE009000E18F500030
:101A10005B0032004E009000E10F50005E003C0081
:101A2000CE0090000100E000E7003200DB0037004C
:101A30004E009000E60F50000E003200CE009000E5
:101A4000E68F500004003C004E009000E50F50006F
:101A500095003200D1003700CE009000E78F500093
:101A6000640032004E009000E80F50005400320035
:101A7000CA003700CBFF0700D7FF3700BE00900039
:101A800030C0B300804878003E0090008000E8003D
:101A900080C0B3008048780021E3A800C0C0B30034
:101AA0000E96020000000000200798003E00900003
:101AB0008080E8002E0090004800DE00804878001A
:101AC0003E009000E30040002E0090008048780027
:101AD000B0C0B3000E96020000000000200798007E
:101AE0003E009000E40040002E0090004800DE0020
:101AF000804878003E009000E50040002E009000F5
:101B000080487800A0C0B3000E96020000000000DC
:101B1000200798003E009000E60040002E00900054
:101B20004800DE00804878003E009000E70040005A
:101B30002E0090008048780090C0B3000E960200FE
:101B400000000000200798003E009000E8004000E0
:101B50002E0090004800DE00804878003E00900093
:101B6000E90040002E0090008048780021E3A900A1
:101B7000A10020003E009000BA00070096FF370049
:101B80002071020000000000104798001E409000E5
:101B90008F00070090FF3700207102000000000056
:101BA000104798002071020000000000004F7800EC
:101BB0009E4078001E409000BC00070086FF370062
:101BC0002071020000000000104798002071020000
:101BD00000000000004F78001E4090000080FB00D5
:101BE000C800DD001E80FB0000807000B0938800FC
:101BF00079FF3700207102000000000010479800B4
:101C00001E4090000080FB00200798001E409000BE
:101C1000E14F500004003A0030C0B30050710200A0
:101C2000000000000300370020C2B3005071020022
:101C30000000000020710200000000001047980022
:101C40002071020000000000004F78009E409000CC
:101C5000A0CAB30080CF500003003A0050C5B300C3
:101C60009E4F1000050032000000EB002007980096
:101C700020C2B3005071020000000000BE009000BE
:101C800070C0B300804878003E0090008000E800FB
:101C90002E00900080487800210020003E00900037
:101CA000700007004CFF37002071020000000000A8
:101CB000104798002071020000000000004F7800DB
:101CC0008560A9001E4090000080FB00C800DD0078
:101CD0001E80FB0000807000100798009E0090009E
:101CE00000002200808F5000020036000000220019
:101CF000100798001E009000670040004300DE00BF
:101D000020079800BE00900050C0B30080487800C3
:101D10003E0090000000E8009E40900001487800DE
:101D20003E0090000080E8001E487800310020004E
:101D30003E0090004B00070070408000004088008B
:101D40002E00900000004000104088000000EB00D2
:101D500020408800714080004083200000804000C7
:101D6000304088000000EB00404088000000EB009D
:101D7000504088009560A800B093800031408000FA
:101D800004408000800178001E019000040078006B
:101D90005A9D0200000000000FFF3700BE009000B7
:101DA0000040EB00804878003E0090008000E80092
:101DB0000040EB0080487800110020003E009000B9
:101DC0002800070004FF37000080FA00000006002A
:101DD0000200FA00004F7800CAC2A900CB22A90075
:101DE000CB02A900CB42A90020C0B3009E4F100037
:101DF00005003A00CAC2A800CB02A800CB22A80066
:101E0000CB42A80004003700CAC2A900CB02A90037
:101E1000CB22A900CB42A90010C0B3009E4F1000F6
:101E20000300320020C0B3009E4F100006003A00AD
:101E3000C8C2A900C922A900C902A900C942A900B3
:101E4000C8E2A80005003700C8C2A800C922A8003F
:101E5000C902A800C942A800C8E2A8000080FA0090
:101E6000000006000600FA001007980021079800FD
:101E70000000EB00000F7800070037009E0078009C
